:1000000000400020A5870000E5870000E78700008A
:1000100000000000000000000000000000000000E0
:10002000000000000000000000000000E987000060
:100030000000000000000000EB870000ED870000DA
:10004000EF8700001D600000518B0000EF8700006B
:10005000EF87000000000000EF870000EF8700003E
:10006000293D0000258F0000EF870000EF8700008A
:10007000EF870000EF870000EF870000EF870000A8
:10008000EF870000D58B0000EF870000EF870000AE
:10009000EF870000EF870000EF870000EF87000088
:1000A000EF870000EF870000000000000000000064
:1000B0000000000000000000000000000000000040
:1000C00010B5064C2378002B07D1054B002B02D02E
:1000D000044800E000BF0123237010BD700200201F
:1000E000000000002CFE0000044B10B5002B03D0D4
:1000F0000349044800E000BF10BDC04600000000F6
:10010000740200202CFE0000164B002B00D1144B73
:100110009D46402292029A1A924600218B460F4633
:100120001348144A121A0CF03BFD0F4B002B00D061
:1001300098470E4B002B00D0984700200021040068
:100140000D000D48002802D00C4800E000BF0CF064
:10015000E7FC2000290008F04DFD0CF0BBFCC04678
:100160000000080000400020000000000000000027
:1001700070020020F42F00200000000000000000AA
:1001800002000120104011D1042A0ED91368180969
:1001900080B2002809D001388000031D11180979A8
:1001A000002902D001309842F8D170470020FCE7C6
:1001B0000378002B03D05AB2002A01DB01307047CC
:1001C0003F229343C03B59424B41C01803789343AD
:1001D000802BF4D10130F9E710B500240378002B0F
:1001E00001D1200010BDFFF7E3FF0134F6E770B541
:1001F000002204000D00411C092004F0BDF8002875
:1002000006D001236200134343600023A34200DBB6
:1002100070BD9A00A958821891600133F6E770B555
:10022000012803DC1C2001F0BBFA70BD01230D681E
:1002300011201D42F7D04868184206D1042804D97D
:100240000F2302681340042B01D00E20EBE703F0CC
:10025000F1FE6D100400002D03DDFFF7BDFFA84285
:1002600006DA1220DFE72000FFF7A2FF0400013DBD
:10027000012DF8D120787F2809DDDF280BDCF82359
:100280003F22DB00800118406378134018430123AC
:1002900040001843C9E7EF280BDCFC226378120109
:1002A0009B0113403F220007000C0343A07810403D
:1002B000ECE7F72812DCFC22637892021B03134060
:1002C000E0228004520310403F221843E378134099
:1002D000FC220343A07812018001E8E7012040429C
:1002E000D5E7F8B54D680F00EB0706D4042D04D907
:1002F0000F232E683340092B03D00B2001F050FA56
:10030000F8BD6B683609B6B25C10731EA3420FD8F5
:10031000032120000AF000FB6421642803DC0100B3
:10032000032800DA03212800891904F057F8050092
:100330002B6800201B099BB2013B9C42E0D23A682B
:10034000A31C9B005A510123013464001C436C60C0
:10035000D6E7F0B585B0012803DC1C2001F020FAB7
:1003600012E001274B683A000093022806D08B6800
:100370003B4203D05F10002F00DC17000125009BDB
:100380002B4203D00120404205B0F0BD009B042B5E
:10039000F8D91B680C680F261900314004292DD1AB
:1003A0002C4205D1042C03D923681E40042E01D011
:1003B0000E20D3E70098FFF7E3FEB842E2DB009897
:1003C00003F038FE0600200003F034FE037801003D
:1003D000002BD7D0781E30180CF098FF041ED1D017
:1003E0003378002B01D0A64202D36800012521E01A
:1003F0003000FFF7DDFE01350600F1E709293ED1A7
:10040000009B5B685B1001939F42BBDC2C422ED1AA
:10041000042C2CD923683340042B28D1200003F06E
:1004200009FE039602907E1C009AB300D0588442C5
:1004300002D178002843A7E728420ED104280CD91E
:100440000368039A1340042B07D103F0F3FD010066
:1004500002980CF025FF0028EBD0019B37009E424C
:10046000E1DD8FE71F00019B9F4200DD8AE77B1CD7
:1004700000999A008A58A242F4D17800B6E703297D
:1004800000D07FE71A0992B25B0F92000B40D31A9B
:1004900001939F4200DD75E72C4229D1042C27D916
:1004A00022681640032E19D1100980B2520F800025
:1004B0003240251D801A019B2E181B1A0193009BA8
:1004C000781E0433019A904200DD5BE72A00191878
:1004D000B2420FD316D10130400087E7042E07D176
:1004E000200003F0A7FD05002000FFF749FEE2E72A
:1004F0000F2033E70C78A4461478A44502D10131CB
:100500000132E5E70130DDE7F0B50D0085B00128E7
:1005100004DC1C2001F044F905B0F0BD0127086897
:10052000384206D1042804D90F2102680A40042A5F
:1005300001D00E20EEE76A681740FAD1042AF8D9F4
:1005400013680B40042BF4D103F074FD04006868B9
:1005500003F070FD02900CF0ADFE039000280FD167
:100560002000FFF739FE0190019B0122591C092050
:1005700003F002FF364E3060002815D10020CBE793
:10058000029920000CF0C2FE001B434243412000B0
:100590000193019B5E1C0028E6D0039B0299C018C2
:1005A0000CF0B4FE0196F4E70122019B5B001343BB
:1005B0004360039B002B18D12000FFF7F9FD019B3E
:1005C0000500BB4201DC3068A6E7291B200003F0D0
:1005D00051FF0028D2D0BB1C32689B0098502800E5
:1005E000FFF7E6FD01372C00E9E7019B012B02D163
:1005F0002B68836090E7029920000CF087FE0125AC
:100600000700019B002F13D0AB42DCDB391B20001D
:1006100003F030FF0028B1D032680135AB009850AC
:10062000039B0299FC1820000CF070FE0700E8E71D
:10063000AB42C8DB20000CF03DFE0100200003F0BF
:1006400019FF00289AD001353368AD00E850BAE7A9
:100650000410002010B503F0D1FC43000120184322
:1006600010BD0000C30711D404280FD90F2302685E
:100670001340032B0AD119400133591AC0234907EB
:10068000DB051940024B1A40114301607047C04618
:10069000FFFFFF9F70B5002805DC1C2001F080F8EB
:1006A0000500280070BD01220C68144201D10D2004
:1006B000F4E701281CD04B681342F8D05B101320DC
:1006C000FF2BEBD81A0619040A431A431B021343E3
:1006D0006410E243D2171440E11C89101A00032071
:1006E00003F04AFE051EDCD02100FFF7BBFFD8E770
:1006F0000023EDE7F7B507000E001C20012F06DDF3
:100700004C68012322001A40009203D10D2001F011
:1007100047F853E0022F02D08A681A42F6D001232C
:1007200035681D4200D0A9E0042D00D8A6E01C4188
:10073000002C00DC1C000F2029680840092828D163
:100740006B685B100093022F05D0B368009A5B10B2
:100750009A4200DD0093009B01221D1B0135EB43F3
:10076000DB171D40691C092003F006FE071E09D097
:1007700001236D001D430300326808334560009972
:10078000A14201DA3800FEBD0134A100515802C374
:10079000F5E7042845D1280003F04CFCFFF71CFDC9
:1007A0000190022F04D0B3685B10984200DD0193E2
:1007B000019BA34204DA002003F050FE0700E1E7AA
:1007C000280003F037FC0700009BA34221DB280030
:1007D000009703F02FFC05003800FFF7E9FC019BB0
:1007E00001340700A342F7DA009BC41A200003F08B
:1007F00035FE071EC6D003F01DFC0190306803F0E3
:1008000019FC2200009B591B411801980CF0ACF90F
:10081000B8E73800FFF7CCFC009B070001330093DA
:10082000D2E703282AD10B099BB2490F9B00014054
:10083000591A022F04D0B2685210914200DD110003
:10084000A14205DA00220320110003F095FDB5E76F
:1008500003200E1B331DD9170140C918891000222F
:1008600003F08AFD071E00D18CE701363100033406
:10087000FFF7F8FE381D29193200C7E7212046E7A7
:10088000F7B5002804DC1C2000F08AFF040014E007
:100890000D6801272E003E4011D03D41FF2D01D9AA
:1008A0001320F1E700223900032003F065FD041E48
:1008B00003D03900FFF7D6FE25712000FEBD042DC0
:1008C000EED90F232A681340042B1BD12800FFF711
:1008D00057FCC31C07000320D9170140C918891011
:1008E000320003F049FD041EE7D03900FFF7BAFEDD
:1008F000280003F09FFB231D01003A0018000CF0B4
:1009000033F9DAE7092B1FD103206B6832005B1043
:1009100001930333D9170140C918891003F02CFD46
:10092000041ECAD00199FFF79DFE019B9E42C4DAC6
:10093000B300EB189B683B4204D05B10FF2BAFD891
:10094000A21913710136F0E7032BA9D12C00B4E7EB
:1009500010B57F2902DC0170013010BD1A4B99429D
:100960000CDC40238A115B42134303703F230B408E
:1009700080214942194341700230EEE7134B9942FE
:1009800010DC20230A135B4213433F2480220370B0
:100990008B1152422340214013430A43437082701B
:1009A0000330DAE70A4B9942D7DCF0230370603B4F
:1009B0004370113B8A11FF3B1A4382703F22114062
:1009C0001943C1700430C8E7FF070000FFFF0000B3
:1009D000FF0F010010B50124044002D04410200094
:1009E00010BD042810D90F2302681340042B07D12F
:1009F00003F020FB21000A220CF024FD0400EEE7A6
:100A0000032B01D10430F5E70D2000F0C9FEE6E725
:100A1000F0B50E0085B0002803DC1C2000F0C0FEFD
:100A200017E00F6801243D00254006D1042F1ED990
:100A30000F233A681340042B0DD13800FFF7CAFF8B
:100A400002AC01002000FFF783FF011B200003F030
:100A500011FD040032E0092B09D17B685B10019382
:100A6000019B9C4205DD00F0A1FE002819D02A2040
:100A7000D4E70134A300F858FFF7ACFF01237F2827
:100A80000DDD154ADB18904209DD144A013390420E
:100A900005DD0021124AC30F82424B419B00ED1835
:100AA000DEE7280003F0DAFC041E07D0376803F005
:100AB000C1FA01250600019B9D4202DD200005B020
:100AC000F0BD0135AB00F858FFF784FF010030009E
:100AD000FFF73EFF0600EEE7FF070000FFFF000004
:100AE000FF0F0100F7B5030001900E001C20012B41
:100AF00011DD0868FFF76EFF07007068FFF76AFFF7
:100B0000019B05000124022B08D0B068FFF762FFAB
:100B1000041E03DC292000F043FEFEBDAF421CDCB6
:100B2000E81B210009F0F8FE451C691C0022092081
:100B300003F022FC0028F0D001226B001343436035
:100B40009440002379009D42E7DD17009E000F438B
:100B50008619B76001330919F5E7781B210009F000
:100B6000DBFE6442451CE0E710B5040001200840AC
:100B700010D104290DD90F230A681340042B08D182
:100B8000080003F057FA010020000CF089FB4342F3
:100B9000584110BD0020FCE7F7B50E00012803DC2A
:100BA0001C2000F0FDFDFEBD4D68EB0706D4042DB2
:100BB00004D90F222B681A40092A01D00B20F0E734
:100BC0006A681B099BB25410A34200D85C1E01271F
:100BD00031680F404810002F35D12648FFF7C4FF79
:100BE00001230190002813D131682348FFF7BCFF8F
:100BF000002811D0002C0DD00122631C013C944030
:100C00009B005A5114436C6004E00137BA00AB50AA
:100C1000BC42FADA0020C6E701233068184223D12B
:100C2000042821D902680E331340042B1CD1FFF78E
:100C3000D1FE002807D131681048FFF795FF002842
:100C400012D01220ADE70028FBDD8442F9DB8300DF
:100C5000EB180433844209DC0123621C013C9C40F4
:100C6000920053511C43CEE711209AE75A68013095
:100C70001A60EEE74BE200004FE2000054E2000091
:100C8000002310B50C000B70C30705D50D494210A9
:100C900020000CF0C9FA08E00B49002802D0042813
:100CA00004D10A4920000CF0DFFA10BD0428FCD959
:100CB0000F2302681340042BF7D103F0BBF904495A
:100CC0000200E5E7D8EE000056E200005CE200001A
:100CD00061E20000F0B593B0060002911C20012EE5
:100CE0001DDD029B01251B681C002C4000D0ADE0DF
:100CF000042B00D8E6E01A680F231A40092A4AD1CB
:100D00000394039A029992008A5817002F4005D144
:100D1000042A03D910681840092806D0222000F0C0
:100D20003FFD0190019813B0F0BD52685210A41815
:100D3000039A013203929642E3D1611C012203F02F
:100D40001BFB0190002802D100230193EAE7019BDD
:100D50006400190025435D600831029ABB00D05839
:100D600002684368120992B25B109A4200D8531E7F
:100D70000022934209DCDA43D21713409B00C918C2
:100D8000039B01379F42E8DBCCE794000519AD686F
:100D900001320D51EDE72700032A59D10193029A40
:100DA000BB00D3582B42B9D1042BB7D9186801998D
:100DB0000140032939D1020992B2430F92000B403E
:100DC000D31A1C190137BE42E9D10320E31CD917FD
:100DD0000140C9188910002203F0CEFA01900028C2
:100DE000B2D000252100FFF73DFC019B1E1D029A99
:100DF000AB00D45801231C421FD1042C1DD90F2154
:100E000023681940032918D1180980B25B0F8000AC
:100E10000B40C01A0023834213DBC343DB17184087
:100E200001353618BD42E2DB7CE7042900D075E7C6
:100E30001800FFF7A5F92418C4E72000FFF7A0F970
:100E4000E8E7E2181279F2540133E4E700273C00A6
:100E50000F25029ABB00D3580122134234D1042B30
:100E600032D9186801002940042935D11800FFF74C
:100E700087F924180137BE42EBD1200003F0EEFAC7
:100E80000190002800D15FE7029FB600BB19041D46
:100E9000029301233D681D4229D1042D27D90F2635
:100EA0002B681E40042E37D12800FFF769F9060091
:100EB000280003F0BFF80100200032000BF054FEC0
:100EC000A41922E02700C3E7180005A9FFF7D8FE00
:100ED00005A80CF0EFF9CCE7032900D01EE70209C2
:100EE00092B2430F92000B40D31A1C19C2E705A916
:100EF0002800FFF7C5FE05A80CF0DCF905A90500E0
:100F0000020020000BF030FE6419029B0437BB4244
:100F1000BFD10023237005E7032EF6D11A0992B240
:100F20005B0F92001E40961B291DC5E7F0B50D0012
:100F300097B0002806DC1C2000F032FC07003800C7
:100F400017B0F0BD0C68012123000B40009306D1BF
:100F5000042C04D922680F331A40092A01D00B202F
:100F6000EAE7626852100392002A03DC009803F05B
:100F700075FAE3E7504A019201280BD068680842ED
:100F800008D1042806D902681340042B02D103F0CB
:100F900051F8019001980CF08DF906000F27039B82
:100FA0000834013B05935E43039B02909B00E318CA
:100FB000049301232068184273D1042871D9016871
:100FC0000B003B409C46042B03D1FFF7D9F8861950
:100FD00009E0032B6CD162460B099BB2490F9B00C1
:100FE00011405A1A9619049B0434A342E1D13000EF
:100FF00003F034FA071EA2D02B680793029B002B44
:1010000003D0686803F016F80190380003F012F876
:101010000400009B079A9B00D3189E68300003F0E1
:1010200009F80123334005000693002B01D1042E5B
:1010300004D809A93000FFF723FE09AD28000CF001
:1010400039F9069B0490002B0ED1042E0CD90F21E8
:1010500033681940032907D11A0992B25B0F920035
:101060000B40D31A351D04932000049A29000BF07D
:101070007BFD049BE418029B002B0AD0059B009A81
:10108000934206DD2000029A01990BF06DFD029B50
:10109000E418009B01330093009A039B9342B8D15C
:1010A0004DE709A9FFF7ECFD09A80CF003F98EE75D
:1010B00002F0C0FFF9E7C046A0E7000010B501222A
:1010C000002400280BDD0B681A40141E03D05C10AE
:1010D000E343DB171C400122904200D04A68611CA8
:1010E000092003F049F9002803D0012364001C43C0
:1010F000446010BD0A6870B510000125284034D145
:10110000042A32D90F24136849681C40092C17D1CE
:1011100054681B099BB22C41A34200D85C1E844238
:1011200005DC02200133984206DB00200FE0850039
:101130005519A9600130F2E7840011510130F2E73E
:10114000032C12D1294203D1132000F029FB70BDDA
:101150004910FF29F8D81B099BB204329B00D31811
:101160009342E2D911700132FAE70B2000F018FB2C
:10117000DBE700000123F7B500254E680C00334083
:101180000193AB420ED11D00042E0BD90F22336800
:101190001A40092A26D172681B099BB25510AB422E
:1011A00000D85D1E27687C10FB0746D439003D48F7
:1011B000FFF7DAFC002826D00BF0D2FF290009F057
:1011C00091FC4C1C019B002B00D069E0042E67D9D8
:1011D00032680F331340092B3BD10134A400A459CA
:1011E0002000FEBD042A04D13000FEF7C9FF05002F
:1011F000D8E7019D032AD5D11D09ADB25B0FAD0023
:101200001340ED1ACEE739002748FFF7ADFC002860
:101210001DD1042F16D90F233A681340042B11D186
:101220003800FFF7D7FB041E07D139001F48FFF72E
:101230009BFC002806D0122005E0002CFBDDA54217
:10124000C0DAF8E7112000F0ABFA0400C8E72C0080
:10125000B8E7042B1CD1300002F0ECFE0500012C95
:101260000EDCFEF7A5FF461B300003F0F7F8041E66
:10127000B6D002F0DFFE320029000BF075FCAFE7BC
:101280002B78013C002BD6D02800FEF791FFE5E734
:10129000032B05D13419E37801245B001C439FE73D
:1012A0000B20D0E744E200004FE2000054E20000CF
:1012B000F7B54D680E002A0001210A402FD1042DF8
:1012C0002DD90F242B68B7681C40092C14D16968EC
:1012D0001B099BB24C100192A34200D85C1E3168DE
:1012E0003448FFF741FC00282DD00F232A68134013
:1012F000092B1DD1012317E0032C10D10F4203D17C
:10130000132000F04DFAFEBD7A100192FF2AF7D8A3
:101310001A0992B25B0F92001C40141BDFE70B20EE
:10132000EFE701339A00AF509C42FADA0020EAE777
:10133000032BFBD12B0001335A1BA242F6DC6A4679
:101340001279DA70F7E736687010F30719D43100B4
:101350001948FFF709FC002822D1042E1ED90F23BB
:1013600032681340042B19D13000FFF733FB0028FB
:1013700007D131001148FFF7F7FB00280ED01220EB
:10138000BFE70028FBDD8442F9DB0F232A68134006
:10139000092B07D1013080004751C7E71120B0E782
:1013A0002000F2E7032BC1D16B461B792D18EB709F
:1013B000BCE7C0464BE200004FE2000054E20000F0
:1013C00070B501240868204207D1042805D90F25EB
:1013D00001680D40092D02D14468200070BD032D25
:1013E00008D10A0992B24B0F92002B40D31A5B002E
:1013F0001C43F2E7042DF0D102F01CFEFEF7ECFED8
:1014000040000443E9E7000010B5034A0E210348F9
:1014100004F002FF10BDC046D4E10000CCE10000A2
:1014200000207047042070470120704710B500204D
:1014300003F014F810BD0020704700207047002012
:101440007047002070470020704700207047002040
:1014500070470020704700207047000010B5034A15
:101460000D21034804F0D8FE10BDC046ECE2000098
:1014700054E3000070470378002B03D05AB2002ACF
:1014800001DB013070473F229343C03B59424B413F
:10149000C01803789343802BF4D10130F9E70000A2
:1014A000F8B50127060014000800394227D10429A5
:1014B0003FD90F230A681A40042A3AD13C4213D17B
:1014C000042C11D922681340042B0DD102F0B2FD77
:1014D0000500200002F0AEFD010028000BF0E0FE48
:1014E00000282EDB1FD127E0E30722D502F0A2FD62
:1014F0000A2200210BF0A6FF0500601010E0174043
:1015000015D1042A15D90F2312681340042B10D1CA
:1015100020004D1002F08EFD0A2239000BF092FFE0
:1015200085420EDB08DD002E09DC00200CE04D10AA
:10153000E3E70F22054B1A700136022EF5D804207E
:1015400002E0042076173040F8BDC046B00200200B
:10155000F8B5060000252C4BEC00E4182379032B8A
:1015600009D00135FF2DF6D1300004F069FE0028C6
:1015700048D1013846E030000BF09CFEEBB202008F
:101580003100180004F0DCFE002839D122685168CF
:101590008842E6D08300D3189B680130F02BF7D146
:1015A00001238000083012181A42DAD1042AD8D94F
:1015B0000F21136819400429D3D11B0998B20123C4
:1015C0000130800010181842CBD10428C9D90F224D
:1015D00003681340042BC4D102F02CFD0327040040
:1015E000092120000BF04EFE0028BAD0013F441C18
:1015F000002FF5D1310020000BF088FE8442B0D1DD
:1016000002482843F8BDC046C825002000FFFFFF60
:1016100010B50124044002D04410200010BD04285D
:1016200010D90F2302681340042B07D102F002FDEA
:1016300021000A220BF006FF0400EEE7032B01D184
:101640000430F5E70D22014B1A70E6E7B0020020E6
:10165000012210B5024018D1042802D903681A09E2
:1016600092B201230B4012D1042902D90B681B0945
:101670009BB20024934206D104309B000431C3186E
:10168000984206D30124200010BD0022E9E7002380
:10169000EFE704780A78002C01D1002AF2D001305B
:1016A00001319442ECD00024EDE70000F7B50700CB
:1016B000009101933049314B002A02D002220A7076
:1016C000013A00261A601B68CE54BE4200DBF7BD0B
:1016D000009AB300D058294B274D1C68C8239B00A3
:1016E00065191C1B0123184206D0254A431021000E
:1016F00028000BF067FD09E0224A002802D00428E8
:101700001BD1214A210028000BF05CFD1A4C20005F
:101710000BF0D0FD194A019B1060002B0BD07B1EF3
:10172000B34208DD194B984205D8431C13602022B0
:1017300022540022E2540136C7E7042819D90F23A6
:1017400001680B40042B04D102F074FC104A030022
:10175000CDE7092B03D143680E4A5B10C7E7032B83
:1017600008D10A0992B2490F92000B40D31A0A4AD3
:10177000BDE70123094ABAE7B1020020D4050020E1
:10178000D8EE000056E200005CE200001F030000FB
:1017900007F50000CCE50000DBE50000E6E5000011
:1017A000014B187000207047B0020020024B1878DF
:1017B000431E98417047C046B0020020002310B578
:1017C0001A00FFF773FF034B0348196805F01DFA71
:1017D000002010BDD4050020B102002070B502F039
:1017E000B7F9094C0100251D1F2228000BF07AFDD6
:1017F00028000BF05FFD042304308008000118432B
:101800002060200070BDC0468C020020C368F0B587
:101810009D00836889B05D19030018330393036941
:10182000039A9F00039B0190DF19436900939B007B
:10183000D3180293D04B1B78002B26D17F222B6824
:10184000CE491C1213409B005B58043500929F4602
:10185000019B587805F0B8F90023019A137027E02E
:10186000C54B1B78002B10D12B68009A1C1213401B
:10187000C24A9B009B580435E9E7039B3A1DD11AE5
:10188000BD4BD82928DD1A221A70019BBA4C9B68DF
:1018900021780093EA1A019B92109B7812021A4356
:1018A000019B587805F098F90023019A2370137072
:1018B000019B039A9B680093ED1A019BAD10DD60BC
:1018C000039BFE1A019BB6101E61029B9B1A019A94
:1018D0009B10536109B0F0BD39001B7817000C60F4
:1018E000002BD2D12B68009A1C121340A34A9B00F4
:1018F0009B580435ABE7039B3A1DD11A9E4BD82960
:1019000002DD1A221A70C0E738001B7817002A6817
:10191000291D0260002B01D00D00B6E76B68009A0C
:101920001C121340954A9B009B5808358FE7039B78
:101930003A1DD11A904BD82902DD1A221A70A4E759
:101940003900A4001B782C1917000C60002B9CD1C7
:101950002B68009A1C121340884A9B009B58043540
:1019600075E7039B3A1DD11A834BD82902DD1A2251
:101970001A708AE739001700814AA400A2581B7820
:101980000A60002B00D080E72B68009A1C121340DD
:101990007A4A9B009B58043559E7043F784B3A68D4
:1019A000A400E250744B1B78002B00D06DE72B682D
:1019B000009A1C121340714A9B009B58043546E75D
:1019C0006F4BA400E058FFF723FE6B4B06001B781B
:1019D000002B09D1043F3868FFF71AFE8619012051
:1019E0007600674B0643E650634B1B78002B00D014
:1019F0004BE72B68009A1C121340604A9B009B58CF
:101A0000043524E7039B391DCA1A5B4BD82A02DD33
:101A10001A221A7039E70398029C0122A04202D2CE
:101A200022000C3A126838001B780F000260002B6D
:101A300000D02AE72B68009A1C1213404F4A9B00E3
:101A40009B58043503E7039A3B1D991A4A4AD82943
:101A500002DD1A23137018E703990298814218D205
:101A600002000C3A1268474952106418A41AA400E4
:101A700022583A601F00404B1B78002B00D004E72F
:101A80002B68009A1C1213403C4A9B009B5804355B
:101A9000DDE6182111700022EBE7039B029A9342C6
:101AA00019D213000C3B1B68364A5B10A418043F84
:101AB000E41A3A68029BA400E2502F4B1B78002BDB
:101AC00000D0E2E62B68009A1C1213402B4A9B00C0
:101AD0009B580435BBE61822274B1A70EDE7039B91
:101AE000029A934228D2274B043FE61814000C3C7C
:101AF00023685B10F31A9B009858FFF789FD049048
:101B00003868FFF785FD2468049B6410341B1E1899
:101B100001207600029BA4000643E650164B1B787A
:101B2000002B00D0B1E62B68009A1C121340134A18
:101B30009B009B5804358AE618220F4B1A70EDE77C
:101B4000039B3A1DD11A0C4BD82902DD1A221A70B8
:101B50009BE639001700029AA400A2581B780A607D
:101B6000002B00D091E62B68009A1C121340034A08
:101B70009B009B5804356AE6B0020020CCE30000CD
:101B8000C02D0020FDFFFF3F043F029B3A68A400E8
:101B9000E250D54B1B78002B00D076E62B68009ADC
:101BA0001C121340D14A9B009B5804354FE6029B00
:101BB000A4001C192368043F38685E10FFF728FD55
:101BC00036180120C84B76001B7806432660002B90
:101BD00000D05AE62B68009A1C121340C34A9B009F
:101BE0009B58043533E6039BA4003F1BBE4CBB420D
:101BF0000CD82378002B00D047E62B68009A1C12E3
:101C00001340BA4A9B009B58043520E6B84802F0BE
:101C100001FA2378002B00D037E62B68009A1C12BB
:101C20001340B24A9B009B58043510E6A300ED1800
:101C3000002C00DA3CE6AC4B1B78002B00D024E6ED
:101C40002B68009A1C121340A84A9B009B5804352D
:101C5000FDE5043F3B68042B04D1A300ED18002CE4
:101C600000DA25E6A04B1B78002B00D00DE62B6890
:101C7000009A1C1213409D4A9B009B580435E6E5D0
:101C8000043F3B68042B04D0A300ED18002C00DABD
:101C90000EE6954B1B78002B00D0F6E52B68009ADA
:101CA0001C121340914A9B009B580435CFE53E1F00
:101CB0003068C3070AD540100138002809DB01232A
:101CC0004000A40018432D193060F1E5FFF7A0FC97
:101CD000F2E7854B1B78002B01D03700D5E52B6848
:101CE000009A1C121340814A9B009B583700043510
:101CF000ADE53E00039802990C36091A891004914B
:101D0000311AD82902DD1A231370BEE539006700A5
:101D1000FF24012064003C4004430C60019C1278C5
:101D2000A468370002942D1B019CAD10A4782D02ED
:101D30002543049C854084400543204388606046D9
:101D40004D60019988706B495B5801998B60002A3E
:101D500003D008331D00029697E51D00009A9B688A
:101D60000C351C121340614A9B009B5802966EE58D
:101D70003B1F1C68029A039B934232D10A20E3075F
:101D800011D4042C18D90F2322681340042B16D128
:101D9000200002F04FF90BF08DFAC8239B00984207
:101DA00000D918000630643004F012FB00280FD16F
:101DB000043D039B02937BE50720042CF3D0200015
:101DC000431E9841FA234042FF3318400730EAE7A8
:101DD000019B2100587804F011FF0023019A137031
:101DE000E7E7029B029A0C3B1B6801995B109B0082
:101DF000D31A0C3B1C601F1D1300083B1B685A10B4
:101E00008A70FF210A403B49D2005B0055589B0A6B
:101E1000019A9B009560ED18029B039A043B1B6896
:101E20005B109B00D31802932F4B1B78002B00D024
:101E30002BE52B68009A1C1213402C4A9B009B58E0
:101E4000043504E53B1F1868FFF7E2FBA400060019
:101E50003F1B1E2827DC00280DDC234B1B78002BA2
:101E600000D012E52B68009A1C1213401F4A9B00F9
:101E70009B580435EBE401F053FE033E361801F0A5
:101E80004FFE1D4B801B9842F9D8174B1B78002B37
:101E900000D0FAE42B68009A1C121340134A9B00EE
:101EA0009B580435D3E40123019A137001F038FEE6
:101EB000019B0A3886195E60FAE43B1F1868FFF739
:101EC000A7FBA40006003F1B002817DC064B1B786D
:101ED000002B00D0D9E42B68009A1C121340034A4F
:101EE0009B009B580435B2E4B0020020CCE3000014
:101EF000F8E50000C82500207F969800D64B984250
:101F000003DD1D22D54B1A70BFE40123019A137023
:101F100001F006FEFA239B005E430A3E3018019B47
:101F20005860C5E4A300FF1A002320001A003900FE
:101F3000FFF7BCFBCA4ECB4C3168200002F09AFA86
:101F4000C94B31681860200004F008FD316820009A
:101F500004F05BFEC14B1B78002B00D095E42B688E
:101F6000009A1C121340C14A9B009B5804356EE432
:101F7000BA4BA4001B783F1B002B00D085E42B68D4
:101F8000009A1C121340B94A9B009B5804355EE42A
:101F9000019804F081FAB14B1B78002B00D074E457
:101FA0002B68009A1C121340B04A9B009B580435C2
:101FB0004DE43B1F1B68002B48D13B000C3B1868CD
:101FC000012303401E1E1FD046103A00012371005A
:101FD000083A0B431360002E00DC93E001237200EB
:101FE0001A43391F0A603A00083A12681A41921BD4
:101FF00004923A000C3A106818422AD0049AA400BD
:10200000D2189A40134330E004281BD90F230268EA
:102010001340092B02D143685E10D6E7042B08D188
:1020200002F008F80378002BCFD0FFF724FA01362E
:10203000F8E7032B06D11609B6B2520FB6001340CB
:10204000F61AC2E71922854B1A701EE45B105E1E59
:10205000C1E7042851D90F2201680A40092A16D184
:10206000049BA40002339B001B58029AA3507B4B95
:102070001B78002B01D0FFF708FC2B68009A1C127C
:1020800013407A4A9B009B580435FFF7E0FB042A73
:102090002BD1029BA4001B19069301F0CBFF060075
:1020A000049C0134012C10DC3000FFF7E4F9831BA1
:1020B0001800049302F0D2F9041E0ED001F0BAFF0A
:1020C000049A31000AF050FD07E03178013C002904
:1020D00006D112220C00614B1A70069B1C60C6E7E9
:1020E0003000FFF7C8F90600DCE7032A05D1049A9F
:1020F000A40082181279520084E71922574B1A70F3
:10210000FFF7C3FB0435B2E7A300039AFB189B1A41
:10211000D82B13DC0122631E002C14DC4F4B1B78E0
:10212000002B01D0FFF7B1FB2B68009A1C12134063
:102130004E4A9B009B580435FFF789FB1A22474BF8
:102140001A70FFF7A2FB3A601C000437E3E7039A1A
:102150003B1D9B1A414ED82B03DD1A233370FFF72A
:1021600094FB039B029AA40093422AD23B1F186857
:10217000FFF74EFA011E21DD029B0C3B1A6852103C
:1021800082421BDB9007801A394B4018C018029B13
:102190008000C2583B1B1A60304B3F1B1B78043732
:1021A000002B01D0FFF771FB2B68009A1C12134023
:1021B0002E4A9B009B580435FFF749FB20233370C0
:1021C000EAE71823FBE7284BA4001A683B1B1F0013
:1021D0001A60224B04371B78002B01D0FFF755FB08
:1021E0002B68009A1C121340204A9B009B58043510
:1021F000FFF72DFB3A1F1368042B02D13A00A4000D
:102200002D19164B1B78002B02D01700FFF73DFB52
:102210002B6800991C120B4014499B005B58170057
:102220000435FFF714FB043F3B68042B04D0002364
:10223000A4003B602D190437084B1B78002B01D0FC
:10224000FFF723FB2B68009A1C121340074A9B00E0
:102250009B580435FFF7FBFA80EE3600B0020020F1
:10226000D4050020B102002008000020CCE30000CB
:10227000FCFFFF3FA3009C46FE1A002C17DC1C222B
:10228000D34B1A70002333606346FF1AD04B0437D8
:102290001B78002B01D0FFF7F8FA2B68009A1C126C
:1022A0001340CC4A9B009B580435FFF7D0FA00201E
:1022B00033685A108300F15801230B4003D10D21DC
:1022C000C34A1170DFE749108A4200DD0A0001307D
:1022D0008442EFDC012352001343D4E7A3009C4661
:1022E000FE1A002C17DC1C22B94B1A700023336035
:1022F0006346FF1AB64B04371B78002B01D0FFF75B
:10230000C4FA2B68009A1C121340B24A9B009B58D7
:102310000435FFF79CFA002033685A108300F15807
:1023200001230B4003D10D21A94A1170DFE74910A9
:102330008A4200DA0A0001308442EFDC01235200B5
:102340001343D4E73B000122083B1968A400114263
:102350001DD03B1F1B68134219D0114113410022AD
:10236000994200DA04323B1B1A60994B3F1B1B78E1
:102370000437002B01D0FFF788FA2B68009A1C1253
:102380001340944A9B009B580435FFF760FA0220E3
:102390003B1F1A684042FFF783F83E1B3060E4E7BA
:1023A0003B00083B19680123A40019421ED03A1FC4
:1023B00012681A421AD019415010CB0FD217884216
:1023C00053413A1B9B001360814B3F1B1B78043722
:1023D000002B01D0FFF759FA2B68009A1C1213400A
:1023E0007C4A9B009B580435FFF731FA01203B1FC4
:1023F0001A684042FFF754F83E1B3060E4E73B00A8
:10240000083B18683B1F1968A600BE1B04238142C5
:1024100002D0042802D80023336016E001231842BA
:10242000F9D10F2302681A40042AF4D1033A114269
:10243000F1D10429EFD90A681340042BEBD1FFF73F
:1024400007F9431E984180003060614BA4001B785F
:102450003F1B0437002B01D0FFF717FA2B68009AB7
:102460001C1213405B4A9B009B580435FFF7EFF9A1
:102470003B00083B18683B1F1968A600BE1B0023E1
:10248000814202D0042802D80423336016E00123DD
:102490001842F9D10F2302681A40042AF4D1033AF2
:1024A0001142F1D10429EFD90A681340042BEBD172
:1024B000FFF7CEF84342584180003060444BA400FF
:1024C0001B783F1B0437002B01D0FFF7DEF92B6888
:1024D000009A1C1213403F4A9B009B580435FFF79B
:1024E000B6F93B000122083B1968A40011421ED036
:1024F0003B1F1B6813421AD05B104A10D80FC91734
:102500009A4241413B1B89001960314B3F1B1B78AC
:102510000437002B01D0FFF7B8F92B68009A1C1282
:1025200013402C4A9B009B580435FFF790F93B1F42
:102530001A680120FEF7B4FF3E1B3060E5E73B0060
:102540000122083B1968A40011421DD03B1F1B68E3
:10255000134219D0114113410022994200DD043287
:102560003B1B1A601A4B3F1B1B780437002B01D012
:10257000FFF78BF92B68009A1C121340154A9B0039
:102580009B580435FFF763F93B1F1A680220FEF7DA
:1025900087FF3E1B3060E5E73B1F1B68A400043B40
:1025A0005A1E93413A1B17009B001360084B0437D7
:1025B0001B78002B01D0FFF768F92B68009A1C12DA
:1025C0001340044A9B009B580435FFF740F9C0466E
:1025D000B0020020CCE300003B00083B1868FFF786
:1025E00017F83B1F06001868FFF712F83218012091
:1025F000A4003B1B1F00520002431A60EB4B043740
:102600001B78002B01D0FFF740F92B68009A1C12B1
:102610001340E74A9B009B580435FFF718F93B002D
:10262000083B1868FEF7F4FF3B1F06001868FEF72A
:10263000EFFF321A0120A4003B1B1F00520002438F
:102640001A60DA4B04371B78002B01D0FFF71DF915
:102650002B68009A1C121340D54A9B009B580435E6
:10266000FFF7F5F83B00083B1868FEF7D1FF3B1F6A
:1026700006001868FEF7CCFF02000120A4003B1BF7
:102680001F007243520002431A60C84B04371B7884
:10269000002B01D0FFF7F9F82B68009A1C121340A9
:1026A000C34A9B009B580435FFF7D1F83B1F1868BD
:1026B000FEF7AEFF061E17D11F23BC4A1370A400FD
:1026C0003B1B1F001E60B94B04371B78002B01D049
:1026D000FFF7DBF82B68009A1C121340B44A9B00EA
:1026E0009B580435FFF7B3F83B00083B1868FEF72A
:1026F0008FFF310008F010F9012640000643DEE7A5
:102700003B1F1868FEF784FF061E17D11F23A74A38
:102710001370A4003B1B1F001E60A44B04371B78E2
:10272000002B01D0FFF7B1F82B68009A1C12134060
:102730009F4A9B009B580435FFF789F83B00083BF4
:102740001868FEF765FF310008F0CCF90126490052
:102750000E43DEE73B1F1868FEF75AFFC2178018CA
:1027600050400122A4003B1B1F0040001043186092
:102770008E4B04371B78002B01D0FFF786F82B68AF
:10278000009A1C1213408A4A9B009B580435FFF79D
:102790005EF8A3000793FB1A0693012C2DD118684D
:1027A000FEF736FFC617A64304900136049B9E42EF
:1027B00001DC04961E00049B0136F61A0AF0D0FCD8
:1027C000310008F08FF9049B069ACB1801215B00B9
:1027D0000B431360079BFF1A744B04371B78002BC5
:1027E00001D0FFF752F82B68009A1C121340704A70
:1027F0009B009B580435FFF72AF8022C0AD1069B50
:102800001868FEF705FF069B06005868FEF700FFF4
:102810000490CBE7012364260493CCE7A300FE1ABF
:1028200031002000049301F073FF049B3060FF1A15
:102830005E4B04371B78002B01D0FFF726F82B687E
:10284000009A1C1213405A4A9B009B580435FEF70D
:10285000FEFF3B00083B1868FEF7DAFE3B1F060050
:102860001868FEF7D5FE02000120A4003B1B1F00E4
:102870003240520002431A604C4B04371B78002B45
:1028800001D0FFF702F82B68009A1C121340484A47
:102890009B009B580435FEF7DAFF3B00083B1868A5
:1028A000FEF7B6FE06003B1F1868FEF7B1FE3200C9
:1028B00002430120A4003B1B1F00520002431A6088
:1028C0003A4B04371B78002B01D0FEF7DEFF2B6854
:1028D000009A1C121340364A9B009B580435FEF7A1
:1028E000B6FF3B00083B1868FEF792FE06003B1F50
:1028F0001868FEF78DFE320042400120A4003B1B09
:102900001F00520002431A60284B04371B78002B2B
:1029100001D0FEF7BAFF2B68009A1C121340244A1C
:102920009B009B580435FEF792FF3B1F1868FEF78B
:102930006FFEC0430122A4003B1B1F004000104358
:1029400018601A4B04371B78002B01D0FEF79DFF4F
:102950002B68009A1C121340154A9B009B580435A3
:10296000FEF775FF3B00083B1868FEF751FE0600B6
:102970003B1F1868FEF74CFE3200824051000122D6
:10298000A4003B1B1F000A431A60084B04371B7846
:10299000002B01D0FEF779FF2B68009A1C12134020
:1029A000034A9B009B580435FEF751FFB0020020FC
:1029B000CCE300003B00083B1868FEF729FE060048
:1029C0003B1F1868FEF724FE32000241510001222D
:1029D000A4003B1B1F000A431A60E94B04371B7815
:1029E000002B01D0FEF751FF2B68009A1C121340F8
:1029F000E44A9B009B580435FEF729FF3B000C3B43
:102A00001868FEF705FE3B00083B06001868FEF755
:102A1000FFFDF1170200C317300008F0B5F83B1FA7
:102A2000049005911868FEF7F3FD020004980599DB
:102A300008F05EF843000120A4003E1B3700184355
:102A4000CF4B30601B780437002B01D0FEF71DFF01
:102A50002B68009A1C121340CA4A9B009B580435ED
:102A6000FEF7F5FEA300FE1A310020000493FEF7E6
:102A700025FB049B3060FF1AC14B04371B78002BE9
:102A800001D0FEF702FF2B68009A1C121340BD4ACA
:102A90009B009B580435FEF7DAFEA300FF1A3900AD
:102AA0002000FEF727FBB64B1B78002B01D0FEF76A
:102AB000ECFE2B68009A1C121340B24A9B009B58F4
:102AC0000435FEF7C4FEA300FE1A31002000049373
:102AD000FEF750FB049B3060FF1AA94B04371B78AC
:102AE000002B01D0FEF7D1FE2B68009A1C12134078
:102AF000A44A9B009B580435FEF7A9FEA300FF1AC9
:102B000039002000FEF7D4FB9D4B1B78002B01D031
:102B1000FEF7BBFE2B68009A1C121340994A9B00DB
:102B20009B580435FEF793FEA300FE1A31002000E7
:102B30000493FEF745FC049B3060FF1A904B04376A
:102B40001B78002B01D0FEF7A0FE2B68009A1C1208
:102B500013408C4A9B009B580435FEF778FE3B1FC0
:102B6000186801F067FA3A00083A12680300A400F6
:102B7000D10729D4042A0CD910680F22104001383B
:102B800008280FD807F02AFE052026220E0E0E0E6A
:102B900024007D4918000AF083FB434258413B1B47
:102BA00080001860764B3F1B1B780437002B01D048
:102BB000FEF76BFE2B68009A1C121340714A9B00B3
:102BC0009B580435FEF743FE7049E3E77049E1E79F
:102BD0007049DFE77049DDE7039B3E1DF31A684C3F
:102BE000D82B03DD1A232370FEF74FFE00F0A2FF5F
:102BF000430001203A001843237837001060002B6F
:102C000001D0FEF742FE2B68009A1C1213405D4A69
:102C10009B009B580435FEF71AFE039B3E1DF31ADA
:102C2000574CD82B03DD1A232370FEF72EFE00F03D
:102C300077FF5A4A4000104001223B0010431860C1
:102C400023783700002B01D0FEF71FFE2B68009A77
:102C50001C1213404B4A9B009B580435FEF7F7FDAE
:102C6000039A3B1D9B1A464CD82B03DD1A23237075
:102C7000FEF70BFE00F05EFF494B1A68831A904284
:102C800001D2484A9B1801203A005B0003431360BD
:102C900023780437002B01D0FEF7F7FD2B68009A4C
:102CA0001C121340374A9B009B580435FEF7CFFD9A
:102CB00000F040FF3A4BA4001860314B3F1B1B78DB
:102CC000002B01D0FEF7E1FD2B68009A1C12134087
:102CD0002C4A9B009B580435FEF7B9FD03F064FBBA
:102CE000A300002810D1FF1A254B1B78002B01D020
:102CF000FEF7CBFD2B68009A1C121340214A9B0063
:102D00009B580435FEF7A3FD3E00FF1A0123200067
:102D10001A003900FEF7CAFC234C2068643003F027
:102D200057FB002803D1043D3700FEF7C1FD019B8E
:102D300021685A781D4803F07AFF0123019A137025
:102D400000F0EEFE1A4B22681B6806325343181837
:102D5000FFF7E5F803F028FBA30000282AD1FF1AAB
:102D6000074B1B78002B01D0FEF78FFD2B68009AD4
:102D70001C121340034A9B009B580435FEF767FD65
:102D8000B0020020CCE3000008E6000010E60000DE
:102D900017E600001EE6000023E60000FEFFFF7FAE
:102DA000DC05002037894100D4050020B102002055
:102DB000040000203E00FF1A2000012300223900F9
:102DC000FEF774FCF14C2068643003F001FB00282E
:102DD000A9D0EF4803F0A8FCAFE7A4003E1BFEF724
:102DE000FDFC3700EB4B30601B780437002B01D023
:102DF000FEF74BFD2B68009A1C121340E64A9B001D
:102E00009B580435FEF723FDE24BA4001B783F1BC3
:102E1000002B01D0FEF739FD2B68009A1C121340DD
:102E2000DD4A9B009B580435FEF711FDA4003E1BB4
:102E3000300000F0B8FE3700D64B30601B78043706
:102E4000002B01D0FEF721FD2B68009A1C121340C5
:102E5000D14A9B009B580435FEF7F9FCA4003E1BA9
:102E6000300000F0A2FE3700CA4B30601B780437F8
:102E7000002B01D0FEF709FD2B68009A1C121340AD
:102E8000C54A9B009B580435FEF7E1FCA300FE1ADF
:102E900031002000049300F037FC049B3060FF1ADF
:102EA000BC4B04371B78002B01D0FEF7EEFC2B68DF
:102EB000009A1C121340B84A9B009B580435FEF739
:102EC000C6FCA4003F1B380000F072FEB14B1B781B
:102ED000002B01D0FEF7D9FC2B68009A1C1213407E
:102EE000AD4A9B009B580435FEF7B1FCA300FE1AC7
:102EF00031002000049300F03DFC049B3060FF1A79
:102F0000A44B04371B78002B01D0FEF7BEFC2B68C6
:102F1000009A1C121340A04A9B009B580435FEF7F0
:102F200096FCA4003F1B380000F09AFE994B1B78DA
:102F3000002B01D0FEF7A9FC2B68009A1C1213404D
:102F4000954A9B009B580435FEF781FC0121200027
:102F500000F060FE8F4B1B78002B01D0FEF795FC34
:102F60002B68009A1C1213408B4A9B009B58043517
:102F7000FEF76DFC0021200000F04CFE854B1B7815
:102F8000002B01D0FEF781FC2B68009A1C12134025
:102F9000814A9B009B580435FEF759FCA4003E1B58
:102FA000300000F08BFE37007A4B30601B7804371E
:102FB000002B01D0FEF769FC2B68009A1C1213400D
:102FC000754A9B009B580435FEF741FCA4003E1B4C
:102FD000300000F087FE37006E4B30601B780437FE
:102FE000002B01D0FEF751FC2B68009A1C121340F5
:102FF000694A9B009B580435FEF729FCA4003F1B3F
:10300000380000F043FE634B1B78002B01D0FEF725
:103010003CFC2B68009A1C1213405F4A9B009B5893
:103020000435FEF714FCA4003F1B380004F090FAAE
:10303000584B1B78002B01D0FEF727FC2B68009A19
:103040001C121340544A9B009B580435FEF7FFFBAB
:10305000A4003E1B300004F049FB37004D4B3060AC
:103060001B780437002B01D0FEF70FFC2B68009A69
:103070001C121340484A9B009B580435FEF7E7FB9F
:10308000A4003F1B380004F00BFA424B1B78002BC6
:1030900001D0FEF7FAFB2B68009A1C1213403E4A3F
:1030A0009B009B580435FEF7D2FBA4003E1B30006A
:1030B00004F010FA3700374B30601B780437002BD0
:1030C00001D0FEF7E2FB2B68009A1C121340324A33
:1030D0009B009B580435FEF7BAFBA300FF1A39008A
:1030E000200001F053FF2B4B1B78002B01D0FEF783
:1030F000CCFB2B68009A1C121340274A9B009B585C
:103100000435FEF7A4FBA300FF1A3900200001F0EC
:1031100043FD204B1B78002B01D0FEF7B6FB2B683C
:10312000009A1C1213401C4A9B009B580435FEF762
:103130008EFBA300FF1A3900200001F0DFFD154BC4
:103140001B78002B01D0FEF7A0FB2B68009A1C1205
:103150001340114A9B009B580435FEF778FBA300EF
:10316000FF1A3900200001F0F1FD0A4B1B78002BFB
:1031700001D0FEF78AFB2B68009A1C121340064A06
:103180009B009B580435FEF762FBC046D405002027
:10319000B1020020B0020020CCE30000A300FE1A20
:1031A00031002000049304F08BFB049B3060FF1A75
:1031B000CA4B04371B78002B01D0FEF766FB2B6847
:1031C000009A1C121340C64A9B009B580435FEF718
:1031D0003EFBA300FE1A31002000049304F078FBAC
:1031E000049B3060FF1ABD4B04371B78002B01D0C5
:1031F000FEF74BFB2B68009A1C121340B84A9B0049
:103200009B580435FEF723FBA300FE1A3100200073
:10321000049304F065FB049B3060FF1AAF4B043746
:103220001B78002B01D0FEF730FB2B68009A1C1294
:103230001340AB4A9B009B580435FEF708FBA300E4
:10324000FE1A31002000049303F0E4FF049B306079
:10325000FF1AA24B04371B78002B01D0FEF715FB99
:103260002B68009A1C1213409D4A9B009B58043502
:10327000FEF7EDFAA300FF1A3900200001F006FE68
:10328000964B1B78002B01D0FEF7FFFA2B68009AB3
:103290001C121340924A9B009B580435FEF7D7FA44
:1032A000A300FF1A3900200001F078FD8B4B1B783A
:1032B000002B01D0FEF7E9FA2B68009A1C1213408C
:1032C000874A9B009B580435FEF7C1FAA300FE1AFB
:1032D00031002000049301F0DDFC049B3060FF1AF4
:1032E0007E4B04371B78002B01D0FEF7CEFA2B68FB
:1032F000009A1C1213407A4A9B009B580435FEF733
:10330000A6FAA300FF1A3900200001F071FC734BEC
:103310001B78002B01D0FEF7B8FA2B68009A1C121C
:1033200013406F4A9B009B580435FEF790FA002C1F
:1033300000DC83E03B1F1E68012C0CD1264207D124
:10334000042E05D90F23326830001340042B10D00F
:1033500001235B4212E0022CFAD13B00083B1868C3
:10336000C307F5D40428F3D90F2302681340042BB4
:10337000EED100F05FFEFEF7EBF80300A200BF1AEB
:103380005A1C5BD00020022C12D101223240824212
:103390002ED1042E2CD90F2130680140092927D1C4
:1033A00071684810FF210840810091421BD17F18AD
:1033B0001A00FF244B49A2438A4221D11C06240C47
:1033C000044323129C46FF2362461340464ADB0017
:1033D000D2181179414A032901D1FEF78AFC022350
:1033E0001370FEF752FAB418A468BC500432DCE73C
:1033F0000B223A4B1A7000233B600437FEF745FA64
:10340000039A0199BA1A86009210BE1B0A61310014
:1034100098470022354B371D1A60304B30601B78BF
:10342000934201D0FEF731FA2B68009A1C12134028
:103430002B4A9B009B580435FEF709FA00233B609A
:10344000264B3A1D1B78002B02D01700FEF71DFA01
:103450002B6800991C120B4021499B005B581700F8
:103460000435FEF7F4F9039B019AFB1A9B101361D4
:10347000A300FF1A3900200003F098F9174B1B78BE
:10348000002B01D0FEF701FA2B68009A1C121340A2
:10349000134A9B009B580435FEF7D9F9039B019A08
:1034A000FB1A9B101361A300FE1A31002000049345
:1034B00003F07CF9049B3060FF1A084B04371B783B
:1034C000002B01D0FEF7E1F92B68009A1C12134083
:1034D000034A9B009B580435FEF7B9F9B00200205F
:1034E000CCE3000000FFFFFFC825002004100020EF
:1034F0000023F7B55A1E0192002B07DA01F05CFD9C
:1035000003F06CFA03F044FC192301930026300009
:10351000194B1968B14212DD184B1A6801328A4200
:103520000FDAF0241A601D68154F6C43E35D002B21
:103530001FD0E419022B06D12000FEF767F9019B8A
:10354000D8E70022EDE7012B0DD1002801D100F0D2
:10355000E7FAF0226A43BB185B680A49C31A8B4238
:1035600001D80223BB54F0235D43054BEB5C022BD7
:10357000E2D00136CCE7C046D8050020000000208C
:10358000681C00207F96980080220B4B52001A6026
:103590000121A822A920094BD20019649A58C00021
:1035A00005321A5006481A50C122C020920000036A
:1035B0009850044B1970704700E100E00080004013
:1035C0004C0500002306002004207047F8B550C9C0
:1035D000012322001A40101E2DD03340181E2AD07D
:1035E000641000201C2C26D81D4B761035009E42FE
:1035F00000DD1D001B4F3B5D012B05D0012120008C
:1036000005F0DCFC01233B55174B1B78002B01D147
:10361000FFF7BAFF0023154A9E420DDCFF2514492F
:103620001448D65CB44202D15E007052D5540133C6
:10363000042BF6D10420F8BDD15C8C4203D10C4A96
:103640005B009D52F6E70133042BF5D10023D15CDA
:10365000FF2901D1D454F2E70133042BF7D1E9E774
:103660008813000004060020230600201C00002010
:103670000E000020DC05000070B530C901232200D7
:103680001A40101E1BD02B40181E18D064101C2C82
:1036900000D90024154E335D012B05D001212000F7
:1036A00005F08CFC0123335569100800104A1038CE
:1036B000104B904204D9012252421A60042070BD7E
:1036C0001C600D4807F028F90C4B040018800C4BC7
:1036D0001B78002B01D1FFF757FF0122094B9A6499
:1036E000A922D200995864189C50E7E704060020EC
:1036F000908601001800002020A107000C00002087
:103700002306002000800040F8B501240B68060065
:103710000D00234204D10D20FEF742F82000F8BD31
:103720005B100A2B1DD1053B104A9B009C58104F83
:103730003B5D002B05D00021200005F03FFC00235D
:103740003B55012E06DD6B68042B03D102212000BE
:1037500005F034FC200005F0DFFA0124400020438E
:10376000DDE72000052BDFD9D9E7C046A0E6000041
:103770000406002070B501240D68254204D10D20F7
:10378000FEF70EF8200070BD6D101C2D17D8002418
:10379000012804DD4C68043C63425C416400094E2E
:1037A000735DA34204D02100280005F007FC745586
:1037B000280005F037FC03000420012BE3D0002093
:1037C000E1E7C04604060020F8B501260D68340084
:1037D000B04200DD4C682B003340181E0BD0230094
:1037E0003340181E07D06D10002D05DCA1230020EA
:1037F0001E4ADB00D650F8BD641000201C2CFAD8FD
:103800001B4F3B5D012B04D00121200005F0D6FBAE
:103810003E552900174807F07FF80A21053007F0C8
:103820007BF8154BA400E258144B12021343A2225A
:103830001349D2008B50134C0C4B9C50124C195115
:10384000012412495C50124B196900219950114A08
:10385000904200DD1000A8228021D2009850012261
:1038600089005A5004201A60C5E7C04600F00140A4
:103870000406002000B4C404ECF8000003000300B8
:103880000060004040A10040140500000405000055
:1038900000A00040FFFF0000030010B50120002B36
:1038A00002DC1B30FDF77CFF10BD10B50124044085
:1038B00002D04410200010BD042810D90F23026844
:1038C0001340042B07D100F0B5FB21000A2209F0B8
:1038D000B9FD0400EEE7032B01D10430F5E70D201C
:1038E000FDF75EFFE6E70000F8B50C00022803DCF8
:1038F0001C20FDF755FFF8BD0868FFF7D6FF06004E
:103900006068FFF7D2FF0500A068FFF7CEFF010057
:10391000794807F001F804001C2D01D90020EAE7DE
:10392000764F7B5D012B05D00121280005F046FB79
:1039300001237B550021280005F05EFB002C0ED0F2
:1039400020000138C046C046C046C046C046C046FA
:10395000C046C046C046C046C046C046F1D1012759
:1039600031002800394005F047FB002C0ED0200024
:103970000138C046C046C046C046C046C046C046E4
:10398000C046C046C046C046C046F1D1711039405D
:10399000280005F031FB002C0ED020000138C04675
:1039A000C046C046C046C046C046C046C046C046E7
:1039B000C046C046C046F1D10127B11039402800A9
:1039C00005F01AFB002C0ED020000138C046C0467E
:1039D000C046C046C046C046C046C046C046C046B7
:1039E000C046C046F1D1F1103940280005F004FB73
:1039F000002C0ED020000138C046C046C046C0464C
:103A0000C046C046C046C046C046C046C046C04686
:103A1000F1D1012731113940280005F0EDFA002CD1
:103A20000ED020000138C046C046C046C046C04641
:103A3000C046C046C046C046C046C046C046F1D19A
:103A400071113940280005F0D7FA002C0ED0200063
:103A50000138C046C046C046C046C046C046C04603
:103A6000C046C046C046C046C046F1D10127B1118C
:103A70003940280005F0C0FA3900002C0ED0200093
:103A80000138C046C046C046C046C046C046C046D3
:103A9000C046C046C046C046C046F1D1F6113140CE
:103AA000280005F0A9FA002C0ED020000138C046ED
:103AB000C046C046C046C046C046C046C046C046D6
:103AC000C046C046C046F1D10121280005F094FA55
:103AD000002C00D122E720000138C046C046C04675
:103AE000C046C046C046C046C046C046C046C046A6
:103AF000C046F1D112E7C04640420F000406002044
:103B00000420704710B5002803DC1C20FDF748FE98
:103B100010BD0B680020DB07FAD40D30F6E700007B
:103B20000122034B1A64A822D20098587047C0465D
:103B3000008000400122054B10B51A64A822FA212A
:103B4000D2009858890006F05DFE10BD008000404C
:103B500000487047B8E600001D20704770B5054E5C
:103B60000400335C0D008B4202D005F027FA355576
:103B700070BDC0460406002070B50024084D635D8A
:103B8000012B09D10021200005F036FA0021200088
:103B900005F014FA0023635501341D2CEED170BDDD
:103BA0000406002070470D2070473B20704700003E
:103BB000F8B501260468344202D04568354203D185
:103BC0000D20FDF7EDFDF8BD64101C2CFBD80B4F4C
:103BD0003B5D012B04D03100200005F0EFF93E558C
:103BE00007496D108D4202DCE943C91729402000C6
:103BF00005F018F90122034B1A55E4E704060020EA
:103C0000FF030000E005002010B50800FFF7D0FF1B
:103C1000002010BD70B505000C001C2814D80E4EF5
:103C2000335C012B04D0012105F0C8F90123735541
:103C30000A4B5B5D002B08D0611E8C4161428905F7
:103C4000890D280005F0EEF870BD210028004C1EFB
:103C5000A14105F0D1F9F7E704060020E0050020B6
:103C6000036810B5DA0703D40D20FDF799FD10BDE8
:103C70004168581004394A425141FFF7CBFFF6E73B
:103C800010B50800FFF7ECFF002010BD37B56946FE
:103C90000A00064B30CB30C203680220042B02D14D
:103CA00001F02CF837BD01F051F8FBE730E60000D9
:103CB00010B50800FFF7EAFF002010BD10B5084C52
:103CC0006379002B05D00021052005F077F900234A
:103CD0006371052005F0A6F943425841800010BDEC
:103CE0000406002010B5084CE37A002B05D0002113
:103CF0000B2005F063F90023E3720B2005F092F925
:103D000043425841800010BD04060020A022002339
:103D10000349D2008B50034910328B507047C04684
:103D200000F0014000600040F7B52F4D2F4EEB6CC6
:103D3000002B14D0A9240023E4003759EB642C4B4A
:103D4000186800280BDB2B4B19784A425141C9B245
:103D5000197005F051F9284B1B88DF1937512B6D6D
:103D6000002B38D00021254B254FF45829653A788F
:103D70000193244D8A4206D02B68032B03D8224A94
:103D8000D05C05F039F92B68204A0133134004D583
:103D90000422013B5242134301331B4900228C464B
:103DA0002B60042B18D06046C05C591CFF2802D140
:103DB0000B000122F5E7002A00D02B60012105F05D
:103DC0001BF901233B702B68114A5B009B5A0C3492
:103DD000E418019BF450F7BD01235B422B600023E4
:103DE0003B700C4BF4E7C046FC8000400080004074
:103DF00018000020220600200C0000204C050000C6
:103E000021060020000600201C0000200300008086
:103E10000E0000205C460000084B094AFF201A8073
:103E20005A809A80DA800023064A07491370074AAD
:103E3000087048708870C870136070470E000020CA
:103E4000DC050000210600201C00002000060020E8
:103E50000122024B52421A607047C04618000020EF
:103E600010B5034A0D21034802F0D6F910BDC04633
:103E700038E600000FF00000E12170B54902194852
:103E800004F0C0FC002401220320174B17491A61DB
:103E90005C50043158508018083158501A60063070
:103EA00004F034FFFF21124AA15401341D2CFBD130
:103EB000012200200F4B01001A6004230E4A0F4D0F
:103EC0001468002CFCD02C680002013B20431160D8
:103ED000002BF5D101220A4B1A6004F04FFE01F0CD
:103EE000B1F970BDF01B0020008000400405000007
:103EF0000406002000D0004000D1004008D500405A
:103F000004D00040F8B50B4E070030000D0004F05F
:103F1000C1FC0400A84200DD2C003D00EB1B9C42CC
:103F200005DD300004F0C0FC28700135F6E7200004
:103F3000F8BDC046F01B002010B50100014804F098
:103F400069FC10BDF01B002010B5054C200004F0EA
:103F50006FFCE1212000490204F054FC10BDC04672
:103F6000F01B0020C3070CD4064B1B68834208D803
:103F7000054B1B68984204D8031F1B68002B00D018
:103F8000180070472C06002028060020002301227C
:103F900010B50A48990001334250642BFAD1084CFD
:103FA000084B00211A602000074A08F0F9FD074B72
:103FB000074A6360074B1A6010BDC046C02D002041
:103FC0003006002008000020D4090000302700003F
:103FD000340600202406002010B5044B044A1A6061
:103FE000044B054A1A60FFF7D1FF10BD2C060020D4
:103FF000300600202806002004100020044B1B6817
:104000001868000980B20238C343DB1718407047B4
:104010002406002000B59BB00200054901A809F064
:1040200003F901A802F09CFB02F0B2FEFCE7C046D7
:1040300090E700000B4BC20704D4042804D80A4BB5
:1040400000D00A4B180070470F2203681A40031D66
:10405000042AF7D0064B092AF4D0064B032AF1D0E4
:10406000054BEFE76AE700005CE2000056E2000063
:1040700074E7000084E700007BE700000020064AA8
:104080000649131F186013681B099BB202339B007B
:10409000D2188A42F5D3704734060020041000205D
:1040A000F7B50F240126314B314A1968314B324D97
:1040B000186813681F002740072F26D813681B09AC
:1040C0009BB202339B00D218AA42F2D300242B4E9B
:1040D000A500AD192868FFF745FF01342860642C5E
:1040E000F6D1274C2068FFF73DFF2060254C206863
:1040F000002802D0FFF736FF20600025224B1B6806
:104100000093009B9D4214DBF7BD1B099BB29B00F3
:10411000D3189A42D2D01F68374208D1B94206D28A
:10412000B84204D3043F3F68002F00D01F60043B17
:10413000EFE7F0236B43154A9B181A78002A01D148
:104140000135DEE71F693C2300266B43DB199B002A
:1041500001930136BB1BF3D4019BB4001C1B0B4B1A
:104160001C19A069FFF7FEFEA061F2E72C060020F3
:10417000340600202806002004100020C02D002056
:104180000800002004100020D8050020681C002032
:10419000F7B50124204246D1234B1B689C46984228
:1041A00041D3224B1B68019398423CD8031F1B68E4
:1041B000002B38D10200036800941B099BB2002B2E
:1041C0000FD10099131F196090422CD015682B1F36
:1041D0001B68990069180C68013B14600A602A008A
:1041E000EDE79D0055192968009C214219D18C45A5
:1041F00017D8019C8C4214D30E1F3468002C10D1A8
:104200000F680F343C40072C08D92F60151F2B6016
:104210000B680A601B099BB20A00D0E70099316065
:10422000CDE7013BCBE7F7BD2C0600202806002098
:104230000D4970B50A000D4D1368141F1B0926683F
:104240009BB2981C002E0BD000238A4200D00B009A
:1042500023608300C91880001218AA42ECD370BDF5
:104260001B011360F7E7C04634060020041000204D
:10427000F8B5124C27000F223B681D09ADB213425E
:104280000DD06E1CB600A74204D0320039002000C9
:1042900008F073FC0022A3190436A4191A60023531
:1042A000AD00074B7F199F42E5D31B1B9B10013BC1
:1042B0001B012360034B1C60F8BDC0463406002080
:1042C0000410002024060020F0B59BB0FFF728FC66
:1042D00000240700214AA300D0580134FFF758FFFB
:1042E000642CF7D11E4B1868FFF752FF1D4B18685E
:1042F000002801D0FFF74CFF00261B4B1B689E4295
:1043000017DBFFF795FFFFF7CBFEFFF7B1FFFFF7D6
:1043100007FC164BC21B1B6815491B6801A81B092B
:104320009BB2023B08F080FF01A802F019FA1BB013
:10433000F0BDF02575430F4BED182B78002B01D104
:104340000136DAE72B695C1E002CF9DBA300EB18C1
:104350009869FFF71DFF013CF6E7C046C02D00201D
:104360000800002004100020D805002024060020AA
:104370004AE70000681C0020F7B5174D4F1C2B685A
:1043800006001B680C001B099BB201929F420BDBCD
:10439000FFF79AFF2B681B681B099BB29F4203DB48
:1043A0000A20FDF7FDF9FEBD2868A71CBA00DB1B3B
:1043B00081181B010B6029600021031F19600F2366
:1043C0001E4003002401264340C3083A9A189A422B
:1043D000E9D9019902C3FAE724060020F7B50300E2
:1043E0000122134004000D000193002B2BD1174B29
:1043F0001B68834227D8164B1B68834223D90F239F
:10440000144F386000681840FFF7B6FF019B3C6806
:10441000061E3B6017D0236804301B099BB29D42E7
:1044200000DD1D00AA00211D251F08F09DFBFFF7E0
:1044300025FE2E60FFF734FE00232B602268064B1A
:104440001340236034002000FEBDC0462C0600202F
:104450002806002004100020F0FF0F000323043082
:1044600010B5C11719400918891000220420FFF760
:1044700083FF10BD70B5050008000C00FFF7EEFFCC
:104480000023002804D170BDE95CC218117101330A
:10449000A342F9DBE343DB171C400023041923711B
:1044A000F1E7F0B50C009BB0022804DC1C20FDF7FE
:1044B00077F91BB0F0BD01230868184206D1042823
:1044C00004D90F2601683140042901D00E20EEE7FF
:1044D00061680D001D40F9D10429F7D90A683240FE
:1044E000042AF3D1A2681A4201D10D20DFE7FFF7B9
:1044F000A1FD06006068FFF79DFDA768010001AC03
:104500007F103000257003F0A7FD390064232200DE
:1045100003F007FE200008F0CDFE01002000FFF7A9
:10452000A9FFC6E710B51C4CA544041E02D1FFF735
:1045300095FF0BE003F0A8FC0138062828D806F008
:104540004DF9090911182904240000208023DB00FB
:104550009D4410BD200003F013FD011B2000FFF758
:1045600089FFF3E7200003F0B9FC43000120184362
:10457000ECE780226946D200200003F0C6FC6846C2
:1045800008F098FE01006846E9E704210348E6E7E1
:104590000020CCE70420D9E700FCFFFFF0E7000093
:1045A00070B50C00022803DC1C20FDF7F9F870BD83
:1045B00001230868184206D1042804D90F25016890
:1045C0002940042901D00E20EFE761681942FAD191
:1045D0000429F8D90A682A40042AF4D1A2681A42A8
:1045E00001D10D20E1E7FFF725FD05006068FFF729
:1045F00021FDA46801006410280003F02DFD2100B6
:1046000003F06AFDFFF78EFFD1E770B50D000128BA
:1046100003DC1C20FDF7C4F870BD012408682042AB
:1046200006D1042804D90F2102680A40042A01D0C7
:104630000E20EFE76A682242FAD1042AF8D91368FB
:104640000B40042BF4D1FFF7F5FC06006868FFF778
:10465000F1FC0100300003F0FFFC03F081FD40009D
:104660002043D9E7F8B507000C001C20012F0BDD13
:1046700001250868284206D1042804D90F210268C0
:104680000A40042A03D00E20FDF78AF8F8BD6268BC
:104690002A42F8D1042AF6D913680B40042BF2D130
:1046A000FFF7C8FC06006068FFF7C4FC0100022F9A
:1046B00014D0A4682C4211D06410300003F0CCFC5C
:1046C000050003F0E1FB012811D1002C02DD0135CA
:1046D000012C06D12800FFF725FFD7E7012464420B
:1046E000EBE7280003F059FC013C0500F0E7022845
:1046F000F0D1002CEEDD0135012CEBD0002228009A
:10470000110003F07CFC03F048FC013C0500F3E7DA
:10471000086870B501240500254006D1042804D995
:104720000F2302681340042B03D00E20FDF738F846
:1047300070BDFFF77FFC03782900233B5A425341A9
:104740001022C01808F07EFE80239B05C218044B7F
:104750009A4201D91420E9E740002043E8E7C04627
:10476000FFFFFF3F10B50124044002D04410200099
:1047700010BD042810D90F2302681340042B07D161
:10478000FFF758FC21000A2208F05CFE0400EEE767
:10479000032B01D10430F5E70D20FDF701F8E6E722
:1047A00010B50868FFF7DEFF08F0C6F804F090FDCA
:1047B000054B002207F0B4FA04F0EAFC08F086F892
:1047C00043000120184310BD00408F4010B5086819
:1047D000FFF7C8FF06F034FB094906F0FFF908F0BF
:1047E000E5F804F02DFD074B002207F099FA04F0DC
:1047F000CFFC08F06BF843000120184310BDC04601
:10480000D30237390000D040F7B50C00042803DC90
:104810001C20FCF7C5FFFEBD0868FFF7A3FF019051
:104820006068FFF79FFF0600A068FFF79BFF050089
:10483000E068FFF797FF07002069FFF793FFAE429C
:1048400001D11F20E5E7019BC01B9B1B5843A91BFF
:1048500006F062F8C71901207F003843DBE700004B
:1048600010B5034A0921034801F0D6FC10BDC0462B
:10487000A8E70000A1E700000020704710B51E2047
:10488000FCF78EFF10BD10B51E20FCF789FF10BD90
:1048900010B51E20FCF784FF10BD10B51E20FCF7DC
:1048A0007FFF10BD10B51E20FCF77AFF10BD10B5BC
:1048B0001E20FCF775FF10BD10B51E20FCF770FF21
:1048C00010BD10B51E20FCF76BFF10BD10B51E20EB
:1048D000FCF766FF10BD10B51E20FCF761FF10BD90
:1048E00010B51E20FCF75CFF10BD10B51E20FCF7B4
:1048F00057FF10BD10B51E20FCF752FF10BD10B5BC
:104900001E20FCF74DFF10BD10B51E20FCF748FF20
:1049100010BD10B51E20FCF743FF10BD10B51E20C2
:10492000FCF73EFF10BD10B51E20FCF739FF10BD8F
:1049300010B51E20FCF734FF10BD10B51E20FCF78B
:104940002FFF10BD10B51E20FCF72AFF10BD10B5BB
:104950001E20FCF725FF10BD10B51E20FCF720FF20
:1049600010BD10B51E20FCF71BFF10BD10B51E209A
:10497000FCF716FF10BD10B51E20FCF711FF10BD8F
:1049800010B51E20FCF70CFF10BD10B51E20FCF763
:1049900007FF10BD10B51E20FCF702FF10BD000080
:1049A00010B5034A1E21034801F036FC10BDC04675
:1049B00048E8000038E900000120034B1860034B71
:1049C0001B68834018437047241000200810002003
:1049D000F0B5EFF310810123194083F31088134AD7
:1049E000A1261268124D013A9340A022114FD20520
:1049F000F600002B17D02C68945103420BD0C04610
:104A0000C046C046C046C046C046C046C0462C68E8
:104A1000D4515B08EDE7D451C046C046C046C046FD
:104A2000C046C046F5E781F31088F0BD20000020A5
:104A3000141000200C05000030B585B001AD0C222B
:104A40000649280008F090F80024285D012101346F
:104A5000FFF784F80C2CF8D105B030BDC5EA000092
:104A600030B585B001AD0C220649280008F07CF86D
:104A70000024285D00210134FFF770F80C2CF8D1D8
:104A800005B030BDC5EA0000F7B56A463B4B01AE44
:104A900013800A2393703A4B33801C23B370FFF7C3
:104AA0003FF8384B384DC0182B68984201D200238C
:104AB0002B602C68002C41D1375D01213800FFF7B5
:104AC0004DF801340021380004F096FA032CF3D19C
:104AD000002401276B461E5D39003000FFF73EF8C9
:104AE00001343900300004F087FA032CF2D1C820D9
:104AF0000138C046C046C046C046C046C046C04653
:104B0000C046C046C046C046C046F1D16B460021F3
:104B10001878FFF723F86B4600215878FFF71EF846
:104B20006B4600219878FFF719F8FEF7F9FFFA2392
:104B300000241B01C01828602000FEBDFEF7F0FF16
:104B40002B6800249842F7D3032004F0E5F8060010
:104B5000042004F0E1F836180A2004F0DDF80B4BCD
:104B60009B1B181A0A4BA04206DB18600023094A57
:104B70002B6013600124DFE71C60F7E703040000EB
:104B80001A1B0000102700001C100020E303000087
:104B900008100020241000200022054B10B51A60D8
:104BA000044B1B68934201D003F00EF9002010BDA6
:104BB00020100020141B002010B5041E0CDA002465
:104BC000084BA400E2581F231A401E3B9340064A9C
:104BD0001360064A136010BDFEF7BEFFA042EEDD73
:104BE000EEE7C046ECF80000141000201805005055
:104BF0000200086810B5C3070FD540101823012A1A
:104C000003DD4A68042A00D10833054A1360FEF721
:104C1000C9FFFFF7D1FF002010BD01204042EDE7A2
:104C20002000002010B500280CDD0A68131F591E53
:104C30008B4107490B60042A06D0FFF711FF0022C1
:104C4000044B1A60002010BDFFF7F6FEFAE7C046DD
:104C5000181000200810002010B50124044002D0D4
:104C60004410200010BD042810D90F2302681340FF
:104C7000042B07D1FFF7DEF921000A2208F0E2FB3E
:104C80000400EEE7032B01D10430F5E70D20FCF71B
:104C900087FDE6E70868F8B5C3071AD5FFF7DCFF1C
:104CA0000300203B5E2B25D80520434301221D181D
:104CB0000020114E9D4219D005211024F75C3C4282
:104CC00000D080180139520064100029F7D1013357
:104CD000F0E704280ED90F2203681A40042A09D1EC
:104CE0001B099BB2002B05D00379DAE701234000B2
:104CF0001843F8BD0120FCE7D1EA000070B5086850
:104D00000D00FFF7A9FF04006868FFF7A5FF621E0A
:104D10000100042A14D8451E042D11D805236B4325
:104D20009B18012215009D402B00064805682B4367
:104D30000360054B1B68002B02D0200003F045F8F0
:104D4000002070BD20100020141B002070B50868E2
:104D50000D00FFF781FF04006868FFF77DFF621E0A
:104D60000100042A13D8451E042D10D805236B43D7
:104D70009B1801229A400748036893430360064B3F
:104D80001B68002B03D00022200003F01EF8002037
:104D900070BDC04620100020141B0020F0B5050097
:104DA00089B008680C00FFF757FF0690022D36DD2A
:104DB0006068FFF751FF0190A068FFF74DFF040006
:104DC0000127231D661E0793731C0293079B9E42B7
:104DD00035D0052373430593019B019D053304934F
:104DE000049BAB421ED0042E16D86B1E042B13D886
:104DF0000122059B2349013B5B199A409446224AB4
:104E00000B681068069A3A4003920DD062461A4326
:104E10000A60012200280DD17F000135E0E701245E
:104E20000194CDE7029ECFE7624693430B600028D2
:104E3000F2D0039A0299280002F0C7FFECE7019B29
:104E40001E1D042E1AD8012C18D1002505273B0061
:104E500021006B439B1999400B000A4A01351168E8
:104E60009943094B11601B68002B05D0019B002260
:104E7000581D290002F0A9FF052DE8D1002009B036
:104E8000F0BDC04620100020141B0020F0B53B4BA5
:104E900085B01B680C00002B03D101204042FFF7B6
:104EA0008BFE012627683E403CD1042F3AD90F23C0
:104EB0003A681340092B35D17B685B100293029B43
:104EC0009E4258DAB300FB189868FFF7C5FEFF232F
:104ED00005000414001218401C4029492B4040438F
:104EE000019305F019FD0304200025496043039355
:104EF00005F012FD039C0002044301982049404341
:104F000005F00AFD1F4B20431B68202B06D1AD0086
:104F1000AD0E1D4BAD00EC5800022043FFF758FDCD
:104F20000136CCE73800FFF797FEFF26050007148F
:104F3000001230401249404305F0EEFC37400404B3
:104F400038000F49784305F0E7FC2E400002044387
:104F500030000B49704305F0DFFC0A4B20431B680F
:104F6000202B06D1AB009B0E074A9B009B580002EA
:104F70001843FFF72DFD002005B0F0BD14100020F0
:104F80005906000020000020ACEC0000086810B5B5
:104F9000C30703D5FFF760FE054B1860054B1B6880
:104FA000002B03D0024B186802F010FF002010BD48
:104FB00020100020141B00209D4B70B51B68002B97
:104FC0000DD19C4C2368002B0AD19B4A1268002A01
:104FD00006D19A4B1B68002B01D0FFF755FD70BD21
:104FE000974D2A68002A1BD1944A1268002A10D0D3
:104FF000FFF74AFD0028F2D0FFF71EFD8E4B226816
:1050000019681A6000290BD0002A09D1FFF728FD82
:10501000E5E7894A1268002AF0D1002BEED0EBE7D1
:1050200000211A2003F0E8FF00211B2003F0E4FF19
:1050300000211C2003F0E0FF2E68012E5CD0022E20
:1050400000D1A2E0002E50D1013631007A4C03206D
:105050002368994303F0D0FF0420216801404B42AC
:10506000594103F0C9FF102123680A2019404B421F
:10507000594103F0C1FF80212368090119404B42C7
:105080005941062003F0B8FF802123680902194026
:105090004B425941072003F0AFFF802123684902AA
:1050A00019404B425941092003F0A6FF8021236893
:1050B000890219404B425941192003F09DFF80217C
:1050C0002368C90219404B425941182003F094FF4C
:1050D000802321681B0319404B425941172003F0DC
:1050E0008BFF31001A2003F087FF2B680321581C27
:1050F00005F0F8FC296072E702214F4C1720236865
:1051000019404B42594103F077FF082123681820CA
:1051100019404B42594103F06FFF80212368C900B9
:1051200019404B425941042003F066FF8021236857
:10513000490119404B4259410A2003F05DFF80218B
:105140002368C90119404B425941032003F054FF21
:1051500080212368890319404B425941092003F0FB
:105160004BFF802321681B0419404B4259411920F1
:1051700003F042FF3100062003F03EFF310007201C
:1051800003F03AFF31001B20ADE720212A4C172005
:10519000236819404B42594103F02EFF40212368F8
:1051A000182019404B42594103F026FF8021236803
:1051B000192019404B42594103F01EFF80212368FA
:1051C000490019404B425941092003F015FF802145
:1051D0002368890019404B425941072003F00CFF16
:1051E00080212368890119404B425941062003F070
:1051F00003FF80212368490319404B4259410A208B
:1052000003F0FAFE80212368C90319404B4259413B
:10521000032003F0F1FE802321685B0419404B4218
:105220005941042003F0E8FE01211C205BE7C04641
:105230001810002020100020101000202410002042
:105240000C100020012010B54042FFF7B5FC10BD46
:1052500010B5034A0A21034800F0DEFF10BDC04626
:10526000ACED0000FCED00008023F0B502255B05ED
:105270001A690A4C0A4BA1261D5103278025F60006
:10528000ED00BA43884202D300221A51F0BD5F59A3
:10529000002FFCD098518018F4E7C04604050000A8
:1052A00000E0014010B5002806D1C020B021400226
:1052B0008902FFF7D9FF10BDB02080218002C9020A
:1052C000F7E7000043425841064B40421840B023E4
:1052D0009B02C018036800201A0E532A01D11B023A
:1052E000180A704700C0FEFF30B501248025054B29
:1052F000054AED009C505C59002CFCD00160002157
:10530000995030BD00E0014004050000434258417F
:10531000074B40421840B0239B02C018A62310B58B
:105320000902DB05090A1943FFF7DEFF10BDC0467D
:1053300000C0FEFFF0B5012480260D4B0D4DF60098
:105340005C51002902DC00225A51F0BD57781478D4
:105350003F022743947824042743D4780432240658
:105360003C439F59002FFCD010C00139E9E7C046EB
:1053700000E001400405000070B505004B680A001C
:105380009C1C2100A400FFF7D5FF281970BD000068
:10539000134B1B68002B0CD08022B023D2029B023F
:1053A00000280BD11A1D5B681B0E522B00D1100078
:1053B0007047B022C02392025B02F1E782420DD90E
:1053C00003681B0E522B09D1436802339B00C0189F
:1053D000824203D903681B0E522BE9D00020E7E775
:1053E00028110020F0B50020B7B00024FFF7D0FF4F
:1053F000270005002600002D2ED1284D2868FFF734
:1054000061FF32003B0001900094254904A807F099
:105410000BFF04A801F0A4F9224B64201C682B6840
:10542000A0215A425341204A5B421340B0229202CB
:105430009B18E41A6043490205F06EFAA02252025A
:10544000030000921949220004A807F0EDFE04A809
:1054500001F086F937B0F0BDFF226B6829689C46E1
:105460000233FF180B12013613409C4200DA1C0075
:10547000FF200A140240039262460140019200910B
:10548000039A0B4904A807F0CFFE04A801F068F9BD
:105490002800FFF77DFF0500ADE7C046281100207A
:1054A00016EF00002C11002000C0FEFFC0EE00002F
:1054B00002EF000070B50020FFF704FF0400012098
:1054C000FFF700FF844200DA04000A4B1D686A42BD
:1054D000554128001D60FFF7E5FEA0226B425202F5
:1054E0001340054A28009B18044A611C1360FFF70B
:1054F0000DFF70BD28110020048001002C11002038
:10550000F8B50020FFF7DEFE07000120FFF7DAFE06
:105510003E00204D0643204C0DD18021C020C90201
:105520004002FFF7A1FE01213000FFF7EFFE1B4B09
:105530002E6023601DE0874209DD0023B0212B602F
:10554000164B8902236023680020012517E0012300
:1055500080212B60124BC9022360F4E7120E522AFD
:1055600008D0002800D023600E4801F0F9F8FFF7BA
:10557000A1FFF8BD28005A68023292009B188B42A6
:1055800005D21A68561CE9D10028F2D0D1E7216073
:10559000EFE7C046281100202C11002004800100F4
:1055A00004C00200DBEE000070B50020FFF7F0FE43
:1055B000FF260500002801D1280070BD03681C14D7
:1055C0003440FFF7E5FEDA2CF4D10500F2E70000E5
:1055D000FF2270B51F4CD2000021200007F0E0FA36
:1055E000FF25FFF7E1FF0026002818D1F0210A224D
:1055F000194849420B00962553432D011B185D198C
:105600002D78002D07D0154D154E5D199B191B786F
:10561000DB00E3582B60013A002AEBD170BD036830
:105620001A142A400A2A0AD11A122A40FF2A03D041
:10563000D200A1180B71A050FFF7AAFED4E7132ADD
:10564000FAD11B122B40FF2BF6D0DB00E2181671AB
:10565000E650F1E7C8250020681C0020680900001A
:105660006109000010B59AB0FFF74AFFFFF7B0FFDD
:1056700000231A000A48D900415801334C1EA141A9
:105680005218FF2BF7D1074901A807F0CDFD01A85B
:1056900001F066F8044801F063F81AB010BDC04686
:1056A000C82500204BEF00005FEF00008022F0B51E
:1056B0005200A1B00021684807F072FA8022002150
:1056C0005200664807F06CFA654BFF271B681A000A
:1056D000049353425A4110000592FFF7E3FD049CE6
:1056E0000020631E9C415F4B64421C405E4BE418EB
:1056F000FFF75AFF0600002E2FD10498FFF7E2FDB6
:10570000411C0598FFF702FE059A554B574D1A604C
:105710002C60FFF75DFFFEF717FC514B64201B6800
:10572000A0215A4253414F4A5B421340B0222C6899
:1057300092029B18E41A6043490205F0EDF8A0229A
:105740005202030000924A49220007A807F06CFDAC
:1057500007A801F005F821B0F0BD32681314121249
:105760003A403B4003921A000A3A092A49D83A4B78
:10577000039A995C002931D110223E4807F010FAB3
:1057800035002B6803991A123A40914209D11A1434
:105790003A400B2A27D0132A2DD00A2A01D1354BA3
:1057A0001D602800FFF7F4FD051EEAD1314B196892
:1057B00000290FD02000FFF7DFFD04002D4B5B19FF
:1057C0005968002903D02000FFF7D6FD04000435F6
:1057D0000C2DF3D1204B0121039A99543000FFF78F
:1057E000D7FD060087E73B40022BDADC214A9B000D
:1057F000D3185D60D5E7102200211E4807F0D0F9CC
:10580000CFE71A00153A082AE8D8144A0399525CDF
:10581000002AE3D13500152B00D0150030000368B5
:105820001A143A40152A0FD01D2A00D10025FFF77F
:10583000AFFD0028F3D1002D04D020002900FFF790
:105840009BFD0400054BC6E7039A1B123B409A429E
:10585000EDD10500EBE7C0462810002030110020F4
:105860002811002000C0FEFF04C002002C110020FF
:10587000A5EE0000502F002010B5FFF717FF10BD58
:10588000F0B585B0039203220333DC17294D144091
:10589000E4182B68284F5A42534180225B42D202BF
:1058A000A4103B409B18A21C0291244E9100009131
:1058B0000190316800980A18934215D2FFF7F6FE5E
:1058C0002B685A42534180225B421F40D202BF18CC
:1058D0003368009A9B189F4206D2194800F040FF97
:1058E0000025280005B0F0BD029B356819066B46FF
:1058F0001A7BA423DB051343FF222F00090C194355
:10590000019B12041B04134019432800FFF7ECFC11
:105910000837281D21003760FFF7E6FC002C04D073
:105920000A9A21003800FFF705FD009B083BFF188D
:105930003760D6E72811002000C0FEFF2C110020A0
:105940007FEE0000704770470021094B094A5960FB
:105950000131516059680029FCD0002119610123EF
:1059600093600222044B8131FF315A501A60704714
:10597000FC1000400010004000E100E00222064B55
:105980000121DA670022054B5A61054A11615A6903
:10599000002AFCD07047C04604E100E0FC10004043
:1059A0000010004010B5044C2378002B01D0FFF705
:1059B000E5FF0020207010BD311200200120024BB5
:1059C0001B685B0018437047B41200200120024B93
:1059D0001B685B0018437047240000201FB5064B6E
:1059E00006491A6801A807F01FFC082101A8FEF764
:1059F00041FD05B000BDC046B8120020F0EF000028
:105A00001FB580235B051A6E044901A807F00CFC42
:105A1000082101A8FEF72EFD05B000BDF0EF000043
:105A200010B5044C200007F045FC01002000FEF7F3
:105A300021FD10BDBD1200200E4B10B51B680E4C91
:105A40005A1C0FD00D4C002B0CD00D4C012B09D043
:105A50000C4C022B06D0094C042B03D00A4C052B0E
:105A600000D1074C200007F025FC01002000FEF7C4
:105A700001FD10BD28000020F5EF000010E6000039
:105A800000F0000017E60000FAEF000070B5040017
:105A90000D001600FEF74EF88023012200215B0561
:105AA0001B6E6270E270020AA271020CE2711A0AA5
:105AB00060716372000EA2721A0C1B0E26702571A3
:105AC000A1702072E272237370BD000070B5214C8A
:105AD0002278002A3DD1204B01215A608022D20534
:105AE00011605A68002AFCD0002207201B4B1C4979
:105AF00001255A500439585008315A5019481A494A
:105B000058501A491A485A501A495A50A622D200D7
:105B10009D50082218495A50043158500220174904
:105B200058501749174858501748043958501820EA
:105B300016495850C12189005A500539FF39585823
:105B4000921802435A501249124A9950FFF7FCFE2C
:105B5000257070BD31120020FC0000400010004094
:105B60000C050000746962751C0500002405000026
:105B7000200004022C05000014050000340500007C
:105B80003C050000FFFF000021100100540500004B
:105B9000321200200405000013B5094B04000093E5
:105BA000084B019307280AD8074B1B78002B01D11B
:105BB000FFF78CFF6B46054A1957054BD15013BDB3
:105BC000E2ECF0F4F8FC0004311200200010004078
:105BD0000C05000070B50E4B06001B78002B01D1A0
:105BE000FFF774FF00200B4D2C7884420ED00A4B37
:105BF000202219780323091B1940084B4901C918B1
:105C0000300006F0B1FF0120013C2C7070BDC04691
:105C100031120020BC12002030120020321200206D
:105C2000002370B588B0984235DD0D6801262C0040
:105C300034409C422FD12300042D2CD90F222B68F5
:105C40001A402300092A26D16A683F2A23DD6846C4
:105C5000FFF7C0FF230000281DD06B4619783300E2
:105C6000A14203DB6B461B5D5B003343A200AA1815
:105C700001349360202CF2D1092169444A780B78D1
:105C800012021A438B781B041A43CB781B0613436A
:105C9000024A13600423180008B070BDB812002037
:105CA00070B5454B8AB01B78002B01D1FFF70EFF72
:105CB00002AC2000FFF78EFF002802D100200AB0BE
:105CC00070BD23780B2BF9D96378012BF6D1E378DB
:105CD000012BF3D100231120384E394D33602B7046
:105CE00068442379374A41781360027809021143E6
:105CF000827812041143C27812060A4332490A60BC
:105D0000002B0ED1152169444A780B7812021A43F0
:105D10008B781B041A43CB781B0613433360002394
:105D200018E0012B1AD1152169444A780B78120228
:105D30001A438B781B041A43CB781A211B06134392
:105D400033600E23627C6944934200DD130000221D
:105D50009A422CD100220420EA54B0E7022B03D14E
:105D6000627B10331621EEE7042B0DD1152108229A
:105D70006944684606F0F8FE0098019903F078F946
:105D800006F0A4FD3060CAE7052BC8D11521082212
:105D90006944684606F0E8FE0098019903F068F946
:105DA00006F094FD3060627D0A231E21CBE7885CFB
:105DB000A8540132CCE7C04631120020B4120020B2
:105DC000BD12002028000020B812002010B5134B8F
:105DD00004001B78002B01D1FFF778FEFFF7CEFD02
:105DE00000200F4A0F49104B54505860013010608A
:105DF00058680028FCD000201861013090601869B4
:105E00000028FCD0094B0A481B785B011B18535033
:105E1000FFF7B4FDFFF798FD10BDC046311200201A
:105E20000010004004050000FC100040301200206B
:105E30003212002010B588B000281DDD0A6801214B
:105E400013000B4018D1042A16D90F2014682040E3
:105E5000092811D150683F280EDD9800101880687D
:105E60000024084201D04010C4B26846C454013333
:105E7000202BF2D1FFF7AAFF002008B010BD0000D0
:105E800010B5002813DD0C68E30710D56410532CFF
:105E90000DD8084B1B78002B01D1FFF717FEFFF739
:105EA0006DFDA123044ADB00D450FFF74DFD002017
:105EB00010BDC046311200200010004010B500286F
:105EC0000EDD0C68E3070BD56410FF2C08D8054BDA
:105ED0001B78002B01D1FFF7F9FD034A034BD45087
:105EE000002010BD311200200010004024050000E9
:105EF00010B5002805DD0868C30702D54010FFF77C
:105F00004BFE002010BD70B588B0002820DD0124B4
:105F1000086804401CD104281AD90F2302681340D2
:105F2000042B15D1FEF786F8060007F0C3F905002B
:105F3000122800D912252A0002210D326846FFF7E7
:105F4000A5FD6B465D73A54205DC6846FFF73EFF85
:105F5000002008B070BD2300325D6B449A73013499
:105F6000F1E7F0B50D008BB0012832DD08680122A1
:105F7000040014402DD104282BD90F2301680B40B5
:105F8000042B26D16B68134223D0FEF753F86E68BA
:105F900007007310019307F08DF905000E2800D952
:105FA0000E252A000121113202A8FFF76FFD6A4673
:105FB000127902AB5A7302AA73129373019B76147F
:105FC0001B0ED67313745574A54205DC02A8FFF7A7
:105FD000FDFE00200BB0F0BD3A5D02A963189A7473
:105FE0000134F1E730B589B0002814DD0C68E3070F
:105FF00011D5102268460021FFF748FD6B466A461E
:1060000065105D73684663122D0E64149373D47328
:106010001574FFF7DBFE002009B030BD174B184A9E
:106020005968002903D00021596001319160196934
:1060300000291FD0002018618023DB00D3581149AC
:10604000012B18D1A923DB00D3585B420B600E490A
:106050000B78032B01D801330B7003200B490B780D
:10606000013303400B700A495B015B180949535027
:106070000123936070470860FAE7C046FC100040B7
:106080000010004024000020BC120020301200202C
:10609000321200200405000010B50A4B1B78002BBB
:1060A0000ED0FFF76BFCA1230722074CDB00E25068
:1060B000FFF74AFC0022054B0620E250FFF76CFD7B
:1060C00010BDC04631120020001000402405000021
:1060D00010B5034A1021034800F09EF810BDC046D9
:1060E00070EF000067EF0000044A05491368C854C8
:1060F00001339B059B0D13607047C046F0160020CE
:10610000F012002070B5124C124A2368834202DC60
:106110000023236018E0115C451C0E00FA3E012E9E
:1061200007D8AB4211DD515D002902D028399F29E3
:1061300001D82800EAE70100151A565C6E540131B7
:106140008B42FADC181A206070BD1170FAE7C04665
:10615000FC1A0020FC16002010B5FDF7E1FC064BF0
:106160001A68824201D900221A601B68C31A0348C8
:1061700098428041404210BDE8120020204E0000AD
:1061800070B5FFF711FAFF250400002801D12000A7
:1061900070BD03681B142B401D2B00D10400FFF7BA
:1061A000F7F8F2E770B5002601250D4C0D4A23687B
:1061B0001268934205D00C4AD05CFDF7BDFE002862
:1061C00006D1002E03D0FDF7B5FC084B186070BD5A
:1061D00023682E0001339B059B0D2360E5E7C04635
:1061E000F4160020F0160020F0120020EC1200201F
:1061F00010B50400064B074A1B6812689B1ADB4364
:106200009B059B0DA34200DB10BDFFF7CBFFF1E721
:10621000F0160020F416002070B5074E33680B2BE3
:1062200008DC0C255D43054C01332851641961607D
:10623000A260336070BDC046F8160020602F0020B9
:10624000F0B5B7B0040007F035F8012802D80020F7
:1062500037B0F0BD23785B2BF9D1013825182B78A6
:106260005D2BF4D101343A21200007F00BF8061E13
:10627000EDD0071B002FEADD210000243A0004A81E
:1062800007F030F804AB711CDC556F1AA742DEDD55
:106290001DAD3A00280007F025F8134BEC551B689C
:1062A00003950193019BA342D1DD0C2666430F4B5E
:1062B00004A9F618306806F0F3FF051E05D17368CF
:1062C000B6680293029B9D4201DB0134EAE7306825
:1062D000039906F0E5FF37000836002801D17868F9
:1062E000B6E70135EEE7C046F8160020602F002023
:1062F00010B5FBF789F8FEF7ABFFFBF7AFF8FDF73A
:10630000AFFDFEF7ADFAFEF74BFBFFF7E1FE01F044
:10631000F3F801F02DFD01F05BFD01F0A5FF10BDCC
:10632000962210B512010021034806F039FC002224
:10633000024B1A6010BDC046681C0020D805002022
:1063400070B514007F22174BC000C0580D00836841
:1063500013401C2B01D0002070BDC36819001140F0
:106360000429F8D101690A40192AF4D11B0A013322
:106370009B000C30C018FDF75DFE0378060001207D
:10638000002BE9D0300006F095FF0023A042E2D1B7
:10639000A34201DB0120DFE7F15CEA5C9142DAD144
:1063A0000133F5E7C825002010B5FDF7C3FB064B08
:1063B0001A68824201D900221A601B68034AC31A74
:1063C00000209A42404110BDEC120020CF0700008F
:1063D000064B074A1B6812689B1ADB439B059B0D03
:1063E0000122834200DC002210007047F0160020DA
:1063F000F4160020F8B505000C0016001F1E0ED183
:106400000320FFF7E5FF002808D0FA20FFF76CFE15
:10641000E8B2FFF769FEE0B2FFF766FEF8BD501D77
:10642000FFF7D6FF0028F9D0FB20FFF75DFEE8B2AA
:10643000FFF75AFEE0B2FFF757FEF0B2FFF754FE47
:106440003012C0B2FFF750FE3C00E31B9E42E5DD78
:106450002078FFF749FE0134F7E7000070B500240B
:10646000F0250B4B1B68A34202DCFFF759FF70BD00
:106470002B006343074A9B181A78002A05D05978E5
:10648000002311201A00FFF7B5FF0134E9E7C046E9
:10649000D8050020681C0020F8B507000024F0256E
:1064A0002B0063430C4A01349E18B74211D0317857
:1064B00000290BD00133D15C002311201A00FFF713
:1064C00099FF2A000021300006F06AFB0A2CE7D170
:1064D000F8BD024B1C60F9E7681C0020D8050020BD
:1064E000F0B5150001222F007A4C1740A544019009
:1064F0000291002F11D005AB1A706A105A70120E5B
:106500001A710522691299706D140299DD70FFF7F6
:1065100071FFCF239B009D44F0BD042D2AD90F2489
:1065200028680440042C32D1022304AA28001371E5
:10653000FDF780FD050006F0BDFEC82302009B00AC
:10654000984200DD1A007C1C97420DD1984206D972
:10655000614804AB03226149C01806F005FB220024
:1065600005AB02990198D2E72700611E695C05AC72
:10657000E155E8E7042D00D0A7E0032304AA043D79
:1065800013716B425D4105AB55710222E9E7092C9D
:106590007ED1042205AB1A706A68511000916946D9
:1065A000521209789A70009A59701F2A01DD202230
:1065B00000926A46127806ACDA70009BBB4202DC9D
:1065C00005ABE21ACDE70126BB00EB189868064040
:1065D00006D1042837D90F210368194002290CD1AC
:1065E000012323704310637042121B0E4014A270EB
:1065F000E070237105340137DFE7042921D102233C
:106600002370FDF717FD039006F054FEA31C0C2821
:1066100009D86070864201D19C19ECE7039A925D1B
:106620009A550136F6E70C226270039A925D9A55EC
:106630000136092EF9D12E23E372237363730E34CE
:10664000D9E7012907D10323043823704342584175
:1066500060700234CFE7092909D10423237043680D
:106660005A1062705B12A370E6700434C3E703290A
:106670000BD1052323700068020992B2430F9200E8
:106680000B40D31A63701B12EDE726700134B2E79A
:10669000032C00D03DE7052205AB01091A7089B231
:1066A000420F890022408A1A11125A709970642A86
:1066B00000DD64220421DA70081F824201DC04320A
:1066C0004FE7685C58540131F6E7002D00D020E711
:1066D00053E7C046C4FCFFFF2203000066E200004F
:1066E00070B502000024F0210D4E080060438019AF
:1066F0004578954203D001340A2CF6D170BDF022C2
:10670000002106F04DFA074A1368013BA34200D16D
:106710001460002329001A001120FFF76BFEEDE73B
:10672000681C0020D805002010B5B2B002236A46CC
:106730000400137006F0BEFDC72800D9C72000234F
:10674000984207DC421C6B46FE211420FFF752FEE4
:1067500032B010BD694601335A1EA25CCA54EFE73D
:1067600030B5B3B00500FFF71FFE002816D0022396
:106770006A462800137006F09DFD0400C72800D962
:10678000C7240023A3420BDB20003230FFF730FD8B
:10679000621C6B46FF211420FFF72CFE33B030BD86
:1067A000694601335A1EAA5CCA54EBE7F0B5BDB086
:1067B00005900C00012803DC1B20FAF7F1FF55E0DF
:1067C0002C4B08680393C30709D4042807D90F2367
:1067D00002681340042B02D1FDF72CFC0390254BDB
:1067E00060680493C30709D4042807D90F230268FB
:1067F0001340042B02D1FDF71DFC049000261E4B14
:106800001B680893089BB3420BDC049B1B4A009354
:10681000C821039B0AA806F0D5FC0AA8FFF7A0FF31
:10682000CAE70C257543164B0399ED18286806F046
:1068300037FD071E05D16B68AD680993099B9F4220
:1068400001DB0136DEE728680499079506F028FD8C
:106850000835069000280BD121000598079B0831C8
:106860005B6802389847074B069A1A603DB0F0BD46
:106870000137E3E7A0E70000F8160020D1F00000A0
:10688000602F002004100020F7B5234B06001B6882
:10689000F02100930023009A9A4211DC0024F02397
:1068A0001A006243019201991C4A55182F78002F53
:1068B00012D001340A2CF3D11948FFF751FF29E017
:1068C0000A005A43154882185078B04202D1127813
:1068D000002A1FD10133DEE7F0223900280006F03C
:1068E0005FF902230D4A0199EB6053540D4AF10000
:1068F0008A58009B6E70AE70AA602F616F61A342D0
:1069000002DC054B01341C60002331001A0010200A
:10691000FFF770FDF7BDC046D8050020681C0020B9
:1069200019F50000C825002010B5FFF797FDFF24DA
:10693000084AE3005B429B18074AD35C043B012BE7
:1069400003D8E043C0B2FFF79FFF013C002CEFD11A
:1069500010BDC046FC070000C8250020F8B50500A2
:106960000E00FDF787FDFF240D4B18600D4AE30074
:106970005B429B180C4AD35C062B01D0032B0BD136
:10698000E743FFB2320029003800FFF7D9FC0028A6
:1069900002D03800FFF778FF013C002CE6D1F8BDAB
:1069A00008000020FC070000C825002070B5050085
:1069B000FF24084AE3005B429B18074AD35CAB42C2
:1069C00003D1E043C0B2FFF75FFF013C002CF0D1E0
:1069D00070BDC046FC070000C8250020F7B5FDF7D4
:1069E0009FF8574B1A68824201D900221A601A6830
:1069F0005449821A8A420DD9FF2253491860D300A4
:106A00005248CB1A1B181B78073B022B0CD9013AB2
:106A1000002AF4D1F7BD0720FFF7C8FF4C4B27E051
:106A20000820FFF7C3FF38E0FDF784F8071E00D108
:106A300001270020FDF742F901900020FDF752F9EF
:106A4000019B0090434C444D002B12D02368002B37
:106A50006ED12B682760002B6ED0404B01261B782F
:106A6000002BD8D10920FFF7A1FF394B1E703B4BFB
:106A70001E70009B002B12D02B68002B0FD12368B7
:106A80002F60002B1ED0324B01261B78002BC7D164
:106A90000920FFF78BFF2E4B1E70304B1E702368B2
:106AA000002B0FD02A4E3278002A0BD19F4200D201
:106AB00027602368FB1A312B04D90720FFF776FFE4
:106AC000012333702B68002B0FD0244E3278002A1C
:106AD0000BD1BB4200D92F602B68FF1A312F04D98C
:106AE0000820FFF763FF012333702368002B0CD0CD
:106AF000019B002B09D1164E3378002B02D10720C1
:106B0000FFF754FF0023236033702B68002B00D164
:106B100080E7009B002B00D07CE7104C2378002BF3
:106B200002D10820FFF742FF00232B60237071E79A
:106B3000009A002AA0D1B5E7009B002B9FD1AEE7B9
:106B4000E41200200F270000C8250020FC070000E9
:106B5000D8120020D4120020DC120020E012002005
:106B600013B50400FFF77AFCFEF7EDFE0023009357
:106B7000134B1B68002B02D16846FDF787F80423EE
:106B800001A901200193FEF74DF800210800FEF74E
:106B900003F8FEF711FAFFF77FFAFDF7B7F8FDF7F4
:106BA0003BF9FDF755F9FEF74DFBFCF7E5FF002C2F
:106BB00004D0FDF7EBF90348FFF7D2FD13BDC04643
:106BC000141B00200AF50000002310B501001A0074
:106BD0001120FFF70FFC10BD07B56B461970694611
:106BE0005A7013128B701314120ECB700A716B460D
:106BF000010005221320FFF7FDFB07BD10B50A00B9
:106C000001001220FFF76CFC10BD70B505000C00F0
:106C1000FFF7CAFB002809D020003230FFF7E8FA5E
:106C20002B00220000211B20FFF7E4FB70BD10B5F4
:106C30000C000300110014202200FFF7DBFB10BD45
:106C4000012370B5FF24084A41185B42884201D3F2
:106C5000D84370BD06781D0A234073409B009B58A3
:106C600001306B40F2E7C046ECF0000013B50400C1
:106C7000FE2813D80A4BC200D05800280ED0436813
:106C800008309900FFF7DCFF01900920FFF7B0FA08
:106C900001AB042221001720FFF7ACFB13BDC04657
:106CA000C8250020F8B500231800254DDA00AA58A1
:106CB0000133511E8A418018FF2BF7D1052444432C
:106CC0000A20FFF795FAFB20FFF70EFA2720FFF7BF
:106CD0000BFA0020FFF708FAE0B22412FFF704FADB
:106CE000E0B2FFF701FA174BFA21186803F014FE1F
:106CF00000260700F300E85800281CD0436808303D
:106D00009900FFF79DFF04000520FFF771FAF0B22C
:106D1000FFF7EAF9E0B2FFF7E7F92004000EFFF70A
:106D2000E3F92002000EFFF7DFF9200EFFF7DCF990
:106D3000380001F041FF0136FF2EDBD1F8BDC0461F
:106D4000C825002004000020F7B50190FFF718FACD
:106D500001250400FF276D42002C01D12800FEBD53
:106D6000266833143B40152B0DD1210001980831C2
:106D700006F096FA002801D135123D402000FEF7BA
:106D800007FB0400E8E71D2BF8D101256D42F5E76C
:106D9000F0B5A1B0FFF706FA8021A94CA94F2068F1
:106DA000C900091AC019FDF7ADF82368C0182060A2
:106DB000002811D0FCF7B4FEA34B18603B78FA2BE7
:106DC00000D04FE12368022B08DCFFF7C5F900284B
:106DD00002D00120FFF796F921B0F0BD7B78BC7896
:106DE000981E242800D91FE103F002FD2500380079
:106DF0003C00400043004C001E01560088009200F9
:106E00009900AF00EE0005011E011E011E011E01CA
:106E10001E011E011E011E011E011E0119011E017F
:106E20001E011E011E011E011E011E011E011E016A
:106E30001E011E019600FF2C0ED02000FFF750FC13
:106E40000022824BE100CA505B181A7121000092A7
:106E500013001320FEF714FD0320BBE72000FFF70B
:106E600013FDF9E72000FFF73BFCF5E7FFF75CFDBA
:106E7000F2E7FFF7F3FA0020FFF772FE7448FFF71E
:106E80006FFCE9E7632CE7D8724BA200D2582100CF
:106E90001520FFF725FBDFE7FFF772F9FF27040056
:106EA000002CD9D025682B143B40152B04D0200092
:106EB000FEF76EFA0400F3E72000083006F0FAF956
:106EC00006000530FFF794F9FB20FFF70DF92D12AE
:106ED0001D20FFF709F9E8B2FFF706F9F0B2FFF756
:106EE00003F93012C0B2FFF7FFF825002B1B9E42BA
:106EF000DDDD287AFFF7F8F80135F7E700211D20DE
:106F000000910B000A00FEF7BBFCFDF73FF8A3E77A
:106F10002000FFF7ABFE9FE7FFF7C4FE9CE7FCF7FE
:106F200017FE07AC4C4A642100904C4B200006F041
:106F300049F902232000237006F0BCF92300020067
:106F400000211620FFF756FA86E7454BFA2118680C
:106F500003F0E2FC002604903C4AF3009B181C68F6
:106F6000002C28D01B790593636808349F00B81D56
:106F70000393FFF73DF9FB20FFF7B6F801207D1CD6
:106F8000FFF7B2F8F0B2FFF7AFF8E8B22D12FFF753
:106F9000ABF8E8B2FFF7A8F80598FFF7A5F8E719EE
:106FA000A7420CD8FFF7FEF8049B0398584301F062
:106FB00003FEFFF7F7F80136FF2ECDD14CE720781E
:106FC000FFF792F80134EBE70024FFF747FA2300BC
:106FD000220021000094DA20FEF752FCFF2221005B
:106FE000D2001A4805F0DCFDFCF7D0FF210020009C
:106FF000FDF7D2FD30E7012C02D1FEF7F3F92BE7C4
:10700000022C02D1FEF738FC26E7032C03D1002125
:107010000800FDF7C1FD0120FFF7A2FD1CE70023DA
:1070200021001A001A208DE71A00C83A052A00D953
:1070300012E7002218001100FAF71CFA0CE7C0460C
:10704000FC1A0020FC160020E8120020C8250020B1
:10705000ECF40000C02D002003F50000FEF4000059
:1070600004000020FB2B00D0B3E62268042A00DCD9
:10707000ABE63E79F878614B360206439E4200DD6E
:10708000A7E6331D9A4200DC9FE6FB5CFE2B00D096
:107090009FE67878BC78751E1B2869D01AD8072817
:1070A0004FD0082824D0012819D1FF2C10D020005F
:1070B000FFF716FB7D79524AB31E009221002A0089
:1070C0000A20FEF7DDFB4F4BE400E0501B191D7159
:1070D000701D7FE61D285DD04FD31E2871D00300A0
:1070E000C83B052BF4D8484A2900FAF7C3F9EFE763
:1070F000632CEDD87A79022A13D0032A1BD0012AF7
:10710000E6D1F979BB79090219433B7AA4001B0443
:1071100019437B7A1B060B435B0013433B4AA35086
:10712000D6E7002DD4DDB11E3548FDF7A3F9374B66
:10713000A400E050CCE7BB79A4005A1E93419B0009
:10714000ECE7632DC4DC07AF2A002F49380005F0B7
:107150000BFD002338007B55FFF7F6FD0028B7DB59
:107160002A4B8000C25821001520FFF7B9F9AFE77C
:1071700029002548FFF7F2FBAAE7FF2CA8D07A796F
:10718000022AA5D81E490B2000912100B31EFEF74C
:1071900077FB9DE7632D00DD6325002307A99D4252
:1071A0000ADCEB430022DB172B40CB181A701520AA
:1071B00000916B1C2100EAE7FA185279CA54013396
:1071C000EDE7022C13D0032C14D0012C00D07FE764
:1071D000002D00DC7CE77B79002B03D01C00322BD8
:1071E00000DD322464235C43094B1C6070E7FEF72A
:1071F000A9FB6DE7FEF7A7FB6AE7C046F6030000B0
:1072000002170020C825002001170020C02D0020F3
:10721000040000200122094B1A60094A1368002B60
:10722000FCD00322074B1B68D8171040C01801235D
:1072300080100638400018437047C04600C0004028
:1072400000C1004008C500400120704710B5064C41
:10725000200001F01DF90549200001F04DF901223F
:10726000034B1A6010BDC046381B0020801A060070
:10727000001B00201FB500210E20FCF76FFC012130
:107280000D20FCF76BFC01210F20FCF767FC1C4C68
:10729000200001F05BF81B4B1B4A1B6812681B495E
:1072A000D2B28B420BD880239B04019301AB1A719D
:1072B0000199029A0023200001F064F81FBD1449CF
:1072C0008B4202D88023DB04EFE712498B4202D8BD
:1072D00080231B05E9E710498B4202D880235B0518
:1072E000E3E70E498B4202D880239B05DDE70C497A
:1072F0008B4202D88023DB05D7E780231B06D4E727
:10730000181B0020300000202C00002048E801005D
:1073100090D0030020A1070040420F0080841E008F
:1073200000093D0010B5002815DD01240B6823423B
:1073300011D023410C4A13600C4AA04209D04B687B
:10734000234206D02341022B09D0032B09D0A342AC
:1073500003D002231360002010BD0023FAE70323AB
:10736000F8E71460F7E7C046300000202C0000204A
:1073700010B500280FDD0C68E3070CD56410012C54
:1073800009DD064B1B68002B01D1FFF75FFF2100D1
:10739000034801F0B1F8002010BDC046001B0020DA
:1073A000381B0020F8B501250868284203D10D20BC
:1073B000FAF7F6F9F8BD4010FCF7F4FB041E14DBF5
:1073C000FCF7CAFBA04210DB02212000FCF7C6FB41
:1073D000FA222900D200200001F020FC0025A8425A
:1073E00005D101002000FCF7B9FB0020E2E70027EF
:1073F0000726FA2201219200200001F00FFC00284C
:10740000F3D0282802DD0123B3401F43013EF0D210
:107410000E4EAF550135052DE9D100212000FCF7B6
:107420009DFB012206210920FCF7A6FF0028DCD0E5
:107430000B23012443600023F25C990052004118A1
:10744000224301338A60052BF6D1B3E7041B0020E9
:1074500070B500281EDD0D68EB071BD4042D19D96B
:107460000F242B681C40032C14D11A0992B25B0F15
:1074700092001C40141B2E00FFF7FCFE731B0648F5
:107480009C4205DD317900F083FF0136F070F5E7AD
:1074900000F07DFF002070BD181B00200120704708
:1074A00010B504680D20E30703D56410FF2C03D941
:1074B0001720FAF775F910BDFFF7DCFEE1B2044CB6
:1074C000200000F065FF200000F061FF0020F2E7DF
:1074D000181B002070B5FFF7CDFE064D00212800D7
:1074E00000F056FF0400280000F051FF0120640066
:1074F000204370BD181B002010B5034A0F2103481C
:10750000FEF78AFE10BDC04630F50000A8F5000069
:107510000D4B70B51B6804000E001500002B01D147
:10752000FFF794FEE1B2094C200001F07CF8F1B2C3
:10753000200000F079FFE9B2200000F075FF200084
:1075400001F0DCF870BDC046001B0020381B002095
:1075500010B501240368234205D04168214202D0BE
:107560008268224203D10D20FAF71AF910BD581093
:10757000802801D91520F7E74910FF2901D91620E5
:10758000F2E75210FF2A01D91720EDE7FFF7C0FFFD
:107590000020EBE7F7B501221400904226DD0D68CC
:1075A0002A4223D0374B15411B684C68002B01D170
:1075B000FFF74CFE344EE9B2300001F034F82700FA
:1075C0000122174014D01441FF2C02D91720FAF7DA
:1075D000E7F8E1B2300000F027FF300001F08EF84C
:1075E0000024A04202D02320FAF7DAF82000FEBDE2
:1075F000042CF2D90F2523681D40092D1CD1636886
:1076000001925B100093009BBB42E6DDBB00E318D8
:107610009D68019B1D420BD06D10FF2D02D91720D4
:10762000FAF7BEF8E9B2300000F0FEFE0137EAE7F3
:107630001720FAF7B5F8F9E7032D0FD127001A093B
:1076400092B25B0F92001D40551B3B1B9D42C4DD57
:107650003979300000F0E8FE0137F6E7042DBCD19F
:107660002000FCF7E7FC0500200005F023FE2C00BD
:107670000700631B9F42B0DD2178300000F0D4FE8C
:107680000134F6E7001B0020381B0020154B70B5B5
:107690001B6805000E00002B01D1FFF7D7FD124C2F
:1076A000EDB22900200000F0BEFFF1B2200000F092
:1076B000BBFE0021200000F0C1FF002801D04042A5
:1076C00070BD72B601222900200000F0A7FF62B64B
:1076D000200000F09AFE0028F2D0200000F09AFE70
:1076E000EEE7C046001B0020381B002010B5012427
:1076F0000368234202D04168214203D10D20FAF7EA
:107700004FF810BD5810802801D91520F7E749100F
:10771000FF2901D91620F2E7FFF7B8FF4000204308
:10772000EFE7000070B50D211D20FFF7AFFF184CEB
:107730005A280CD101222A2122703D38FFF7E8FE99
:10774000022001F039FA0122124B1A6070BD0F219C
:107750001920FFF79BFF332805D102238F222370C6
:1077600020211A38EAE70D211E20FFF78FFFC728D6
:107770000AD1032500222A21A9382570FFF7C8FE67
:107780002A002A211E20D9E700232370D8E7C0460B
:10779000340000200C1B002010B5002803DC1C2046
:1077A000F9F7FEFF10BD01240B681C4001D10D202C
:1077B000F6E75B10012B2BDD022B03D00224042BF8
:1077C00000DD0134194B1B68002B01D1FFF7AAFF24
:1077D000174B1B785BB2022B1CD0032B1ED0012B46
:1077E00011D1032C00D1013C00222A211D20FFF7DA
:1077F0008FFE22000E211D20FFF78AFE01222A2182
:107800001D20FFF785FE022001F0D6F90020C9E710
:107810000024D7E7220123211920F2E7032C00D10D
:10782000013C22000E211E20EBE7C0460C1B00206D
:1078300034000020204B10B51B680400002B01D140
:10784000FFF770FF1D4B1B785BB2022B0AD0032B96
:1078500029D0012B2CD121001D200124FFF716FF78
:10786000644205E0012C13D129211920FFF70EFFF6
:107870007F2801DD0138FF3803007F3301DA7F20E4
:107880004042C8237F21584303F046F8604310BDAF
:10789000032C0BD12B211920FFF7F8FE043CE7E75E
:1078A0002D211920D9E721001E20D6E7052CF7D07D
:1078B000012400206442E4E70C1B00203400002077
:1078C00010B50120FFF7B6FF43000120184310BD9B
:1078D00010B50320FFF7AEFF43000120184310BD91
:1078E00010B50520FFF7A6FF43000120184310BD87
:1078F000144B70B51B68002B02D10120FFF79AFFD3
:10790000114B1B785BB2013301D1FFF70BFF012054
:10791000FFF790FF04000320FFF78CFF0500052010
:10792000FFF788FF6D43644340436419201805F056
:1079300003F801F0CDFC04F0C9FF43000120184317
:1079400070BDC0460C1B002034000020F8B5514B20
:1079500005001B68002B01D1FFF778FC4E4C237803
:107960007F2B00D892E007210E20FFF78FFEC4285E
:1079700033D101220E26494B10211A70484B30009A
:107980001A702670FFF7C4FD802211213000FFF726
:10799000BFFD0021615600291EDB424EC9B23000F6
:1079A00000F041FE3D4B3000197800F03DFD300005
:1079B00000F0A4FE21780622300000F02FFEAC1D5E
:1079C000300000F022FD002806D0300000F022FD3B
:1079D00028700135A542F3D1F8BD0F211920FFF71A
:1079E00055FE33280FD168222C4B1E261A70002218
:1079F0002B4B60211A7030000C322670FFF788FD87
:107A000002226121C2E700211820FFF73FFEFA2879
:107A10001CD14222214B10261A700022204B4B21F0
:107A20001A70300001322670FFF772FD042001F059
:107A3000C3F838224C213000FFF76AFD0F22512194
:107A40003000FFF765FD1B2252219FE70F211C200C
:107A5000FFF71CFE3D289CD128221C2600270F4B37
:107A600020211A700E4B263A30001F702670FFF747
:107A70004FFD3A0022213000FFF74AFD3A00232152
:107A80003000FFF745FD402224217FE700216156A9
:107A900083E7C046001B002035000020370000208F
:107AA00036000020381B002073B500260622002176
:107AB000684605F075F86846FFF748FFFFF768F974
:107AC0001A4B6A469E576C466B4691781878D57863
:107AD0005B7812796479002E1FD0000209020343FB
:107AE00029431BB209B2120211482243007812B294
:107AF00040B2102802D15210DB10C910D8171B1841
:107B00004340C8170918414001205918D317D2180B
:107B10005A408A185200104376BD1B022D020343BF
:107B200029431BB209B22402DEE7C046360000201A
:107B300035000020F8B501231C0098422BDD0F68AA
:107B40003B4228D04E6835001D4024D1042E22D956
:107B50000F2231680A40092A1DD173685C10202C5D
:107B600000DD2024144B1B68002B01D1FFF76EFBB6
:107B700072B67F10F9B2114F2200380000F04EFDAE
:107B800062B6A54214DA380000F03FFC002804D1A8
:107B900001246D002C432000F8BD380000F03AFCB1
:107BA0000122AB004000F31810439860AD18E8E7DD
:107BB00064000125EEE7C046001B0020381B0020B2
:107BC00010B5054C2368002B02D01B20F9F7E8FD07
:107BD0000020206010BDC046101B002010B50028FA
:107BE00003DC1C20F9F7DCFD10BD0B68DA0706D4B6
:107BF000042B04D90F221B681340032B01D024202F
:107C0000F0E7034B25201B68002BEBD01B20E9E796
:107C1000101B002010B5002803DC1C20F9F7C0FD64
:107C200010BD0B68DB0701D40D20F7E71B20F9F727
:107C3000B7FD0020F4E700001D4B70B51B680C0079
:107C4000002B03D12520F9F7ABFD70BD012801DC25
:107C50001C20F8E708680121084207D1042805D94B
:107C60000F2302681340DD1E8D4201D92420EAE76C
:107C700065680D4201D11120E5E7042B0BD1FCF71B
:107C8000D9F905F017FB63685B10013B01D483420F
:107C900008DB1220D7E7100980B252008000920F53
:107CA000801AF0E71B20F9F77BFD0120CDE7C046E5
:107CB000101B002010B50400802803DD2620F9F7F2
:107CC0006FFD10BD002CFCDD1B20F9F769FDFEF7F0
:107CD00085FEFFF75DF8012000F06EFFF2E700007F
:107CE00010B5002805DC1C20F9F75AFD040020001F
:107CF00010BD184B1B68002B01D12520F4E701248F
:107D0000086804400FD04010FF2801D92820EBE775
:107D10001B20F9F745FDFEF761FEFFF739F801205A
:107D200000F04AFFF4E70428E1D90F21026811406E
:107D3000042906D1FCF77EF905F0BCFAFFF7BAFF7B
:107D4000D5E70329D3D1100980B2520F80000A4031
:107D5000801AF3E7101B0020044B10B51B68252088
:107D6000002B00D01B20F9F71BFD10BD101B0020BD
:107D700010B5034A06210348FEF74EFA10BDC0466F
:107D800054F6000084F60000002070470120704780
:107D90000020704700207047012070470020704786
:107DA0000020704700207047002070470020704777
:107DB0000020704700207047002070470020704767
:107DC00000207047002070477047704770470000E0
:107DD00010B5034A10210348FEF71EFA10BDC04635
:107DE000A4F6000024F700000378013B1F2B00D904
:107DF00070470130F8E710B5FFF7F6FF0378002B66
:107E00000BD00130222B11D10378002B03D0421C60
:107E1000222B03D11000FFF7E7FF10BD5C2B03D12D
:107E20004378002B00D0821C1000EDE73A2BF2D0F3
:107E30002C2BF0D07B2B0BD1FFF7D6FF0378002B38
:107E4000E9D07D2B01D10130E5E7FFF7D4FFF5E75D
:107E500020225B2B14D1FFF7C7FF0378002BDAD069
:107E60005D2BF0D0FFF7C7FFF7E7202BD3DD2C2BDE
:107E7000D3D0190091435D29CFD0222BCDD0013032
:107E80000378002BF1D1C6E7002210B5904216D03E
:107E9000FFF7AAFF03780422222B10D0023A7B2B93
:107EA0000DD0013A5B2B0AD0190030390232092972
:107EB00005D92D2B05D14178303909290AD8100070
:107EC00010BD0522742BFAD00132662BF7D0013297
:107ED0006E2BF4D0581E83415A42F0E770B5FFF77D
:107EE00083FF037801222D2B01D18018023A002351
:107EF0000A2502E06B430130CB1801783039CCB24F
:107F0000092CF7D95A43100070BDF8B50C001500C4
:107F1000FFF76AFF0378222B02D000232370F8BDFD
:107F20000D236A1E210008250C260A279C460130D5
:107F30000378222B02D100230B70F0E7002BFAD03C
:107F4000441C5C2B0BD14378841C622B0ED0662B17
:107F50000ED06E2B0ED0722B0ED0742B0ED0002AAA
:107F6000E9DD0B70013A01312000E1E72B00F6E773
:107F70003300F4E73B00F2E76346F0E70923EEE75E
:107F800010B50400FFF737FFA04203D90378013B87
:107F90001F2B00D910BD0138F6E710B5002815D009
:107FA0000378002B13D0FFF71FFF20210378020076
:107FB0008B4300205D2B09D01000FFF71CFF0378D6
:107FC0002C3B5A425341C018FFF70EFF10BD18005A
:107FD000FCE70300002070B50C0081420EDD1A782A
:107FE0005B2A0BD1581CFFF7FFFE0125AC4205D0E0
:107FF000FFF7D3FF002801D00135F7E770BD70B55A
:108000000C001500002901D000230B70002820D09F
:108010000378002B1ED0FFF7E7FE037806002C2B19
:1080200003D10130FFF7E0FE0600337800207D2BFE
:108030000FD0844204D02A0021003000FFF765FFF2
:108040003000FFF7D8FE03783A2B02D10130FFF75A
:10805000CBFE70BD1800FCE7F0B50D0004009DB02C
:108060002E78002E35D02E21280005F00BF9071EA2
:1080700014D0431B0193303E092E14D82800FFF77B
:108080002DFF01002000FFF7A4FF0400002C20D0EA
:10809000002F1ED0019B0133ED18E1E7280005F009
:1080A00009F90190E7E723787B2B11D1601C64224A
:1080B00003A9FFF7A4FF041E0BD0019A290003A80F
:1080C00005F0FFF80028E1D02000FFF794FEEEE76E
:1080D000002420001DB0F0BD70B5050000200C008C
:1080E00081421DDD2800FFF7CFFE0300681C012B35
:1080F00014D00020022B13D10022681C1100FFF7BE
:108100007EFF012C0CD0FFF748FF00221100FFF783
:1081100076FF013CF5E7FFF740FF013C012CFAD167
:1081200070BDF8B5050000200C0016001F0081424C
:108130000DDD2800FFF7A8FE03000020022B06D16A
:10814000681C3A003100FFF75AFF012C00D1F8BD3E
:10815000FFF723FF3A003100FFF751FF013CF4E73E
:1081600010B50024A04218D0FFF73EFE03787B2B09
:108170000AD1013000221100FFF741FF00280CD086
:10818000FFF739FE0134F5E75B2B06D10130FFF72D
:1081900004FF002801D00134F9E7200010BDF8B534
:1081A000002816DD0D68EB0713D56D10013D012485
:1081B000FDF7FAF90026FF27644200280CD1002EB3
:1081C00021D0300005F076F801003000FCF752F9BC
:1081D000F8BD01256D42EAE703681A143A40152AF2
:1081E0000BD11B123B409C4200DA1C009D4201D186
:1081F00006000836FDF7CCF8DFE71D2AFAD1012486
:1082000000266442F6E70120013464002043DFE7E2
:1082100010B508680C00FBF70DFFFEF795FD002870
:1082200003DB6268024B8000C250002010BDC046D4
:10823000C02D002010B50868FBF7FCFEFEF784FD9A
:108240000123002802DB024B8000C358180010BD38
:10825000C02D002010B50868FBF7ECFEFEF774FD9A
:10826000C043C00F800010BD10B5034A042103486D
:10827000FDF7D2FF10BDC046C8F70000C3F70000ED
:1082800010B5FBF7F9FDFBF7A7FEFEF731F8044840
:10829000FEF766FAFDF7E6F9FEF746FB10BDC046AD
:1082A00017F8000010B5FBF723F910BD70B50025D5
:1082B00004AC24780573A94205D10A4B0A4A25214A
:1082C0000A4804F0E3FB01600949920052589B0000
:1082D00002715B58A4008371635885604371022367
:1082E000C37170BD2FF800008EF800003DF800004B
:1082F000ECF80000037B002B04D14373837303610C
:1083000001330373704700001FB50191A0210024C1
:108310000068C900D2B24450012A10D0A24209D04C
:10832000032A0AD0074A8350074B019AC2500123FF
:1083300043501FBD02221343F4E70422FBE7062249
:10834000F9E7C046540500002405000010B50400FC
:10835000FFF7D0FFA1222368A179D200995061795B
:10836000064A20009950217904329950044B19682B
:108370005A689B68FFF7C8FF10BDC0460C05000097
:108380002C1B00201FB5FFF7BFFF05B000BD7047D5
:108390000368074A99501A00FC32D1680029FCD0C2
:1083A000A321C90058580023C0B2D3607047C0460B
:1083B0001C05000007B58022074BD2051A60002279
:1083C0009A6002321A710F230C3200930349023B68
:1083D0000348FFF76BFF07BD2C1B00200030004057
:1083E000181B0020F8B505000E0017000024BC4241
:1083F00008D02B68315D1B6828009847002801D001
:108400000134F4E72000F8BD704710B51C3000F0CF
:10841000AFF910BD10B51C3000F09CF910BD10B5BF
:108420001C3000F0ABF910BD70B5437E0D00002B81
:1084300001D1002070BD6430040000F0A8F90028CC
:10844000F7D12000290000F076F90120F2E70000C2
:10845000F7B50193FA23002504009B0083600B4BC2
:108460004560083303601C300F00160000F058F917
:108470002000643000F054F96B461B792761667563
:108480006576A5762000A375FEBDC046CCF8000039
:10849000012330B5A024C375837D13499B005A582E
:1084A000437DC132114DFF32E40592009B005B58C1
:1084B0001551CC22C133FF339B001D5104690C4B75
:1084C0005204E25005220469243BE250837D046992
:1084D0009B005A58A123DB00E250437D02699B00B8
:1084E0005958044BD15030BDECF800000C06000088
:1084F000240500000C050000A022002310B504692B
:10850000D200A3500A4CA1420FD90A4C8C425B41C5
:1085100009495B420B40CD21C9045B180469074936
:10852000635005210369995010BDCC235B04F5E726
:10853000A086010090D00300000098FD24050000F3
:10854000F7B5040000200D000193824265D01600AB
:10855000402A00D9402627001C37380000F0F6F8E2
:10856000B1232269DB00D5508022012321699200CA
:108570008B50A27E002A03D1226913622269136004
:108580000025731EAB4207D1019B002B04D0802233
:108590000221236992009950012223691A622369FA
:1085A000FC33DA68002A02D19A6A002AF9D09A6A62
:1085B000002A0BD1DA60A3232269DB00D1583800EE
:1085C000C9B2013500F0B7F8B542DAD3019B226990
:1085D000002B0FD11300FC339B6A002B0AD101330F
:1085E000A376D3612369FC33DA6C002AFCD0002225
:1085F000DA640AE000230121A37651611A0023699D
:10860000FC3399680029FCD09A602369FC339A6A8C
:10861000002A01D000229A62E8B2FEBD10B5012303
:10862000FFF78EFF10BD0300AC3310B504001970C6
:10863000643000F08BF80123637610BD0023020044
:1086400070B5AC3243760D001178B1220400006998
:10865000D20081508022216992008B50226901331F
:1086600013622269936026006436300000F080F8BF
:10867000002812D0300000F06DF81E4B2269D05057
:108680002369FC331A6A002A02D19A6A002AF9D0B7
:108690009A6A002A01D11A62E5E723690122002DB6
:1086A0000DD11900FC31896A002908D1DA612369EA
:1086B000FC33DA6C002AFCD00022DA6407E05A614D
:1086C0002369FC339A68002AFCD000229A600020BB
:1086D0002369FC339A6A82420BD098622169064A68
:1086E0008B588B501800022B03D0181F431E984143
:1086F000033070BD1C050000C404000010B501214A
:10870000FFF79CFF10BD000010B51323142202498F
:108710000248FFF79DFE10BD00400040381B0020BE
:1087200010B540220021040004F03AFA0023200092
:108730002364636410BD10B53F24026C531C2340B6
:10874000446C9C4201D08154036410BD0023036437
:1087500043647047436C026C934206D03F21C25C75
:1087600001330B4043641000704701204042FBE797
:10877000036C406C181A00D540307047436C026C93
:10878000934201D0C05C704701204042FBE73F228A
:10879000036C406C01331340181A43425841C0B275
:1087A0007047000003210A4802680A430260094832
:1087B00002680A4302600849084A094B9B1A03DD14
:1087C000043BC858D050FBDC00F012F8F7F79CFCD3
:1087D000240500405405004038FE00000000002041
:1087E00070020020FEE7FEE7FEE7FEE7FEE7FEE799
:1087F000014B024A1A607047380000200024F40040
:108800000120704710B503681322DB69984710BD3B
:1088100070470000054B0269D1500369FC331A6AA6
:10882000002AFCD0002201201A6270471C050000BB
:10883000030010B55C331A781F231A401E3B190041
:108840009140114AD167C222042104699200A150CB
:10885000026953600269D360A02300220169DB0032
:10886000CA5001230169094A5B428B500169084AD9
:108870008B5001690C3A8B50016908328B501430CF
:10888000FFF764FF10BDC04604E100E00C050000E6
:108890001405000010B51430FFF76AFF10BD10B5C5
:1088A0001430FFF76BFF10BD10B51430FFF752FF07
:1088B00010BD0000030070B55E331A780469724B76
:1088C000E25003005D331A780469704BE2500300F4
:1088D00061331C7802696E4B012C00D09EE00500CC
:1088E0005F352E78A225ED005651020060321578D2
:1088F000A1220669D200B5500269D4509623DB004C
:10890000994200D88CE096231B01994200D88AE056
:1089100096235B01994200D888E096239B019942F7
:1089200000D885E0E1239B01994200D882E096239C
:10893000DB01994200D880E0E123DB01994200D8B5
:108940007DE096231B02994200D87AE0E1231B02C6
:10895000994200D877E096235B02994200D874E0F0
:10896000E1235B02994200D871E0E1239B02994226
:1089700000D86EE0474B994200D86CE0E123DB025F
:10898000994200D86AE0E122002312038A425B4147
:10899000414A5B421340802252059B1801693F4ABD
:1089A0008B50A02304220169DB00CA500021036917
:1089B000FC33D9600369FC331962012301690B6040
:1089C00001698B60C1210469890062501F215C30FC
:1089D00002780A4093406231314AFF3153500021FE
:1089E000415600293CDA0F230B40083B2D4C9B08D5
:1089F0009B001B1903242140A140FC348C40DD69FD
:108A0000A5432C00C0258D4029002143D9611F2397
:108A1000017819401E3B8B40136070BD00246CE749
:108A20009E23DB02BAE79D231B03B7E71E4BB5E786
:108A30001E4BB3E7EC239B03B0E71D4BAEE71D4B8A
:108A4000ACE71D4BAAE71D4BA8E71D4BA6E71D4B46
:108A5000A4E71D4BA2E78023DB049FE71B4B9DE7A8
:108A60008C080F4BA400E41803230B40FF21C02502
:108A7000DB009940AD0066598E433100C0269E4010
:108A800033000B436351C2E70C05000014050000DE
:108A90006C05000090D0030000D0BEFE240500004D
:108AA00000E100E000ED00E000B0130000502700FE
:108AB00000A04E0000F0750000509D0000F0EB009B
:108AC00000903A0100E0D70100B0AF0300705F07EB
:108AD000F7B5009308AB1B7800250193FA23040037
:108AE0009B0083600E4B45600833036014300F0019
:108AF0001600FFF715FE23005C3327611E70009BF4
:108B0000084A9B00995823005D331970019B20008F
:108B10009B009A5823005E33DD701A70FEBDC0467C
:108B200070F90000ECF80000036910B51A00FC327F
:108B3000D2680400002A0AD0A322D2009958143027
:108B4000C9B2FFF7F8FD00222369FC33DA6010BDDB
:108B500010B50248FFF7E8FF10BDC046F01B00202B
:108B6000162307B5022200930249013B0248FFF792
:108B7000AFFF07BD00200040F01B002010B500280B
:108B800001D004F0C9FA10BD0849094A094B10B5D3
:108B90001B688858FA22190A1B0618439200002302
:108BA00001F0F2FF4904C00B084310BD0010014062
:108BB00004050000541C002070B5041E09D0FFF706
:108BC000E3FF050000F014F8FFF7DEFF401BA042B2
:108BD000F8D370BD0022044B9A60044A1368013335
:108BE000DBB213607047C046FC100140541C0020EB
:108BF0007047704710B500F05FF8FFF7FAFF0120EB
:108C0000FFF7DAFFFFF73CFBFFF74CFB024B002BB3
:108C1000FAD000E000BFF7E700000000F8B54C1EF6
:108C2000A1410125104B114F8000C3584C423868B8
:108C30000F499D40160001F0E5FD0A21704301F047
:108C4000E1FD2C400300220029000A4800F016F83C
:108C5000FA21094C89004443386801F0D3FD010032
:108C6000200001F0CFFDF8BDECF800003800002036
:108C700040420F00100500501027000030B5046876
:108C80000C40944206D1013B002BF8D112E0013B8D
:108C9000002B0FD004680C409442F8D100240568E2
:108CA0000D40954204D101349C42F8D1002002E0ED
:108CB000201C00E0181C30BDC420114B80001A5845
:108CC00010491140C02212020A431A50C0218022CA
:108CD000490092025A501A608023A3220021DB052A
:108CE000D20099500122F9309A60074BFF30195099
:108CF000C120023180001950403019501A6070476D
:108D000000E100E0FF00FFFF00100140014B186090
:108D10007047C04684000020F7B5002320285AD8A9
:108D2000384B8000C258042A5BD007D8022A54D09E
:108D300055D80423012A09D000234CE0062A54D038
:108D400051D31A2A53D002231B2AF5D12E4A116877
:108D500008294ED909294FD00A240226A02001252E
:108D60002A4AC00015502A482A4D07681C20BF0017
:108D700007402948019700685759009027481B026F
:108D800007401F43C02300989B020340FF20575118
:108D90005759000207401F43019B1F43009B580186
:108DA0006023184007433E43565101251C4B156074
:108DB00058680028FCD000205860A1230125DB0062
:108DC000D3585560A025ED0050511BB2A14202D0EE
:108DD00015D2611ACB401800FEBD0823B6E7102358
:108DE000B4E72023B2E74023B0E78023AEE70123B6
:108DF000ACE708240026B1E70C000126AEE7091B0A
:108E00008B40E8E7ECF80000800000200070004094
:108E10003C0000200405000040000020FF00FFFF90
:108E2000FC700040F0B520285BD8364B8000C2585B
:108E3000354B1E68002E30D1C227344BBF00D859A5
:108E4000334C03250440C02000022043D851C024E5
:108E500080206400800018512E4F18602E4B803CFB
:108E6000D859FF3CA043D8510437D859A8432043D0
:108E7000D8510837D8590C35A84384460720654691
:108E80002843D851A820C0001E50C1208026800051
:108E900076021E501C601C4B1C60142500202B0009
:108EA0001E4C2E0046433659771C1BD14343E250DB
:108EB000A0230325C132FF329200DB05D550184BA9
:108EC0001A68082A14D114234343E3189A681248F5
:108ED0005132FF32920059601150DA68C1239B0071
:108EE000C250F0BD9642E1D001300328D9D1F8E755
:108EF000082A02D9083AD140E5E708239A1A914096
:108F0000E1E7C046ECF80000581C002000E100E05A
:108F1000FF00FFFF04050000009000404400002017
:108F2000840000202149F0B54A6C2148002A14D061
:108F3000A025A12600230124ED05F600C258571CE8
:108F400006D0C7187F68002F02D027009740AF5186
:108F500014333C2BF2D100234B64A0230121DB0509
:108F600000260F009C4614234B43C3181A1F126897
:108F7000104C0E4D920014195219526C002A10D048
:108F80001A00143A1268551C09D0103B1B68FF2BBD
:108F900005D03B00934065461A00074BEA50FC346D
:108FA000666401310429DED1F0BDC046FC9000406A
:108FB00044000020009000400C05000000B520286F
:108FC00010D80C4A8000835803290BD8A02208002F
:108FD000C133FF33D2059B0001F000FC02090507F5
:108FE0000021D15000BD0C21FBE70421F9E703214A
:108FF000F7E7C046ECF8000020280AD8074B8000AD
:10900000C25801239340A022D205002902D104496D
:1090100053507047A121C900FAE7C046ECF80000A0
:109020000C05000003000020202B0AD8A021A2225A
:10903000C905D2008858034A9B009B58D840012399
:1090400018407047ECF80000F7B506000D000C0062
:109050008B180193019B671B9C4207D033682178D2
:109060001B683000984701340028F3D13800FEBD5A
:10907000F0B5C64600B5CB0F9846404A4B005B0D95
:109080009A1882B00D000400132A2FDC002A49DB55
:109090003B4F17413E000E40064323D07F08390066
:1090A00029400C430AD03749BD438C4663445C4297
:1090B0005C418023DB021341E4071D434146CE009F
:1090C00031492B008E192200346875682000290070
:1090D00001F000FF009001910098019922002B00FF
:1090E00003F090F802B004BC9046F0BD332A08DDCE
:1090F0008023DB009A42F5D102000B0001F0EAFE6A
:10910000F0E7224A9446012263445242DA40024286
:10911000E8D052080242D1D094438022D2051A41AD
:109120001443CBE74B005B080343DBD00B031B0B63
:109130001C436342234380244D0C24031B0B234018
:109140006D042B4319004346DA000F4B9B181C6833
:109150005D6802000B002000290001F0BBFE0090BA
:1091600001910098019922002B0003F04BF8424630
:109170004B005B08D60733431900B3E701FCFFFF40
:10918000FFFF0F00EEFBFFFFA0F90000EDFBFFFF6C
:10919000F8B5274A4B005B0D9A180C000700132AFC
:1091A00010DC002A36DB234B13410B423AD08024DB
:1091B00024031441002064189C430600250030005D
:1091C0002900F8BD332A0EDD80230600DB000D00E8
:1091D0009A42F4D102000B003800210001F07AFE1F
:1091E00006000D00EBE7144D0600AC460125634474
:1091F0006D42DD40AC4663460D000342DFD03323B1
:109200009A1A323B93401818874200D94C1C634687
:109210009843D2E7C90FCC070020531CCDD1074B90
:109220001C43CAE706000D000028C0D1C7E7C046AE
:1092300001FCFFFFFFFF0F00EDFBFFFF0000F03F11
:1092400030B5214A4B0087B05B0893421EDD1F4AB0
:10925000934205DD02000B0002F0D4FF07B030BDE1
:1092600002AA00F095F803231840049A059B0128F0
:1092700013D002281DD0002814D00298039900F0C2
:109280006FFB80231B069C466144E7E70023002216
:109290000093002301F0DEF8E0E70298039900F064
:1092A0005FFBDBE7012402980399009401F0D2F8F8
:1092B000D4E7012402980399009401F0CBF88023AD
:1092C0001B069C466144C9E7FB21E93FFFFFEF7F96
:1092D000F0B54746CE4680B58DB004000D0000F0D5
:1092E00067FA294B06001B780F005BB298460133E2
:1092F00010D022002B002000290003F0CBFA814679
:10930000002807D1002200232000290001F014FCCE
:10931000002806D1300039000DB00CBC90469946AB
:10932000F0BD01230293194B0694079503934B4616
:109330000A93434604940595002B15D00023002280
:109340001900100002F0E2F8434608900991022B40
:109350000ED103F0B9FB212303600A9B0193002B7C
:109360000CD1089E099FD5E7002300240893099497
:1093700002A801F0C1F90028EFD1EAE703F0A4FB4D
:109380000A9B01930360ECE788000020B0F900001D
:10939000F0B54E464546DE465746E0B5E14B4C003B
:1093A0008FB09046894664089C4200DC87E0DE4B23
:1093B0009C4222DCDD4A002900DC92E0DC4B02F01A
:1093C00021FFDB4B06000F009C4200D17EE1D94A11
:1093D000D94B02F017FF02000B00414630000A6033
:1093E0004B60390002F00EFFD34BD24A02F00AFF65
:1093F000434601259860D9606BE0D04B9C4200DC6D
:109400008FE0CF4B9C4200DD55E1CE4A23159246BA
:109410009A4451460905631A19001D00040003F01F
:1094200055FA03F089FA02000B0020002900089287
:10943000099302F0E7FE0022C34B02F071FC0F001B
:10944000060003F043FA03F077FA04000D0002006F
:109450000B00300039000A940B9502F0D3FE002275
:10946000B94B02F05DFC002200230C900D9101F03D
:109470005DFB002800D192E100230022200029009A
:1094800001F054FB434243410133B04A414601924B
:10949000022208A80092524600F07CFB4B460500D1
:1094A000002B16DA802243461206944642465B6839
:1094B000454263445360D3686344D36009E00B00C2
:1094C000020041460A604B600022002300258A60AA
:1094D000CB6028000FB03CBC90469946A246AB46F4
:1094E000F0BD934B01F0F6FC914B06000F009C423F
:1094F00000D13DE18F4A904B01F0ECFC02000B00E3
:10950000414630000A604B60390002F07BFE894A18
:10951000894B01F0DFFC012543466D429860D9601C
:10952000D7E701F049F88A4A8A4B06000F0002F09B
:10953000F7FB0022884B01F0CDFC03F0C7F90500D2
:1095400003F0FAF9794A7A4B0490059102F0E8FBAE
:1095500002000B003000390002F054FE754A06008C
:109560000F0004980599744B02F0DAFB0290039106
:109570001F2D00DCC7E0029A039B3000390002F087
:1095800041FE83468A4653465B0024155B0DE31A71
:10959000102B6CDD04980599D322674B520502F01D
:1095A000BFFB02000B00300039000292039302F06F
:1095B00029FE0A00010013000691079202003900FB
:1095C000300002F01FFE029A039B02F01BFE060011
:1095D0000F0004980599614A614B02F0A1FB32002B
:1095E0003B0002F00FFE069E079F0B0002003900B1
:1095F00030000292039302F005FE4B005B0D8346A0
:109600008A46E41A312C32DD04980599B822544B6D
:10961000920502F085FB03000C0002000293039404
:109620000B000698079902F0EDFD02000B00060002
:109630000F000698079902F0E5FD029A039B02F0DD
:10964000E1FD484A0290039104980599464B02F0C7
:1096500067FB029A039B02F0D5FD02000B0030006D
:1096600039000292039302F0CDFD83468A465A46A2
:109670005346414630000A604B60390002F0C2FD9B
:10968000029A039B02F0BEFD44460B000200A2605A
:10969000E3604B46002B00DB1BE75B462360802327
:1096A0001B065344636080231B069C466144A060F4
:1096B000E1606D420DE70B00020002F0A3FD43469E
:1096C00000259860D9601860596002E7D3221A4BD0
:1096D000520502F097FD214A214B0D00040002F0D3
:1096E00091FD02000B00414620000A604B602900FA
:1096F00002F088FD1A4B194A02F084FD4346012509
:109700009860D960E5E602000B003000390002F0F5
:1097100079FD6B1E154A9B009B5883468A46A342DF
:10972000A5D130E7FB21E93F7BD90240000040543E
:10973000FB21F93F3163621A61B4D03DFB2139410D
:10974000FFFFEF7FEAFBFFFF0000704138FA0000E7
:1097500083C8C96D305FE43F0000E03F7370032EA3
:109760008A19A33BC14920259A837B39B8F90000A7
:10977000D3220C4B520501F0ADFB0B4A0B4B0400FE
:109780000D0001F0A7FB02000B00414620000A601B
:109790004B60290002F036FD034A044BB9E603236F
:1097A00073E6C04661B4D03D7370032E8A19A33BA3
:1097B000F8B54746CE46674B80B50A000F00190042
:1097C00005003940994200D19BE004000100002FC0
:1097D00069DD3F1500D1B4E05F4B12039C46802346
:1097E000120B5B0313435B00CA0F67449B184A00CC
:1097F000F80703D5D20F5B009B188A0079108C46BE
:10980000002180201624894680030D189D4202DC29
:1098100029185B1B8144D50F5B00013C5B1952008A
:109820004008002CF1D10020804680202025002710
:10983000000609E08B425CD0D40F5B00013DE318C9
:1098400052004008002D16D0C4198B42F2DD2718B3
:109850000E00002C49DB5B1AA242894149425B1A87
:10986000121BD40F5B00013D80443100E31852000D
:109870004008002DE8D113434ED143465B083749D9
:109880004A468846494652104244C90702D58021BB
:1098900009060B4361460F05BD18180029000CBCD2
:1098A00090469946F8BD7B005B0803433900002BC6
:1098B000F5D0002F3CD1E30A153A6405002BFAD00D
:1098C0008020400303423FD1002700E00F005B00EF
:1098D000791C0342FAD0250020208D40401A29002F
:1098E000D71B2200C2401A4376E7FE43F60F8E19BB
:1098F000B1E79442A0D82718002CF6DB1E00002305
:10990000AEE702003B002800390002F009FA2A0005
:109910003B0001F0DFFAC2E74346013303D0434680
:1099200001335B08ABE7012398460023C144A6E757
:109930003B00020002F066FC02000B0001F0E6FDB5
:10994000ADE713000022BBE70127210020207F4262
:10995000C6E7C0460000F07F01FCFFFF0000E03FCB
:10996000F0B54746CE4680B587B000920193754B5F
:109970004F00814688467F089F4263DC02F0A6FFC5
:10998000002800D1D4E04A4643464846414602F00A
:10999000C7F904000D006C4A6C4B02F0C1F96C4A27
:1099A0006C4B01F097FA22002B0002F0B9F96A4AD9
:1099B0006A4B02F027FC22002B0002F0B1F9684A42
:1099C000684B01F087FA22002B0002F0A9F9664AE1
:1099D000664B02F017FC22002B0002F0A1F9644A4A
:1099E000644B01F077FA22002B0002F099F9029003
:1099F00003910022604B2000290002F091F9029AA5
:109A0000039B06000F002000290002F089F9009A4C
:109A1000019B04000D004846414602F081F9020016
:109A20000B002000290002F0EDFB02000B003000CB
:109A3000390002F0E7FB02000B0000204F4902F062
:109A4000E1FB70E002000B0002F06AF904000D0077
:109A50003D4A3E4B02F064F93D4A3E4B01F03AFA72
:109A600022002B0002F05CF93B4A3C4B02F0CAFB9F
:109A700022002B0002F054F9394A3A4B01F02AFA3D
:109A800022002B0002F04CF9374A384B02F0BAFBA7
:109A900022002B0002F044F9354A364B01F01AFA45
:109AA0002B00220002F03CF9354B029003919F42BB
:109AB0009FDD344B00229F423DDC334900207B1860
:109AC0002E4916001F0002F09DFB04900591002214
:109AD000294B2000290002F023F932003B0002F05C
:109AE00091FB029A039B06000F002000290002F060
:109AF00017F9009A019B04000D004846414602F008
:109B00000FF902000B002000290002F07BFB02008D
:109B10000B003000390002F075FB02000B000498C6
:109B2000059902F06FFB07B00CBC90469946F0BD5A
:109B300000201249F7E7154B002604920593144FB5
:109B4000C5E7C046FFFF3F3ED43888BEE9FAA8BD4E
:109B5000C4B1B4BD9EEE213EAD529C804F7E923E7C
:109B60009015CB19A001FA3E7751C1166CC1563F32
:109B70004C5555555555A53F0000E03F0000F03FBE
:109B80003233D33F0000E93F0000E0FF0000E73F31
:109B90000000D23FF0B5DE464E4645465746E0B59A
:109BA000DC4CA5440D9114001900A49A0993DA4BDA
:109BB0009200D6584D1E03901821E01E069602957D
:109BC00000F0AAFEC3430100DB1719404B1C9A00AA
:109BD0009B1ADB001B190B9105934C1B771918D4AA
:109BE000A59BA5009C463F1922AE6544013707E0BE
:109BF000286802F0A1FE013403C60435BC4208D037
:109C0000002CF5DA00200021013403C60435BC42E3
:109C1000F6D1069B002B01DA00F0FDFB069B0399B1
:109C20000133DB009A46099BDA0094460092002239
:109C3000914672AA0492B94A6144934688469AAB07
:109C400063449B44029B002B00DABCE15D46002686
:109C50000027039C4D442A686B6803CC02F060F82F
:109C600002000B003000390001F034F9083D060015
:109C70000F004445EFD1049B4B441E605F600823F6
:109C80009C46E144D145DDD10EA8042184464942D9
:109C900061448C46069A93009C44614684460A912E
:109CA0000399083B63448C460C93009B00926344E9
:109CB0009B46009A0498D10003008C4663440891A7
:109CC0001E685F68002A33DD954980468C466244F1
:109CD000D300984470AB9A460EAB99460022914B44
:109CE0003000390002F01CF802F0F0FD02F024FE12
:109CF00000228D4B04000D0002F012F802000B0050
:109D00003000390002F07EFA02F0E0FD4B4601C35C
:109D10009946434620001A685B68290001F0DAF88A
:109D200008235B429C46E04406000F00D045D5D195
:109D3000059B30001A003900984600F0DFFCFF2335
:109D400000229B0504000D0001F0EAFF00F038FC42
:109D50000022764B01F0E4FF02000B0020002900F6
:109D600002F050FA0D00040002F0B0FD814602F04E
:109D7000E3FD02000B002000290002F043FA060078
:109D800040460F00002800DCEEE0009B18215A1E20
:109D900092000EAB9B58091A1D000D41A9448D403D
:109DA0005D1B0EAB9D5017231B1A1D41002D2DDD91
:109DB00001239C46009BE144002B00DC1CE20E9C2E
:109DC0000123002C00D0B5E0009A012A09D09900A7
:109DD0000EAA54580133002C00D0ACE0009A9A42ED
:109DE000F5D1059B002B0EDD012B00D1A8E1022B44
:109DF00009D1009B0EA95A1E92000EAB9B580793E7
:109E00009B029B0A8B50022D00D1C1E0002300224F
:109E10003000390000F08AFE009B002800D194E257
:109E2000069A591E8A4210DC414A0A9894460EAAA4
:109E30006344944600229B0063441C68043B224315
:109E40008342FAD1002A00D0C0E0069B0EAA013B53
:109E50009B00D358002B00D0B3E001220C9B043BA5
:109E6000596801320029FAD0009B9C4662441100D7
:109E700007921A0001338B4246DC0B9863468046FA
:109E8000A59C4344A046099C9B00A1464A44984493
:109E9000D30022AA9146049A99449446089BA59A15
:109EA00063448446614494469A468B00634400931D
:109EB0004346586802F040FD4B4618605960029BCB
:109EC000002B24DB4D46039C0026002701E0286878
:109ED00069680CCC01F024FF02000B00300039004F
:109EE00000F0F8FF083D06000F005C45EFD1534637
:109EF0009E60DF6004239C460433E0449C46009B44
:109F0000E144E2449845D3D1079B0093D1E6002673
:109F10000027ECE794FDFFFF80FB000018FEFFFF29
:109F2000FFFFFF1F0000703E000070410000204056
:109F3000FFFFFF3F002180225204141B0EAA545041
:109F4000009999420EDD0EA884469B000EAA890056
:109F5000D25861446344CF4800E01A68821A04C3AF
:109F60008B42FAD101243CE7059B002B06D1009BD4
:109F70000EAA013B9B00D558ED1517E70022C64BF2
:109F8000300000F0F7FD002800D024E100253DE777
:109F900032003B000020C14902F034F906000F00F6
:109FA000002C00D132E7059A0020BC4900F0A6FB46
:109FB00002000B003000390002F024F906000F0007
:109FC00024E7012250E70026002754E64B46059A75
:109FD000079388468B000EA9CB58183A089505922E
:109FE000002B0DD18C464146AD4B43449B0063444E
:109FF000043B58680139183A0028F9D08846059280
:10A00000059A0020A54900F079FB434604000D00A5
:10A01000002B00DA05E29E000EAB9C464346DB00B7
:10A0200066449C46059370AB9946049F674400972D
:10A03000306802F081FC22002B0001F071FE00224A
:10A0400038607960974B2000290001F069FE083FD5
:10A0500004000D00043EB945EAD14AAB03939B4688
:10A0600000239A46069B4246994643460132029295
:10A0700004934B46002B00DAAAE080208A4B009D17
:10A080009846C005894900260027002408E00823D7
:10A090009C460835E044544511DC4346186859682D
:10A0A0002A686B6801F03CFE02000B0030003900AA
:10A0B00000F010FF013406000F00A145E7DA5B460F
:10A0C000C0C39B4601239C46009BE244083B00938F
:10A0D000029B9A45CDD1049B9846A49B022B00DDA0
:10A0E0008EE0002B37DC1FD1059B00271D00039B52
:10A0F00000249C461E006544083E2A686B683800B0
:10A10000210000F0E7FE083D07000C00AE42F4D14C
:10A11000089B002B03D080231B069C4664443A0016
:10A1200023000D990A604B600720079B18409B2372
:10A130009B009D443CBC90469946A246AB46F0BD70
:10A14000009B0EA95A1E92000EAB9B5807935B0210
:10A150005B0A8B5057E64346002B00DA70E1002083
:10A160000021DB004AAAD61848AF32687368083E5F
:10A1700000F0B0FEB742F8D1089B002B00D025E1DB
:10A180000B0002004A984B990D9C2260636002F01C
:10A1900039F8434607000C00002B13DD01254CAEB7
:10A1A000B14638002E0021004C4601360CCC00F0A0
:10A1B00091FEA146B045F7DA089B07000C00002B82
:10A1C00000D015E13A0023000D998A60CB60ABE71F
:10A1D0000026002773E701239C46009BE1440225EB
:10A1E000002B00DDEBE532003B0000202B4902F0A4
:10A1F00009F806000F0009E60024F2E54AAB0393D4
:10A20000A49B032B00D08FE74346002B00DC14E116
:10A21000039ADB009B46130091465B441E685F680F
:10A22000234B43440293DB00994448AB9A464B4688
:10A230005C681B681800210032003B00009001910F
:10A2400000F048FE04000D0002000B000098019988
:10A2500001F0D8FF3B00320000F03CFE4B46986016
:10A26000D9601C605D6008235B429C46E144260087
:10A270002F00CA45DBD14346012B00DCE3E0039A03
:10A2800013005B441E685F68029BDB0099464A44EA
:10A29000904610E0FFFFFF000000E03F0000F03FAD
:10A2A000FFFFFF3F0000703E40FB0000FB21F93F35
:10A2B000FFFFFF1F984643465C681B68180021009B
:10A2C00032003B000090019100F004FE04000D00FC
:10A2D00002000B000098019901F094FF32003B004E
:10A2E00000F0F8FD4346039A9860D9601C605D60F9
:10A2F000083B26002F009A42DCD14D4694460026AA
:10A3000000244746083565442A686B683000210000
:10A3100000F0E0FD083D06000C00AF42F4D1039BC5
:10A320004A9F5D689968D868089B002B65D0802299
:10A33000120694460D9B6544604464441F605D6052
:10A340009960D8601E615C61EEE69A464B460793C1
:10A35000059B30005A423900089500F0CFF90022E1
:10A360003A4B06000F0000F005FC002824D0384BC3
:10A3700000223000390001F0D3FC02F0A7FA524667
:10A380000400950002F0D8FA0022304B01F0C8FC1E
:10A3900002000B003000390001F034FF02F096FAA1
:10A3A0000EAA50510122059B524418339046059342
:10A3B00093000EAAD45023E65346300039009C0087
:10A3C00002F084FA0EAB1851D04619E680230D9A9C
:10A3D0001B06CB18106053600B0002004A984B9983
:10A3E00001F010FF434607000C00002B00DDD5E60E
:10A3F00080231B069C466444E4E62B003A000D9D36
:10A400002A606B600A000300AA60EB603200230040
:10A410002A616B6188E6099BDB00009372AB0493B1
:10A4200032E4A49B022B00DDE8E6002B00DD92E67F
:10A4300000D079E6002700246AE6002600246EE7B3
:10A440000020002198E60026340068E700007041F3
:10A450000000703EF0B5CE46474680B587B000920A
:10A460000193474A4B00814688465B08934207DCCC
:10A470004146484602F02AFA4146031E484666D045
:10A480004A4643464846414601F04AFC04000D0056
:10A4900002000B004846414601F042FC394A3A4B63
:10A4A00006000F002000290001F03AFC374A384B23
:10A4B00001F0A8FE22002B0001F032FC354A364B99
:10A4C00000F008FD22002B0001F02AFC334A344B37
:10A4D00001F098FE22002B0001F022FC314B324AA1
:10A4E00000F0F8FC0E9B02900391002B34D00098F2
:10A4F000019900222D4B01F013FC029A039B04905A
:10A5000005913000390001F00BFC02000B000498AB
:10A51000059901F077FE22002B0001F001FC009A62
:10A52000019B01F06FFE224A04000D00214B300018
:10A53000390001F0F5FB02000B002000290000F0BB
:10A54000C9FC02000B004846414601F05BFE07B023
:10A550000CBC90469946F0BD02000B00200029007B
:10A5600001F0DEFB124A134B01F04CFE32003B00BF
:10A5700001F0D6FB4A46434600F0ACFCE7E7C04694
:10A58000FFFF3F3E7CD5CF5A3AD9E53DEB9C2B8A65
:10A59000E6E55A3E7DFEB157E31DC73ED561C119C0
:10A5A000A0012A3F1111813FA6F810110000E03FE1
:10A5B000495555555555C53F49004B081900704739
:10A5C000474AF0B54F4691464B005B0D99444646CD
:10A5D000D6464A46C0B505000C000E008846070066
:10A5E000132A27DC002A4BDB3E4B13419A460B0013
:10A5F00052461340034318D03B4A3C4B28002100ED
:10A6000000F068FC0022002300F0AAFA002847D0DE
:10A61000002C04DA80234A465B03134198444646E3
:10A62000534600279E43380031001CBC9046994693
:10A63000A246F0BD332A08DD8023DB009945F4D122
:10A6400002000B0000F046FCEFE7294A9446012285
:10A6500063445242DA4092460242E6D0224A234BF9
:10A660002800210000F036FC0022002300F078FAD8
:10A67000002815D0002C1EDB534646469F430FE0B2
:10A68000194A1A4B2800210000F024FC0022002364
:10A6900000F066FA002803D0002C04DB0027002617
:10A6A00038003100C1E76400640825430027002D0D
:10A6B000F6D0104EF4E74B46142B0BD03422D21AAE
:10A6C000012393405D19BD4208D201239C462F000F
:10A6D000E044D1E7133B9C46E044CDE72F00CBE7B5
:10A6E00001FCFFFFFFFF0F009C7500883CE4377EF4
:10A6F000EDFBFFFF0000F0BF002070474B0070B57E
:10A700005B0D14000A00002B1AD14B005B080343B9
:10A7100015D0234B002201F003FB224B9C422DDB82
:10A720000A004B005B0D363B1F4DE318AB422ADCA1
:10A73000002B0DDD1D4C1B0522401A43110070BD7E
:10A740001B4DAB42F0D102000B0000F0C3FBF6E75B
:10A750001D00353519DA174B02009C4209DD0B004C
:10A760001548164900F032F8134A144B01F0D8FA94
:10A77000E5E70B001248134900F028F8104A114B86
:10A7800001F0CEFADBE70200E9E7084C363322405D
:10A790001B051343190000220B4B01F0C1FACEE751
:10A7A00000005043B03CFFFFFE070000FFFF0F809A
:10A7B000FF07000050C300009C7500883CE4377E12
:10A7C00059F3F8C21F6EA5010000903C30B54A0055
:10A7D000DB0FDB0752081A43110030BD02B471468B
:10A7E00049084900095C49008E4402BC7047C046D4
:10A7F00003B47146490840004900095A49008E4493
:10A8000003BC7047002243088B4274D303098B4278
:10A810005FD3030A8B4244D3030B8B4228D3030C30
:10A820008B420DD3FF22090212BA030C8B4202D3D2
:10A830001212090265D0030B8B4219D300E0090AFA
:10A84000C30B8B4201D3CB03C01A5241830B8B4203
:10A8500001D38B03C01A5241430B8B4201D34B03EC
:10A86000C01A5241030B8B4201D30B03C01A524151
:10A87000C30A8B4201D3CB02C01A5241830A8B42D6
:10A8800001D38B02C01A5241430A8B4201D34B02BF
:10A89000C01A5241030A8B4201D30B02C01A524123
:10A8A000CDD2C3098B4201D3CB01C01A52418309D7
:10A8B0008B4201D38B01C01A524143098B4201D311
:10A8C0004B01C01A524103098B4201D30B01C01A3C
:10A8D0005241C3088B4201D3CB00C01A52418308B6
:10A8E0008B4201D38B00C01A524143088B4201D3E3
:10A8F0004B00C01A5241411A00D201465241104643
:10A900007047FFE701B5002000F0F0F802BDC04637
:10A910000029F7D076E7704703460B437FD4002227
:10A9200043088B4274D303098B425FD3030A8B42E3
:10A9300044D3030B8B4228D3030C8B420DD3FF224D
:10A94000090212BA030C8B4202D31212090265D01B
:10A95000030B8B4219D300E0090AC30B8B4201D3CE
:10A96000CB03C01A5241830B8B4201D38B03C01A15
:10A970005241430B8B4201D34B03C01A5241030B8C
:10A980008B4201D30B03C01A5241C30A8B4201D33D
:10A99000CB02C01A5241830A8B4201D38B02C01AE8
:10A9A0005241430A8B4201D34B02C01A5241030A5F
:10A9B0008B4201D30B02C01A5241CDD2C3098B4244
:10A9C00001D3CB01C01A524183098B4201D38B01C1
:10A9D000C01A524143098B4201D34B01C01A524164
:10A9E00003098B4201D30B01C01A5241C3088B42A9
:10A9F00001D3CB00C01A524183088B4201D38B0094
:10AA0000C01A524143088B4201D34B00C01A524135
:10AA1000411A00D201465241104670475DE0CA0F0C
:10AA200000D04942031000D34042534000229C46CC
:10AA300003098B422DD3030A8B4212D3FC228901D6
:10AA400012BA030A8B420CD3890192118B4208D3AC
:10AA5000890192118B4204D389013AD0921100E00E
:10AA60008909C3098B4201D3CB01C01A5241830922
:10AA70008B4201D38B01C01A524143098B4201D34F
:10AA80004B01C01A524103098B4201D30B01C01A7A
:10AA90005241C3088B4201D3CB00C01A52418308F4
:10AAA0008B4201D38B00C01A5241D9D243088B424A
:10AAB00001D34B00C01A5241411A00D201466346ED
:10AAC00052415B10104601D34042002B00D5494251
:10AAD000704763465B1000D3404201B5002000F090
:10AAE00005F802BD0029F8D016E770477047C04648
:10AAF000D0400B1C1141203A03D49C46134118430B
:10AB000063465242934018437047C0468446101C27
:10AB100062468C46191C634600E0C0461FB501F032
:10AB200097F8002801D40021C8421FBD10B500F0DD
:10AB3000EFFF4042013010BD10B501F089F8002848
:10AB400001DB002010BD012010BDC04610B501F092
:10AB50007FF8002801DD002010BD012010BDC04697
:10AB600010B501F011F8002801DC002010BD012013
:10AB700010BDC04610B501F007F8002801DA00202A
:10AB800010BD012010BDC046F0B5CE4647461504A5
:10AB90002D0C2E0080B50704140C3F0C9946030CB5
:10ABA0007E435D43674363437F19340CE4199C463D
:10ABB000A54203D980235B029846C4444B464343D5
:10ABC0005143250C36046544360C2404A4195B1942
:10ABD000591820000CBC90469946F0BDF0B54E4681
:10ABE00057464546DE46E0B543025B0A450083B062
:10ABF0000F1C99462D0EC60F002D57D0FF2D24D0C7
:10AC00008020DB00C0041843002381469A469B46FF
:10AC10007F3D7C027A00FB0F640A120E984623D017
:10AC2000FF2A4BD0E30080240020E4047F3A1C4339
:10AC3000AD186B1C47460193534677403A000F2BE3
:10AC400048D87D499B00CB589F46002B00D085E01B
:10AC500008339A46063B9B467C027A00FB0FFF2591
:10AC6000640A120E9846DBD1002C00D090E05246C8
:10AC700001231A4392460120DBE74C465846170051
:10AC8000022824D0032800D1CFE00022002301288D
:10AC90004DD15802D205400AFF071043384303B094
:10ACA0003CBC90469946A246AB46F0BD002B5BD11A
:10ACB00004239A46033B00259B46AAE7FF35002C58
:10ACC00060D1524602231A4392460220B1E7FF2286
:10ACD0000023DEE74B461B0C9C464B462604360CF5
:10ACE000180461463300220C6446000C43434E4373
:10ACF0005043544380191A0C1218964203D98021EC
:10AD000049028C4664441B041B0C1004C0188301C8
:10AD10005E1EB341800E1843130C1B199B010343A5
:10AD20001C00230179D5012362081C401443019AB9
:10AD30007F32002A4DDD630704D00F232340042B0C
:10AD400000D00434230103D53C4B019A1C408032CF
:10AD5000FE2ABCDCA3015B0AD2B29AE70C239A4616
:10AD6000093BFF259B4654E7180001F071FE4A4657
:10AD7000431F76259A4000236D4291462D1A9A462C
:10AD80009B4646E7524603231A439246032050E768
:10AD9000200001F05DFE431F2D1A9C40763D0020EF
:10ADA00047E780230027DB03FF2272E7424666E77E
:10ADB0004C463200584662E780234A46DB031A427B
:10ADC00022D01C4220D123435B025B0A4746FF226C
:10ADD0005FE701239A1A1B2A21DC23000199D34043
:10ADE0009E318C401A0023005C1EA34113435A0776
:10ADF00004D00F221A40042A00D004335A0111D47F
:10AE00009B015B0A002244E780234A46DB0313438D
:10AE10005B025B0A3700FF223BE7019587E70022D0
:10AE2000002336E70122002333E78023DB0323439B
:10AE30005B025B0AFF222CE790FB0000FFFFFFF79D
:10AE400070B500283DD0C317C5185D40C40F280059
:10AE500001F0FEFD9E22121A962A07DCD2B20828C3
:10AE600033DD083885406802400A23E0992A0BDD6B
:10AE7000052329001B1AD94003001B339D402B00DA
:10AE80005D1EAB4119430D00052801DD431F9D40A8
:10AE90002B000F490B406E0709D00F263540042DBB
:10AEA00005D004335D0102D59F220B40121A9B018D
:10AEB000580AD2B24002D205400AE40710432043A8
:10AEC00070BD002400220020F4E76802400AF1E788
:10AED000FFFFFFFBF0B54F464646D6460C00090380
:10AEE000C0B5490A470F5E0039431F03DB0F9C467C
:10AEF00065007B0A570F1F436D0DE40F760DA146C9
:10AF0000C000B846D200AB1B64457BD0002B5FDD90
:10AF1000002E00D0A4E03E00164300D112E15E1ED8
:10AF2000002E00D09EE1871A4346B8428041012599
:10AF3000C91A4042091A0B0200D431E149024E0AF3
:10AF4000002E00D16EE1300001F082FD0300083BCD
:10AF50001F2B00DD61E120223900D21A9E40D14032
:10AF60009F400E439D4200DD51E15D1B6B1C1F2B7A
:10AF700000DD7CE12021C91A3D0030008F4088406F
:10AF8000DD40791E8F41310007222843D94000253A
:10AF900007433A40002A09D00F233B40042B05D039
:10AFA0003B1DBB42BF417F42C9191F000B0200D4A9
:10AFB00026E26A1CC64B55056D0D9A4200D106E18A
:10AFC000C44AFF080A40530752023B43120B8EE06B
:10AFD000002B00D0B8E06B1C5B055B0D012B00DC87
:10AFE00030E1871A4346B842B641CB1A76429E1BDF
:10AFF000330200D54CE13B003343A1D100220024B1
:10B00000002570E0002B00DCE5E0002E00D183E09D
:10B01000AF4EB54260D0802636043743B846382B51
:10B0200000DC3EE1434613431F007A1E97413F1860
:10B0300087428041404209180B0200D4B0E0A44B83
:10B0400001359D4200D1C3E0A24A7B080A4001219C
:10B050000F401F435108D30707221F433A4099E787
:10B060009B4EB54238D0802636043743B846382B3D
:10B0700000DDDCE01F2B00DC30E11E004746203EF7
:10B08000F740BC46202B04D04026F31A46469E408B
:10B090003243170063467A1E97411F43CCE0002BD2
:10B0A00000D104E24346134300D159E14B07C008E5
:10B0B00018438023C9081B03194208D04546ED08F0
:10B0C0001D4204D14346D008590708432900420FC6
:10B0D000C9007F4D1143C0004B07CA087C49C00816
:10B0E00003438D4268D012036D05120B6D0D0021D4
:10B0F00012031800130B0A0D12051A43764B2D0587
:10B1000013402B435B00E4075B08234319001CBC7E
:10B1100090469946A246F0BD3E00164312D05E1EF0
:10B12000002E00D000E18718874280414144404210
:10B13000091801250B0233D5022585E76446330043
:10B14000414610001D00C7E7002D00D0DAE00C00DA
:10B150000443F3D05C1C00D19FE15D4CA64200D1BA
:10B160002FE1DB43382B00DD66E11F2B00DD83E19F
:10B1700020240500E41A0F00DD40D940A0404346DA
:10B18000A7405B1A441EA04198462F433843171A24
:10B19000BA42924143465242991A64463500CAE681
:10B1A00007223A40002A00D0F6E64B07CA08484971
:10B1B000FF083B438D4296D11900114300D19EE117
:10B1C000802109030A431203120B414D8FE715003A
:10B1D000002200238BE7002B00D0C7E06B1C5F052B
:10B1E0007F0D012F00DCF1E0394DAB4200D1B9E019
:10B1F00085180A0085428941424449425118072274
:10B20000CF076D082F4349083A401D00C2E60722C8
:10B210003049ED1A31403A40BCE63E0028388640BD
:10B2200000279FE6380001F013FC20308EE64346ED
:10B2300013431F007A1E9741C71BB842804140420A
:10B24000091A78E60E003B0006431343002D61D136
:10B25000002E00D0F4E0002B00D11BE16446390041
:10B26000100039E71A4FBB427AD03300FFE63000B6
:10B270001F3DE840202B03D04021CB1A9E4037438E
:10B280007B1E9F41072207433A400021002589E7A2
:10B29000171A4346BA42B641591A76428E1B644683
:10B2A0004EE61F2B00DDADE020264746F61AB740DC
:10B2B000B9461700B246DF404E463E433700564679
:10B2C000B240561EB24117434246DA408918AEE6F4
:10B2D000FF070000FFFF7FFFFFFF0F80202647468C
:10B2E000F61AB740B9461700B246DF404E463E4315
:10B2F00037005646B240561EB24117434246DA4026
:10B30000891A99E77F4CA6425BD0802424045B42D3
:10B31000214327E7002E0CD1002B00D1CBE064465F
:10B3200039001000774DD7E6764FBB4218D0330076
:10B3300075E6002B14D04B07C00818438023C908BA
:10B340001B03194207D0FC081C4204D17907D0081E
:10B350000843E14621004C46420FC9001143C0009A
:10B36000684DB9E61D0000220023C0E6002D5BD128
:10B370000D00054300D1E2E65D1C00D1B0E0614D57
:10B38000AE421FD0DB43382B71DC1F2B00DD96E073
:10B3900020250F00ED1AAF40B9460700AA46DF404E
:10B3A0004D463D432F005546A840D940451EA84173
:10B3B00088440743BF1897429241514241443500A7
:10B3C0003AE6644635004146100085E60B0003432B
:10B3D000002D00D063E6002BF5D04346134300D187
:10B3E0007AE6871887428041072241444042091883
:10B3F0003A400B0200D4D5E6434B01351940C9E56C
:10B40000380069E61E004746203EF740BC46202B28
:10B4100004D04026F31A46469E4032431700634646
:10B420007A1E97411F4302E6364DAE42CAD08025B0
:10B430002D045B422943A6E70843411E8841A6E646
:10B44000002B00D148E6871A4346B842B641CB1AD2
:10B4500076429E1B33024BD5171A4346BA4292419D
:10B46000591A5242891A072264463A4092E501432A
:10B470000F00791E8F419DE71C000F00203CE74024
:10B48000202B03D04024E31A99400843411E8841F1
:10B4900038437CE60022002425E6171A4346BA42C8
:10B4A0009241591A5242891A6446350043E5414691
:10B4B0001000144D10E680220024120380E61D00C7
:10B4C0000F00203DEF40BC46202B03D04025EB1A57
:10B4D0009940084307006346781E87411F4369E788
:10B4E000871897429B4141445B42C9183500A3E548
:10B4F0003B003343CED0072231003A4052E60023CE
:10B500001A00F4E5FF070000FFFF7FFFF0B5574684
:10B51000DE464E464546E0B5834607000E0348002A
:10B5200085B092461C00360B400DCD0F002800D18F
:10B530009DE0954B984239D08023F6001B041E43B2
:10B54000924A7B0F33439946944603006344009329
:10B5500000230026FF00029323031B0B9846630081
:10B56000E40F52465B0D019400D1B3E086498B4253
:10B5700000D19EE04246D100802212040A43514687
:10B58000490F11438B46814952468C4600996344CA
:10B59000CB1A0021D20000932B0063409A460F2E55
:10B5A00000D905E17A4BB6009B599F465B46334371
:10B5B000994600D0B8E002230826002700900293A5
:10B5C000CAE7CB463A0002990195019B9A460229A7
:10B5D00027D0032900D180E2012944D06D49009B86
:10B5E0008C4663441C00002C38DD530700D013E266
:10B5F000D2085B46DB0109D55946674B19408B469B
:10B600008021C9008C46009B63441C00634B9C4214
:10B6100007DC5B4664055F075B0217431B0B620D8B
:10B6200002E000230027584A00211B031C0B0B0DCE
:10B630001B05234314055A4A380013401C43534644
:10B640006400DB0764081C43210005B03CBC904645
:10B650009946A246AB46F0BD0122524201231B1B74
:10B66000382B00DCADE1002200230027DCE75B463D
:10B67000334399465ED0002E00D18AE1300001F0BC
:10B68000E7F903000B3B1C2B00DD7BE11D22D31AE5
:10B690005A460100DA4008398E4013005F463343B2
:10B6A00099468F403F4B00261B1A009300230293BC
:10B6B00052E7414653460B433B499B468C46009B11
:10B6C000634400935B46002B3BD1022300221E43C0
:10B6D000022161E7434613439B4637D04346002B84
:10B6E00000D162E1404601F0B3F903000B3B1C2B93
:10B6F00000DD53E102004146083A914088461D2191
:10B70000CB1A5146D9400B0041460B439B4653464A
:10B7100093401A00009B25499C46604403008C46D8
:10B7200063440093002137E70323B14600900C26C1
:10B73000029311E7002300930133042600270293AC
:10B740000AE70323C3461E43032125E701331E43B3
:10B750000022012120E700239A46802300271B03B3
:10B76000094A61E7802349461B03194200D1E2E000
:10B770005946194200D0DEE00B431B0317001B0B98
:10B78000A246014A50E7C046FF07000001FCFFFF48
:10B79000D0FB0000FF030000FFFFFFFEFE070000DC
:10B7A000FFFF0F800DFCFFFF01F8FFFFF303000018
:10B7B000D94500D9CBE000D1C6E03C00484600277F
:10B7C000009B013B00935B46160E1B021E431302B7
:10B7D000984633041B0C9946310C0191FFF798F8F9
:10B7E0004A4642430B04210C050019438A4207D9FB
:10B7F0008919013D8E4203D88A4201D9851E8919D3
:10B80000881A0199FFF784F809048C464A462104F6
:10B8100064464243090C030021438A4204D9891932
:10B82000013B8E4200D8F1E02D041D43AB46434658
:10B83000891A4246280C12041D0C5B46140C220087
:10B840001B041B0C5A4303946B4344430295684307
:10B850001B19150CEB189C4203D980246402A446E2
:10B8600060441C0C15041B042D0C20185D1981422A
:10B8700077D373D00C1AA24A7D1BAF42BF419446C6
:10B88000009B7F426344E01B1C00864200D1DBE04A
:10B890000199FFF73DF84A4642430B04290C070083
:10B8A00019438A4207D98919013F8E4203D88A4237
:10B8B00001D9871E8919881A0199FFF729F8090407
:10B8C0004A46894629044D464243090C0300294350
:10B8D0008A4207D98919013B8E4203D88A4201D98D
:10B8E000831E89193F04891A3A00039F1A433800BE
:10B8F00013041B0C584381460298150C6F434343B5
:10B9000045434846000C8446DB1963449F4203D9F3
:10B91000802040028446654448461F0C00041B04F6
:10B92000000C7D191818A94200D284E000D17FE0F4
:10B9300001231A4357E680234A461B0313431B0384
:10B940001B0BAA466F4A6FE6BA4200D935E74B4651
:10B95000DC0758087B081C43FF0734E70024AF428C
:10B9600089D247444745A4415B466442A419641800
:10B97000013BA6421ED2A0426DD800D1B6E0241AE7
:10B980009B4678E703005A46283B9A400027914699
:10B9900088E6584601F05CF8203072E60300524613
:10B9A000283B9A4093460022B4E6504601F050F8F6
:10B9B00020309AE6A642E2D1B845DCD9341A9B463B
:10B9C00059E71F2B65DC504C0099A4465C46614446
:10B9D00008008C4011008240D940501E82410C4327
:10B9E00014435A46DA401300620709D00F2222405E
:10B9F000042A05D02200141D9442894149425B1853
:10BA00001A0262D50122002300270DE68A4200D8DF
:10BA10000AE7831E891907E70F231340042B00D17F
:10BA2000E6E5171D9742924153429B44FA08E0E530
:10BA3000002800D1D7E57118531EB14227D3A9427F
:10BA400015D358D01A0073E7002B00DC04E601235D
:10BA500000229B44CDE502234744474589415B4290
:10BA60009C46494289190C19E344241A03E74346CA
:10BA70005F0047459B41B8465B429E19023A8919CF
:10BA8000A94200D054E7404500D051E7ABE51A0089
:10BA9000F6E71F215F4649420C1BE740202B07D0E9
:10BAA0001A49009B8C46634418005B4683401A4346
:10BAB000501E82413A4307270023174009D00F2127
:10BAC000002311401400042995D122005F075B0276
:10BAD0001B0BD20817430022A6E5802359461B03FF
:10BAE0000B431B0317001B0B064A9DE5BD42B2D852
:10BAF0009B460024BFE68045B9D31A00C3E7C04681
:10BB0000FF030000FF0700001E0400003E040000C9
:10BB1000F0B54F464646D6468446C0B58046194ED7
:10BB200018030F034D00000B5C0082463F0B6D0DA8
:10BB3000C90F9146640DDB0F0120B5420AD0B44213
:10BB400003D0A54201D157450CD01CBC9046994664
:10BB5000A246F0BD66463E43F7D1AC42F5D154460D
:10BB60001443F2D10120C845EFD1994207D0002DEE
:10BB7000EBD163461F433800471EB841E5E700207C
:10BB8000E3E7C046FF070000F0B54F464646D646FD
:10BB90004D00C0B50E03C90F8A462C491F035C0037
:10BBA0008046360B6D0D91463F0B640DDB0F8D42C9
:10BBB0001ED08C4216D0002D1ED130438446002C5E
:10BBC00001D13A4323D06246002A1AD09A4529D09F
:10BBD000514602200139084001381CBC9046994664
:10BBE000A246F0BD39001143E5D002204042F4E7FF
:10BBF0003043FAD1AC420FD0002C0FD13A43E7D0FA
:10BC00000CE00122013B934318000130E5E7634655
:10BC10000020002BE1D0DBE73A43E6D19A45D7D1AB
:10BC2000A542D5DCA54205DBBE42D1D808D0002014
:10BC3000BE42D2D250460123013898430130CCE7AE
:10BC4000C845C5D80020C845F4D3C6E7FF070000A3
:10BC5000F0B54F464646D6464D00C0B50E03C90F57
:10BC60008A462E491F035C008046360B6D0D9146B7
:10BC70003F0B640DDB0F8D4218D08C4211D0002D8C
:10BC800018D130438446002C1ED13A431CD1634660
:10BC90000020002B30D051460220013908400138E5
:10BCA0002AE039001143EAD0022025E03043FBD1DD
:10BCB000AC4226D0002C26D13A4324D15146022052
:10BCC00001390840013817E06246002A0FD09A4532
:10BCD000E1D1A54205DBBE42DDD819D00020BE422D
:10BCE0000AD25046012301389843013004E0012272
:10BCF000013B9343180001301CBC90469946A24674
:10BD0000F0BD3A43D0D19A45C5D1A542C3DCE0E7A6
:10BD1000C845C0D80020C845E3D3EDE7FF070000C1
:10BD2000F0B55746DE464E464546E0B5834606002A
:10BD30000F03480087B092461D003F0B400DCC0F0B
:10BD4000002800D16FE0DE4B984238D08023FF00FE
:10BD50001B041F43730F3B430193DA4B00279946A3
:10BD600000239B46F60081442B0369001B0B5246BF
:10BD70009846490DED0F002900D185E0D04B99423E
:10BD800000D173E04346DA0080231B04134352467C
:10BD9000CC48520F84461343524600206144D200DF
:10BDA00089442100694000918C46012149448A461A
:10BDB0000F2F00D990E0C449BF00CF59BF465B4662
:10BDC0003B43019300D06AE1022308270026814605
:10BDD0009B46C9E732005846019B61460091022804
:10BDE00000D175E0032800D1FEE1012800D02CE14C
:10BDF00000230027002600253F032A0D3F0BB348F0
:10BE000012053A4302401B051343009A5B00D10719
:10BE10005B080B433000190007B03CBC90469946C4
:10BE2000A246AB46F0BD5B463B43019300D12FE1F8
:10BE3000002F00D1A5E1380000F00AFE03000B3B03
:10BE40001C2B00DD96E11D22D31A5A460100DA4070
:10BE50005E4608398F4013008E403B4301939C4B54
:10BE600000271B1A994600239B467DE7414653460F
:10BE70000B4393498C46E144002B00D01AE1022287
:10BE80000220174300228CE7134300D10DE1434603
:10BE9000002B00D181E1404600F0DAFD02000B3AB0
:10BEA0001C2A00DD72E10100434608398B409846A8
:10BEB0001D239A1A5346D3401A0043461343524651
:10BEC0008A404946081A824989468144002068E729
:10BED0007B4B002700268EE7140C1204120C110075
:10BEE000370C3604350C794328008C462E0060430D
:10BEF0006044834656432100300C804658467943BF
:10BF000040440291844506D98846802149028C46E6
:10BF1000E044414602913604010C360C00048B4685
:10BF200081191E0C1B041B0C0391190079438C46CC
:10BF3000280075436544A8465843050C454477439B
:10BF4000A94203D9802149028C466744290C8C46BA
:10BF500039000004000C2D042D186144AB440591F8
:10BF60005946049101990F043F0C080C39005143C4
:10BF70004243904602008C46090C8B4662437C4348
:10BF800044445C44A04503D9802149028846424488
:10BF9000210C884661460904090C8C463900594336
:10BFA000434370437E430F0CF6182404BE196444C7
:10BFB00042448C46B34203D980235B0298464044F6
:10BFC000029B61469846049B370443449B46AB451D
:10BFD000AD416B420D0405992D0C8C467F196744C9
:10BFE000FD18A8465D462D19A542A441934664421A
:10BFF000A446C344DC448F42BF4198459B419345CE
:10C000009241A445A4415B427F421F43360C5242F9
:10C010006442BF192243BF18624638184302D20D4A
:10C02000039913436A020A43501E82416146ED0D93
:10C030002A434E023243D90100D4B3E0012650080E
:10C0400032400243DE0732435B08224C5444002C4A
:10C0500062DD510709D00F201040042805D0101DC3
:10C060009042924152429B180200D90104D580248B
:10C070001948E400034054441848844200DD27E78F
:10C080005E075B02D2081F0B630516435B0DB2E629
:10C09000002399460133042700269B4664E60323C8
:10C0A000019781460C279B465EE60122012017433B
:10C0B000002276E6032303201F43434671E6C04671
:10C0C000FF07000001FCFFFF10FC0000FFFF0F80D6
:10C0D0000DFCFFFFFF030000FFFFFFFEFE07000057
:10C0E0000023802700933F030026434B83E6019BF8
:10C0F0003200A446584670E6AC466EE680270199A9
:10C100003F0339422DD03B422BD11F433F033F0B0E
:10C1100000951600384B6EE601252D1B382D00DDED
:10C1200066E61F2D40DC35481C0050441600824056
:10C130008440EE40501E824134431443EB4062077A
:10C1400009D00F222240042A05D02200141D944257
:10C15000804140421B181A023ED5012300270026C9
:10C1600049E68027019B3F031F433F033F0B009499
:10C17000214B40E603005A46283B9A400026019294
:10C180006DE6584600F064FC203057E60300524646
:10C19000283B9A401300002293E6504600F058FCDA
:10C1A00020307BE6CA4650E71F201E004042041B99
:10C1B000E640202D03D0124C5444A3401A43501E95
:10C1C0008241324307260027164009D00F20002362
:10C1D000104014000428B9D122005E075B021F0B37
:10C1E000D2081643002306E680273F031F433F0380
:10C1F0003F0B1600004BFEE5FF0700001E04000089
:10C200003E040000F8B557464E464546DE460C0053
:10C210000903E0B5490A460F5F0031431E03DB0FF7
:10C22000760A9B46530F3343C84E6500C000E40FA7
:10C23000D2006D0DA24681467F0D9C469046B742C6
:10C2400000D1B9E05B46012673409B46EE1BA34537
:10C2500000D183E0002E63DD002F00D0B1E0634603
:10C26000134300D123E1731E002B00D0BAE1861ADC
:10C270006346B04280410125C91A4042091A0B02A7
:10C2800000D447E149024B0A98464346002B00D1AF
:10C2900089E1404600F0DCFB0300083B1F2B00DD7A
:10C2A0007CE120223000D21A4146D0409940020061
:10C2B0009E400A439D4200DD6AE15D1B6B1C1F2B03
:10C2C00000DD94E1202110003500C91A8E40DA40CB
:10C2D0008840DD40711E8E41110007222843002551
:10C2E00006433240002A09D00F233340042B05D0E7
:10C2F000331DB342B641764289191E000B0200D4A9
:10C300003DE26A1C914B55056D0D9A4200D119E131
:10C310008F4AF6080A40570752023743120B9BE038
:10C32000002E00D0C5E06E1C7605760D012E00DCD7
:10C3300048E16746861ACB1BB042BF417F42B846F0
:10C340001F004346FF1A3B00B8461B0200D55FE1C1
:10C3500037439AD100220024002579E0002E00DC2A
:10C36000FAE0002F00D18DE0784B9D4267D080230A
:10C3700067461B041F43BC46382E00DC52E163466F
:10C3800013435A1E93411E188642804140420918A9
:10C390000B0200D4BEE06D4B01359D4200D1D2E0CE
:10C3A0006B4A73080A4001210E401E435108D3070F
:10C3B00007221E43324095E71E00164300D045E792
:10C3C00040E7624B9D423AD0802367461B041F43DF
:10C3D000BC46382E00DDEBE01F2E00DC3AE13300D6
:10C3E0006746203BDF403B00202E05D04027BF1B87
:10C3F0006646BE40324390464646721E96413343DF
:10C40000DAE0002B00D114E26346134300D168E167
:10C4100080234E07C008C9081B030643194208D0F1
:10C420006046C008184204D163460100D2085E0786
:10C430001643F3009946C900720F444D11434B4611
:10C44000DE08424B4F073743CA089D4200D16EE0D9
:10C4500012036D05120B6D0D00211203130B0A0D53
:10C4600012051A433B4B2D0513402B435B00E40799
:10C470005B082343380019003CBC90469946A2460D
:10C48000AB46F8BD6346134311D0731E002B00D09A
:10C4900007E186188642804161444042091801251F
:10C4A0000B0237D502257BE73E00614691463500F9
:10C4B000C5E75C46002D00D0E1E00B000343F3D05C
:10C4C000731C00D1ACE1214B9F4200D13AE1F34310
:10C4D000382B00DD6FE11F2B00DD8CE120250E00E5
:10C4E000ED1AAE40B0460600AA46DE40454635434A
:10C4F0002E005546D940A8406346451EA8415B1A08
:10C500009C463043161AB242924163465242991AEF
:10C510003D00B4E607223240002A00D0E4E60B4B8F
:10C52000F6084F073743CA089D4200D090E73B000A
:10C53000134300D1A6E180231B031A431203120BFD
:10C54000024D89E715000022002785E7FF0700005C
:10C55000FFFF7FFFFFFF0F80002E00D0C7E06B1CA6
:10C560005E05760D012E00DCF0E0C84DAB4200D137
:10C57000B9E085180A008542894162444942511850
:10C580000722CE076D082E43490832401D00A9E658
:10C59000BF49ED1A114007223240A3E63200283885
:10C5A0008240002686E6300000F052FA203073E622
:10C5B000634613435A1E9341C61AB042804140421B
:10C5C000091A5CE60E00674606431743002D5ED14C
:10C5D000002E00D0F3E0002F00D11EE15C46614642
:10C5E00091462CE7A94FBE427BD01E00F1E6100019
:10C5F0001F3DE840202B03D04021CB1A9A40164320
:10C60000731E9E410722064332400021002583E726
:10C61000161A6346B2428041591A40420B1A984694
:10C620005C4632E61F2E00DDABE02027BB1B9A469E
:10C6300063465746BB40994613004F46F3401F439D
:10C640003B005746BA40571EBA4113436246F24078
:10C65000891898E62027BB1B9A4663465746BB407D
:10C66000994613004F46F3401F433B005746BA40DC
:10C67000571EBA4113436246F240891A9CE7834B26
:10C680009F425FD080252D047342294320E7002E6E
:10C690000CD1002F00D1D0E05C46614691467B4D25
:10C6A000CDE67A4FBE421CD01E0065E6002F18D0A2
:10C6B000C0084E0706438020C9080003014208D085
:10C6C0006346DC08044204D12100DA46D2085E0742
:10C6D0001643F300994601245346C900720F1143D3
:10C6E0001C406A4DABE61D0000220027B4E6002D79
:10C6F00059D10B00034300D1D6E6731C00D1B2E040
:10C70000624B9F421ED0F343382B6FDC1F2B00DDA2
:10C7100097E020250E00ED1AAE40B0460600AA466E
:10C72000DE40454635432E005546A840D940451EBB
:10C73000A8418C440643B618964292415142614446
:10C740003D0025E63D006146914678E60B00034337
:10C75000002D00D055E6002BF5D06346134300D1E1
:10C760006DE68618864280416144404209180022E5
:10C770000B0200D4D0E6464B01351940B2E5B14674
:10C780005DE633006746203BDF403B00202E05D0AE
:10C790004027BF1B6646BE40324390464646721E47
:10C7A00096413343EFE5394B9F42CBD080252D0492
:10C7B00073422943A8E70843411E8841A2E6002F9F
:10C7C00000D13CE66346861ACF1AB0429B415B42D9
:10C7D000FB1A98461B024ED5161A6346B242924186
:10C7E000591A5242891A5C4600227BE501430E0029
:10C7F000711E8E419FE71D000E00203DEE40B046A9
:10C80000202B04D04025EB1A994008438146484626
:10C810004346411E8841184374E60022002417E66F
:10C82000161A6346B2429241591A5242891A3D0081
:10C8300025E561469146154D01E68022002412034C
:10C8400079E61D000E00203DEE40B046202B04D0BE
:10C850004025EB1A9940084381464E464346711ED7
:10C860008E411E4367E7861896429B4161445B42B6
:10C87000C9183D008CE547463743CED007224146D4
:10C88000324049E600273A00E6E5C046FF070000CF
:10C89000FFFF7FFF70B50C4E0D031C0349005B00CA
:10C8A0002D0B490D240B5B0DB14208D00649002029
:10C8B0008B4203D114432000441EA04170BD0543A8
:10C8C0000120002DFAD1F1E7FF07000030B5144D2B
:10C8D0000A034B00120B5B0DC90F0024AB4211DDA4
:10C8E000104CA34210DC8024640322430E4CE41A53
:10C8F0001F2C0CDD0D48C31ADA4013005C420029DE
:10C9000000D11C00200030BD094BCC18FAE7094DBE
:10C91000E040AC4663449A4013000343EEE7C04650
:10C92000FE0300001D040000330400001304000097
:10C93000FFFFFF7FEDFBFFFF70B500282DD0C31771
:10C94000C5185D40C40F280000F082F8154B1B1A73
:10C950005B055B0D0A2815DD0B38854000222D0391
:10C960002D0B002110002D030A0D2D0B12052A435B
:10C970000D4D1B052A4013435B00E4075B0823436E
:10C98000190070BD02002900153291400A000B21E8
:10C99000081AC5402D032D0BE3E7002400230025D2
:10C9A0000022DEE71E040000FFFF0F804100090E99
:10C9B0004B1C70B5DBB24602750AC40F012B14DDA7
:10C9C000E0239B006D07360BCB1800210A0D2800D1
:10C9D00012051C4D32435B052A405B0813435B0084
:10C9E000E4075B082343190070BD002914D1002D12
:10C9F0001ED0280000F02CF80A281CDC0B232A008B
:10CA00001B1ADA40030015339D400F4B12031B1A0B
:10CA10005B05160B5B0DD8E7002D06D0320B802688
:10CA200036036D071643094BCFE7084B0026CCE7CA
:10CA300000230026C9E703002A000B3B9A4000258B
:10CA4000E3E7C046FFFF0F8089030000FF070000F7
:10CA50001C2101231B04984201D3000C10391B0A2E
:10CA6000984201D3000A08391B09984201D30009F2
:10CA7000043902A2105C40187047C0460403020249
:10CA800001010101000000000000000030B51C00A1
:10CA9000094B05001B6885B0D868084B002A01D1F6
:10CAA000074B1A000292019300912B0022000549C6
:10CAB00000F026F800F0A6FD8C00002050FC0000DD
:10CAC000A0E700005DFC0000014B18687047C046FD
:10CAD0008C000020084B10B50400002B02D0002170
:10CAE00000E000BF054B1868836A002B00D0984710
:10CAF000200001F05DFBC046000000008CFC00003F
:10CB00000EB403B5010003AB044804CB00680193E5
:10CB100000F076F802B008BC03B018478C00002083
:10CB200070B500260C4D0D4C641BA410A64209D113
:10CB3000002601F03FFB0A4D0A4C641BA410A642DC
:10CB400005D170BDB300EB5898470136EEE7B3004E
:10CB5000EB5898470136F2E75C0200205C020020A7
:10CB60005C0200206C020020002310B59A4200D124
:10CB700010BDCC5CC4540133F8E710B5884202D92B
:10CB80008B18984203D3002307E08B5C8354013A4F
:10CB9000FBD210BDCC5CC45401339A42FAD1F8E701
:10CBA00003001218934200D1704719700133F9E75E
:10CBB000936810B5013B9360002B04DA9469A3429B
:10CBC00007DB0A2905D01368581C1060197008008B
:10CBD00010BD00F04BFC0100F9E7F8B506000F00AE
:10CBE0001400D518AC4201D1002007E021783A00AA
:10CBF0003000FFF7DDFF0134431CF3D1F8BD000026
:10CC0000F0B59FB002900F0016000593002805D0E4
:10CC100083690493002B01D100F0F4FD7B4B9F420C
:10CC20005BD1029B5F68BB891B0762D53B69002B08
:10CC30005FD0002306AC6361203363761033A376A4
:10CC400035002B78002B01D0252B5CD1AB1B049336
:10CC50000CD0320039000298FFF7BFFF431C00D10F
:10CC6000C4E06269049B9446634463612B78002BA3
:10CC700000D1BBE0012200235242626002A954327B
:10CC800052186E1C2360E360A3601370A3653178B3
:10CC900005225F4800F0D4FE751C002835D12268BB
:10CCA000D30604D5532302A95B182021197013075A
:10CCB00004D5532302A95B182B21197033782A2B32
:10CCC0002CD0350000210A20E3682A786E1C303A07
:10CCD000092A64D900292ED026E04E4B9F4202D16A
:10CCE000029B9F689FE74C4B9F429CD1029BDF6851
:10CCF00099E73900029800F00FFC002899D0012034
:10CD000040421FB0F0BD01359BE7414B2268C01A7D
:10CD100001238340134323602E00B8E7059B191DB0
:10CD20001B680591002B01DB099304E05B42E36083
:10CD30000223134323602B782E2B0AD16B782A2BE6
:10CD400035D1059B02351A1D1B680592002B2BDB84
:10CD50000793324E29780322300000F071FE00283C
:10CD600006D04023801B8340226801351343236093
:10CD7000297806222A486E1C217600F061FE0028E0
:10CD80003AD0284B002B25D10722059B073393432C
:10CD9000083305936369039A9B18636150E7434323
:10CDA00001219B18350090E701235B42D0E7002367
:10CDB0000A201A000135636029786E1C3039092970
:10CDC00003D9002BC5D00792C3E742430123521871
:10CDD0003500F1E705AB00933A00134B21000298B0
:10CDE00000E000BF0390039B0133D3D1BB895B06F6
:10CDF00000D584E70B9884E705AB00933A000A4B13
:10CE00002100029800F080F8ECE7C046E4FC000046
:10CE100090FC000004FD0000C4FC000096FC000033
:10CE20009AFC000000000000DBCB0000F7B5150005
:10CE300001938A680B6900900C00934200DA13009A
:10CE400022002B6043321278002A01D001332B607C
:10CE500023689B0602D52B6802332B6006272368C4
:10CE60001F4027D0230043331B785A1E934122686A
:10CE7000920630D42200019943320098089EB047B0
:10CE8000431C25D0062320682A68E168034000255A
:10CE9000042B03D18D1AEB43DB171D40A3682269D5
:10CEA000934201DD9B1AED180027BD4220D10020DE
:10CEB00010E00137E3682A689B1ABB42D2DD2200EA
:10CEC0000123193201990098089EB047431CF0D104
:10CED00001204042FEBD3020E1184331087021009E
:10CEE0005A1C45310978A218433202331170C1E748
:10CEF000220001231A3201990098089EB047431C72
:10CF0000E6D00137D1E70000F0B589B004920A00FD
:10CF100043320593039002920A7E0C000E9B6E2A08
:10CF200000D186E01FD8632A33D008D8002A00D168
:10CF30008CE0582A4DD0250042352A7030E0642A12
:10CF400001D0692AF7D1196825680A1D280629D554
:10CF500008681A60002803DA2D23029A40421370F1
:10CF60006B4E0A274FE0732A74D008D86F2A1FD05F
:10CF7000702AE0D1202209680A43226003E0752A62
:10CF800016D0782AD7D12200782145321170614E0F
:10CF900022E025001A684235111D196013682B70B4
:10CFA000012365E008681A606906D3D500B2D1E7AD
:10CFB00019682568081D186008682E0605D5544EA6
:10CFC00008276F2A1BD00A2719E06D06F7D580B213
:10CFD000F5E745314E4E0A7018682268011D006859
:10CFE0001960150621D5D30702D520231A432260E4
:10CFF0001027002803D1202322689A4322602300AF
:10D00000002243331A706368A360002B58DB0422AC
:10D01000216891432160002854D1029D002B5AD0F1
:10D020002500337842352B7055E05506DBD580B2AC
:10D03000D9E71A680D68101D4969186013682E0633
:10D0400001D5196002E06D06FBD519800023029D11
:10D0500023614FE01A68111D19601568002162688C
:10D06000280000F0EDFC002801D0401B60606368E0
:10D0700023610023029A13703CE023692A0004997B
:10D080000398059DA847431C3ED023689B0715D4F1
:10D09000079BE068984239DA180037E02200012344
:10D0A000193204990398059EB047431C2CD00135D2
:10D0B000E368079A9B1AAB42F0DCE9E70025F7E743
:10D0C0000028ADD0029D3900FDF722FC735C013DC4
:10D0D0002B700028F7D1082F09D12368DB0706D56C
:10D0E00063682269934202DC3023013D2B70029B6E
:10D0F0005B1B2361059B07AA00932100049B0398F7
:10D10000FFF794FE431CB8D10120404209B0F0BDA6
:10D11000A1FC0000B2FC00000D4B70B51C680500BE
:10D12000A36B002B0FD1182000F06EFC094BA063FD
:10D130000360094B01224360084B83600B2383810A
:10D140000023026143610022A36B1D615A6170BD1F
:10D150008C0000200E33CDAB34126DE6ECDE050002
:10D16000124B10B51C68A36B002B0FD1182000F0D8
:10D170004BFC0F4BA06303600E4B012243600E4B30
:10D1800083600B238381002302614361A46B0B4AFC
:10D19000206961690A4BFDF7F7FC01220023801822
:10D1A0005941206161614800400810BD8C00002099
:10D1B0000E33CDAB34126DE6ECDE05002D7F954CC1
:10D1C0002DF451580CB430B5164B9DB00C1E1D6893
:10D1D00008DA8B2301202B6040421DB030BC08BC14
:10D1E00002B01847822302A99B008B810023029082
:10D1F00008619C4200D0631E8B604B6101235B423F
:10D20000CB81209A21AB2800019300F055FD431CEF
:10D2100001DA8B232B60002CDFD00023029A1370DD
:10D22000DBE7C0468C0000200EB400B50B499CB073
:10D230001DAB02900690079104910948094904CB5F
:10D240000591006802A9019300F036FD0023029ABF
:10D2500013701CB008BC03B01847C046FFFFFF7F27
:10D260008C0000200802FFFF020010B51378541C48
:10D27000002B05D1CC5CD4540133002CFAD110BD65
:10D280002200F3E7C9B20378002B04D08B4200D10F
:10D2900070470130F7E74B42594149420840F7E7F0
:10D2A00002780B78002A03D0013001319A42F7D07E
:10D2B000D01A70470023C25C0133002AFBD1581EEC
:10D2C0007047002330B59A420AD0013AC45CCD5C65
:10D2D000AC4204D1934202D00133002CF6D1631B3F
:10D2E000180030BD30B50500002A00D130BD0C78E3
:10D2F000013A6B1C2C700131002C05D19A189A420E
:10D30000F4D01C700133FAE71D00EDE710B5037887
:10D31000002B0FD10B785A4253415B42184010BD8D
:10D320000023CA5C002AFAD0C45C944201D10133C4
:10D33000F7E701300378002BF2D11800EFE7000087
:10D34000F0B51F000E0087B00590019102920C9875
:10D35000347800F0EAFA082200194378751C13406B
:10D3600036D12D2C36D1B51C74780126002F62D011
:10D37000102F09D1302C07D120222B789343582B22
:10D3800054D110276C7802352D4B3900F318180052
:10D390000393FDF7BDFA04910121002349420200E5
:10D3A0008C4618002100303909291AD80C00A742F0
:10D3B00023DD591C09D06346824206D302D1049969
:10D3C000A14202DB0123784320182C780135E9E7DC
:10D3D0002E00BCE72B2C01D01E00C7E7B51C7478CB
:10D3E000FAE721004139192901D8373CDFE721004C
:10D3F0006139192901D8573CD9E75A1C08D1059A37
:10D4000023331360029B0398002B09D107B0F0BDB2
:10D41000002E00D04042029A002AF7D0002B01D003
:10D420006B1E0193029B019A1A60EFE73024002FD4
:10D43000AAD10827A8E7302C9ED00A27A4E7C04627
:10D44000FFFFFF7F37B51300064A05001068046A26
:10D45000002C00D1044C0A0000942900FFF770FF53
:10D460003EBDC0468C000020F0000020F8B505004D
:10D470000E001400002804D08369002B01D100F0B5
:10D48000C1F9224B9C422DD16C68A369A360A3898A
:10D490001B0731D52369002B2ED023682269F7B2F0
:10D4A000981A6369F6B2834205DC2100280000F077
:10D4B0003BF9002826D1A3680130013BA360236813
:10D4C0005A1C22601F706369834204D0A389DB0762
:10D4D0001AD50A2E18D12100280000F025F90028BD
:10D4E00012D00FE00A4B9C4201D1AC68CDE7094B4A
:10D4F0009C42CAD1EC68C8E72100280000F00CF873
:10D500000028CAD0012676423000F8BDE4FC0000B5
:10D5100004FD0000C4FC0000364B70B51D68060019
:10D520000C00002D05D0AB69002B02D1280000F0C3
:10D5300069F9314B9C420FD16C680C23E25E93B2C7
:10D5400019072DD4D90611D40923012033603733AC
:10D550001343A381404270BD284B9C4201D1AC686B
:10D56000EBE7274B9C42E8D1EC68E6E75B0713D575
:10D57000616B002908D023004433994202D0300067
:10D5800000F06AFA002363632422A3899343A381F2
:10D5900000236360236923600823A2891343A381C6
:10D5A0002369002B0BD1A0218022A389890092003E
:10D5B0000B40934203D02100300000F0E1F9012339
:10D5C000A289134011D00023A36063695B42A36169
:10D5D000002023698342BED10C23E25E1306BAD534
:10D5E00040231343A3810138B5E7920700D4636950
:10D5F000A360EDE78C000020E4FC000004FD0000C7
:10D60000C4FC000010B5062000F090FC012000F0E2
:10D61000CFFD0000F7B58A8905000C00130760D420
:10D620004B68002B04DC0B6C002B01DC0020FEBDE2
:10D63000E76A002FFAD000232E682B6080235B015D
:10D64000216A1A4034D0606DA3895B0706D56368F0
:10D65000C01A636B002B01D0236CC01A0200216A30
:10D6600000232800E76AB847A189431C06D12B682C
:10D670001D2B30D82B4ADA40D3072CD5002363600A
:10D6800023692360CB0405D5431C02D12B68002BF2
:10D6900000D16065616B2E600029C7D02300443340
:10D6A000994202D0280000F0D7F900206063BEE75D
:10D6B00001232800B847431CC6D12B68002BC3D0D8
:10D6C0001D2B01D0162B01D12E60AFE74023A2897C
:10D6D0001343A381ABE740230B430120A3814042C6
:10D6E000A5E70F69002FA1D00B680F60DB1B01932A
:10D6F0000023920700D14B69A360019B002B00DC43
:10D7000094E7019B3A00216A2800A66AB0470028E6
:10D7100003DC4023A2891343DFE7019B3F181B1A58
:10D720000193EAE7010040200B6970B505000C0089
:10D73000002B01D1002070BD002804D08369002B8C
:10D7400001D100F05FF80B4B9C4209D16C680C22B0
:10D75000A35E002BEED021002800FFF75BFFEAE775
:10D76000054B9C4201D1AC68F1E7044B9C42EED1E1
:10D77000EC68ECE7E4FC000004FD0000C4FC0000E1
:10D78000002310B504000360436083608181436619
:10D79000C281036143618361190008225C30FFF795
:10D7A000FFF9054B24626362044BA362044BE362FE
:10D7B000044B236310BDC0466DDF000095DF000001
:10D7C000CDDF0000F9DF000010B5024900F08CF851
:10D7D00010BDC04629D7000070B568254A1E5543C4
:10D7E0000E002900743100F081F9041E08D00021D8
:10D7F0002A00016046600C30A0606832FFF7D0F963
:10D80000200070BD836913B50400002B28D1836408
:10D81000C3640365134B144A1B68826201939842E8
:10D8200001D101238361200000F020F86060200016
:10D8300000F01CF8A060200000F018F80022E06062
:10D8400004216068FFF79CFF01220921A068FFF70F
:10D8500097FF02221221E068FFF792FF0123A361E4
:10D8600013BDC0468CFC0000C9D70000F8B51C4BA6
:10D8700007001E68B369002B02D13000FFF7C2FF1A
:10D880004836B4687368013B04D53368002B07D071
:10D890003668F6E70C22A55E002D0DD06834F2E75D
:10D8A00004213800FFF798FF30600028F0D10C23E6
:10D8B00004003B602000F8BD20000A4B656625602F
:10D8C0006560A560E36025616561A56108222900A6
:10D8D0005C30FFF765F96563A563A564E564E9E776
:10D8E0008CFC00000100FFFFF7B5040007000026D4
:10D8F00001914834002C01D13000FEBD6368A56859
:10D900000093009B013B009301D52468F2E7AB89AB
:10D91000012B08D90E22AB5E013304D02900380058
:10D92000019B984706436835EBE7EC300068704789
:10D9300070B50E001D000E23C95E96B014000029BC
:10D9400007DA00232B60B3891B0611D48023DB0088
:10D950000FE06A4600F088FB0028F2DBF022019B12
:10D9600012021340054A9B185A4253412B60EDE7BF
:10D9700040230020236016B070BDC04600E0FFFFCA
:10D98000F7B502268B8905000C00334206D0230030
:10D9900047332360236101236361F7BD01AB6A460E
:10D9A000FFF7C6FF00990700280000F09FF8002845
:10D9B00008D10C22A35E9A05EFD4032293431E43A1
:10D9C000A681E4E70F4BAB628023A289206013435A
:10D9D000A381009B20616361019B002B0DD00E236E
:10D9E000E15E280000F052FB002806D00322A38944
:10D9F00093431A0001231343A381A0893843A081D4
:10DA0000CBE7C046C9D7000010B5034B010018682A
:10DA100000F06CF810BDC0468C00002082B00029D8
:10DA200000D101A9101E06D0002B06D013780B6080
:10DA30001078431E984102B0704702204042FAE736
:10DA4000C9B28218904201D10020704703788B42FE
:10DA5000FBD00130F6E7000070B50500002910D0BA
:10DA60000C1F2368002B00DAE418280000F034FBB8
:10DA70001D4A1368002B05D163601460280000F074
:10DA80002CFB70BDA34209D9216860188342F3D1F1
:10DA900018685B6841182160EEE713005A68002A95
:10DAA00001D0A242F9D919685818A0420BD12068B8
:10DAB0000918581819608242E0D11068526841185C
:10DAC00019605A60DAE7A04202D90C232B60D5E72F
:10DAD00021686018824203D11068526841182160A1
:10DAE00062605C60CAE7C0465C1C0020032370B51E
:10DAF000CD1C9D43083506000C2D1ED20C25A942D5
:10DB00001DD8300000F0E8FA254A146821000029E9
:10DB100019D1244C2368002B03D1300000F0CAF93E
:10DB200020602900300000F0C5F9431C2BD10C23E4
:10DB30003000336000F0D1FA03E0002DDFDA0C236F
:10DB40003360002070BD0B685B1B19D40B2B03D90D
:10DB50000B60CC18256003E04B688C420DD113603C
:10DB6000300000F0BAFA200007220B30231D90434A
:10DB7000C31AE7D05A42E250E4E763600C00EFE7D3
:10DB80000C004968C3E70323C41C9C43A042E1D0B6
:10DB9000211A300000F08EF9431CDBD1C7E7C046E4
:10DBA0005C1C0020601C0020F8B507000D0016006A
:10DBB000002905D11100FFF799FF04002000F8BDEE
:10DBC000002A03D1FFF748FF3400F7E700F086FA98
:10DBD0002C00B042F2D231003800FFF787FF041E5C
:10DBE000ECD029003200FEF7BFFF29003800FFF714
:10DBF00033FFE3E7F0B58E6885B007000C000392B1
:10DC000001939E423CD890238A89DB001A4234D08B
:10DC10000325096923685B1A0293636902985D43CF
:10DC2000EB0F5D19019B6D1001331B18AB4200D93E
:10DC30001D00530532D529003800FFF757FF061E97
:10DC400009D10C233B6040230120A28940421343A9
:10DC5000A38105B0F0BD029A2169FEF785FFA38973
:10DC6000144A1A4080231343A381029B2661F618AD
:10DC700026606561019EED1AA560019B9E4200D958
:10DC8000019E320003992068FEF777FFA368002009
:10DC90009B1BA36023689E192660DAE72A003800E0
:10DCA000FFF782FF061EE0D121693800FFF7D4FE9E
:10DCB000C7E7C0467FFBFFFFF0B59FB0029005931A
:10DCC0008B890F0016001B0611D50B69002B0ED196
:10DCD0004021FFF70BFF38603861002805D10C2385
:10DCE000029A013813601FB0F0BD40237B6100230E
:10DCF00006AC6361203363761033A37635002B784E
:10DD0000002B01D0252B46D1AB1B04930CD0320045
:10DD100039000298FFF76EFF431C00D1AEE0626944
:10DD2000049B9446634463612B78002B00D1A5E0EB
:10DD3000012200235242626002A9543252186E1C22
:10DD40002360E360A3601370A36531780522544813
:10DD5000FFF776FE751C00281FD12268D30604D574
:10DD6000532302A95B1820211970130704D55323EC
:10DD700002A95B182B21197033782A2B16D0350095
:10DD800000210A20E3682A786E1C303A092A4ED90D
:10DD9000002918D010E00135B1E7414B2268C01AC4
:10DDA00001238340134323602E00CEE7059B191DFA
:10DDB0001B680591002B01DB099304E05B42E360E3
:10DDC0000223134323602B782E2B0AD16B782A2B46
:10DDD00035D1059B02351A1D1B680592002B2BDBE4
:10DDE0000793304E297803223000FFF729FE0028E0
:10DDF00006D04023801B83402268013513432360F3
:10DE00002978062228486E1C2176FFF719FE002883
:10DE10003CD0264B002B25D10722059B073393438B
:10DE2000083305936369039A9B18636166E743436C
:10DE300001219B183500A6E701235B42D0E70023B0
:10DE40000A201A000135636029786E1C30390929CF
:10DE500003D9002BC5D00792C3E7424301235218D0
:10DE60003500F1E705AB00933A00114B2100029811
:10DE700000E000BF0390039B0133D3D1BB890B9813
:10DE80005B0600D42FE7012040422CE705AB00934E
:10DE90003A00074B21000298FFF736F8EAE7C04640
:10DEA00090FC000096FC00009AFC000000000000BE
:10DEB000F5DB0000002370B5064C05000800236068
:10DEC00000F060F9431C03D12368002B00D02B60C5
:10DED00070BDC046F02F002070B504000D001F2952
:10DEE00004D9162303600120404270BD436C002B0F
:10DEF00004D08A009B181A68002A08D1200000F07C
:10DF000031F82A000100200000F01AF8EDE70020A7
:10DF1000012AEAD0511C03D1162301302360E4E723
:10DF2000002428001C6090472000DEE710B5034B5A
:10DF300001001868FFF7D0FF10BDC0468C0000201C
:10DF4000002370B5064C050008001100236000F0A6
:10DF500001F9431C03D12368002B00D02B6070BD56
:10DF6000F02F002010B500F0E5F810BD70B50C00E2
:10DF70000E25495F00F0BAF8002803DB636D1B181B
:10DF8000636570BDA389024A1340A381F9E7C046C7
:10DF9000FFEFFFFFF8B51F008B8905000C0016008E
:10DFA000DB0505D50E23C95E0022022300F080F8B0
:10DFB000A389054A28001340A38132000E23E15EA5
:10DFC0003B0000F02BF8F8BDFFEFFFFF70B50C0031
:10DFD0000E25495F00F06CF8A389421C03D1054A65
:10DFE0001340A38170BD802252011343A381606559
:10DFF000F8E7C046FFEFFFFF10B50E23C95E00F043
:10E0000021F810BD0B1E04D0FF2A04D98A23036017
:10E010008B3B180070470A700123FAE770B50500C2
:10E02000080011000022064C22601A0000F0B8F827
:10E03000431C03D12368002B00D02B6070BDC04669
:10E04000F02F0020002370B5064C05000800236067
:10E0500000F060F8431C03D12368002B00D02B6034
:10E0600070BDC046F02F0020002370B5064C05009F
:10E0700008001100236000F055F8431C03D1236809
:10E08000002B00D02B6070BDF02F0020002370B556
:10E09000064C05000800236000F054F8431C03D12F
:10E0A0002368002B00D02B6070BDC046F02F0020ED
:10E0B00070B50500080011000022064C22601A000D
:10E0C00000F050F8431C03D12368002B00D02B60D4
:10E0D00070BDC046F02F0020704770470B1F1B68B3
:10E0E000181F002B01DA0B58C018704770B50500D7
:10E0F000080011000022064C22601A0000F03AF8D5
:10E10000431C03D12368002B00D02B6070BDC04698
:10E11000F02F002058220120014B40421A60704726
:10E12000F02F002058220120014B40421A60704716
:10E13000F02F002058220120014B40421A60704706
:10E14000F02F00205822024B00201A607047C04672
:10E15000F02F002058220120014B40421A607047E6
:10E16000F02F002058220120014B40421A607047D6
:10E17000F02F002058220120014B40421A607047C6
:10E18000F02F0020044A1368002B00D1034B18180D
:10E19000106018007047C046641C0020F82F002053
:10E1A00058220120014B40421A607047F02F002096
:10E1B000FEE7C046F8B5C046F8BC08BC9E467047AE
:10E1C000F8B5C046F8BC08BC9E46704764617461EF
:10E1D000000000006AE20000EF01000073E20000AE
:10E1E000E50A000079E20000E302000081E200009D
:10E1F000990B000088E20000D50C00008DE20000C1
:10E200000905000093E20000F50600009EE2000010
:10E2100053030000A3E200002D0F0000AFE2000056
:10E220001F020000B9E20000110A0000C7E200006E
:10E2300095060000D4E2000081080000E0E2000042
:10E240005506000072616E646F6D00616C6C006C4D
:10E2500061737400300066616C736500747275657B
:10E2600000252E3135732E2E2E006D616B654C69A5
:10E2700073740072616E6765006164644C617374ED
:10E280000064656C657465006A6F696E0073706C1C
:10E29000697400636F707946726F6D546F006669C0
:10E2A0006E64006A6F696E537472696E677300758D
:10E2B0006E69636F6465417400756E69636F646550
:10E2C000537472696E67006E657742797465417246
:10E2D000726179006173427974654172726179008B
:10E2E000667265654D656D6F7279000059E30000D7
:10E2F000211400005EE300003F14000081E20000F2
:10E300004314000064E30000251400006EE30000E5
:10E310004714000077E300004B14000081E3000085
:10E320004F1400008AE300005314000095E300003E
:10E3300057140000A1E3000029140000AAE3000024
:10E3400037140000B4E300002D140000BFE3000008
:10E350003B14000066696C65006F70656E00636C4D
:10E360006F736500656E644F6646696C6500726523
:10E3700061644C696E6500726561644279746573AD
:10E380000072656164496E746F00617070656E64DF
:10E390004C696E6500617070656E64427974657376
:10E3A0000066696C6553697A650073746172744CB8
:10E3B000697374006E657874496E4C697374007388
:10E3C000797374656D496E666F0000005018000027
:10E3D000601800007A180000F61800002E190000DE
:10E3E000621900009A190000C0190000041A000008
:10E3F000461A00009A1A0000DE1A0000401B0000B6
:10E40000881B0000AE1B0000E61B00002C1C000057
:10E41000521C0000801C0000AE1C0000C233000033
:10E42000701D0000441E0000BA1E0000241F0000E2
:10E43000701F0000901F0000B21F000008210000A4
:10E440004E210000C6210000F42100002622000019
:10E4500074220000DC22000044230000A0230000FE
:10E46000FE23000070240000E22400003E2500008E
:10E4700098250000D82500001E2600006426000014
:10E48000AC2600000027000054270000922700005F
:10E490001C280000522800009A280000E2280000F2
:10E4A0002A29000064290000B4290000FC2900008A
:10E4B0005E2B0000801C0000E61B0000642A0000A8
:10E4C000501800009A2A0000C62A0000FC2A00000A
:10E4D000282B0000501800005018000050180000B1
:10E4E00050180000D82B00001A2C0000602C0000EF
:10E4F000B02C0000DC2C0000542D0000DA2D0000B0
:10E50000082E000050180000501800002C2E0000AB
:10E510005C2E00008C2E0000C22E0000EC2E0000AD
:10E52000222F00004C2F0000742F00009C2F0000B1
:10E53000CC2F0000FC2F00002630000050300000DF
:10E5400080300000AA300000501800005018000071
:10E55000501800005018000050180000DA30000079
:10E5600006310000323100005E3100009C310000B5
:10E57000D2310000083200003E3200007432000048
:10E58000A0320000CC32000002330000501800001E
:10E5900050180000501800005018000050180000DB
:10E5A00050180000501800005018000050180000CB
:10E5B0005018000050180000501800002E330000C2
:10E5C0002E330000663400009C3400005B2564207C
:10E5D0006974656D206C6973745D00282564206220
:10E5E000797465732900286F626A65637420747991
:10E5F00070653A2025642900537461636B20756E41
:10E60000646572666C6F7700626F6F6C65616E0037
:10E610006E756D62657200737472696E67006C6905
:10E620007374006279746520617272617900000010
:10E630000700000003000000C2E60000C93500002A
:10E64000CAE6000079360000D3E60000013B000076
:10E65000DCE60000CD350000E5E60000053B0000EB
:10E66000EDE6000099380000F6E60000E938000009
:10E6700004E70000C93700000FE70000B13C0000CC
:10E680001AE700000937000025E70000093C0000F8
:10E6900031E70000753700003DE70000813C0000D5
:10E6A0000000000001000000020000000300000064
:10E6B000040000000A0000006D6963726F3A62692D
:10E6C0007400686173546F6E6500706C6179546F8B
:10E6D0006E6500686173536572766F00736574537D
:10E6E0006572766F00646163496E6974006461638A
:10E6F000577269746500736F667457726974654206
:10E700007974650073717561726557617665007320
:10E710006574557365724C454400616E616C6F673A
:10E720005265616400616E616C6F675772697465F0
:10E73000006469676974616C52656164006469674B
:10E740006974616C577269746500474320746F6F18
:10E750006B2025642075736563733B206672656565
:10E7600020256420776F726473003C496E7465677E
:10E7700065723E003C4C6973743E003C4F626A65B2
:10E7800063743E003C4279746541727261793E0067
:10E790000D0A564D2050616E69633A2025730D0AAB
:10E7A000006D697363000000F5E700001147000089
:10E7B000FEE700000948000006E80000CD47000021
:10E7C0000AE80000A14700000FE80000BD170000A4
:10E7D0001EE800006546000026E800000B46000029
:10E7E00030E80000A14500003CE80000A344000020
:10E7F0006E756C6C00686578546F496E7400726554
:10E800007363616C650073696E007371727400628A
:10E81000726F616463617374546F494445006A7335
:10E820006F6E476574006A736F6E436F756E740028
:10E830006A736F6E56616C75654174006A736F6EB2
:10E840004B657941740000003CE900007948000004
:10E8500044E900007D4800004EE900009B480000AC
:10E8600057E90000A548000062E90000AF48000039
:10E870006EE90000B94800007CE90000C3480000D0
:10E8800084E90000CD4800008AE90000D748000074
:10E890009FE90000E1480000B4E90000EB480000F7
:10E8A000C0E90000F5480000D0E90000FF48000082
:10E8B000DCE9000009490000E9E900001349000013
:10E8C000F2E900001D490000FAE9000027490000B4
:10E8D00008EA00003149000019EA00003B49000045
:10E8E0002CEA0000454900003AEA00004F490000C8
:10E8F00049EA0000594900005CEA00006349000051
:10E9000072EA00006D4900007EEA000077490000CD
:10E910008EEA0000814900009DEA00008B4900005A
:10E92000ABEA000095490000B3EA00008748000008
:10E93000BBEA0000914800006E657400686173577F
:10E94000694669007374617274576946690073742B
:10E950006F705769466900776966695374617475A9
:10E9600073006D7949504164647265737300737408
:10E97000617274535349447363616E0067657453E5
:10E98000534944006D794D41430068747470536578
:10E99000727665724765745265717565737400723D
:10E9A0006573706F6E64546F4874747052657175DE
:10E9B0006573740068747470436F6E6E6563740081
:10E9C000687474704973436F6E6E65637465640038
:10E9D00068747470526571756573740068747470CE
:10E9E000526573706F6E73650075647053746172F5
:10E9F000740075647053746F700075647053656E45
:10EA0000645061636B657400756470526563656919
:10EA100076655061636B65740075647052656D6FE7
:10EA20007465495041646472657373007564705213
:10EA3000656D6F7465506F727400776562536F63B4
:10EA40006B6574537461727400776562536F636BA6
:10EA500065744C6173744576656E740077656253B6
:10EA60006F636B657453656E64546F436C69656E58
:10EA700074004D515454436F6E6E656374004D5174
:10EA800054544973436F6E6E6563746564004D51F1
:10EA90005454446973636F6E6E656374004D5154D2
:10EAA000544C6173744576656E74004D51545450E6
:10EAB0007562004D515454537562004D5154545574
:10EAC0006E737562001A1B1C03040607090A1718E7
:10EAD00019000000000008080800080A4A40000069
:10EAE0000A5FEA5FEA0ED92ED36E19324489330CDD
:10EAF000924C924D0808000000048808080408049D
:10EB0000848488000A448A4000048EC48000000087
:10EB1000048800000EC000000000080001224488A4
:10EB2000100C9252524C048C84848E1C824C901E89
:10EB30001EC244924C06CA525FE21FF01EC13E0242
:10EB4000448ED12E1FE24488100ED12ED12E0ED12C
:10EB50002EC488000800080000048004880244884D
:10EB60000482000EC00EC008048244880ED126C064
:10EB7000040ED135B36C0C925ED2521C925C925C46
:10EB80000ED010100E1C9252525C1ED01C901E1EF5
:10EB9000D01C90100ED013712E12525ED2521C88CF
:10EBA00008081C1FE242524C125498149210101084
:10EBB000101E113B75B131113935B3710C9252529F
:10EBC0004C1C925C90100C92524C861C925C9251A0
:10EBD0000ED00C825C1FE4848484125252524C1179
:10EBE00031312A44113135BB7112524C9252112AE3
:10EBF0004484841EC488101E0EC808080E10080421
:10EC000082410EC242424E048A40000000000000D1
:10EC10001F0804800000000ED2524F10101C925C9E
:10EC2000000ED0100E02424ED24E0C925C900E0698
:10EC3000C81C88080ED24EC24C10101C92520800FC
:10EC4000080808024002424C101498149208080860
:10EC50000806001B75B131001C925252000C9252F2
:10EC60004C001C925C90000ED24EC2000ED01010D0
:10EC70000006C8049808080EC807001252524F0038
:10EC800011312A4400113135BB00124C8C92001115
:10EC90002A4498001EC4881E06C48C84860808086E
:10ECA000080818080C881800000C83600000000099
:10ECB000010000000200000003000000040000004A
:10ECC000050000000600000007000000080000002A
:10ECD000090000000A0000000B0000000C0000000A
:10ECE0000D0000000E0000000F00000010000000EA
:10ECF00012000000140000001600000018000000C0
:10ED00001A0000001C0000001E000000200000008F
:10ED10002300000026000000290000002C00000055
:10ED20002F00000032000000360000003A00000012
:10ED30003E00000042000000460000004B000000C2
:10ED400050000000550000005A0000006100000063
:10ED5000680000006F000000760000007D000000E9
:10ED6000840000008B000000920000009900000069
:10ED7000A0000000A7000000AE000000B5000000E9
:10ED8000BC000000C3000000CA000000D100000069
:10ED9000D8000000DF000000E6000000ED000000E9
:10EDA000F4000000FB000000FF00000004EE000083
:10EDB000B94900000FEE00008D4F000019EE000071
:10EDC000994B000026EE0000FD4C00002DEE0000E7
:10EDD0004D4D000036EE00009D4D000042EE00005B
:10EDE000954C000053EE0000254C000063EE00003F
:10EDF0008D4E000070EE0000F14B000064697370EE
:10EE00006C6179006C696768744C6576656C006D3F
:10EE100062446973706C6179006D62446973706CEF
:10EE200061794F6666006D62506C6F74006D62555B
:10EE30006E706C6F74006D624472617753686170BC
:10EE400065006D625368617065466F724C657474DD
:10EE50006572006D62456E61626C65446973706CC9
:10EE60006179006E656F506978656C53656E6400FA
:10EE70006E656F506978656C53657450696E004EAD
:10EE80006F7420656E6F75676820726F6F6D206597
:10EE900076656E20616674657220636F6D70616364
:10EEA00074696F6E00436F6D7061637465642046B2
:10EEB0006C61736820636F64652073746F72650A98
:10EEC0002564206279746573207573656420282534
:10EED00064252529206F6620256400426164207224
:10EEE00065636F726420666F756E64206475726905
:10EEF0006E6720696E697469616C697A6174696FA3
:10EF00006E00256420256420256420282564207750
:10EF10006F72647329002564207265636F72647375
:10EF20002C20256420776F7264732C206D617849E2
:10EF3000442025642C20636F6D70616374696F6E6B
:10EF4000206379636C657320256400526573746F68
:10EF50007265642025642073637269707473005352
:10EF600074617274656400726164696F000000000E
:10EF700005F00000A559000012F00000A15C00009F
:10EF800022F00000215C000030F00000355E00003F
:10EF90003BF00000BD5900004BF00000395A000062
:10EFA0005FF00000215A00006EF00000E55F0000F5
:10EFB0007AF00000635F000083F00000075F00004C
:10EFC0008EF00000815E000099F00000BD5E000040
:10EFD000A2F00000F15E0000ABF00000CD5900008F
:10EFE000BAF00000015A0000C3F00000DD59000033
:10EFF00025303878006E6F6E65006F74686572003A
:10F00000706169720064697361626C655261646900
:10F010006F006D65737361676552656365697665D9
:10F0200064007061636B6574526563656976650041
:10F030007061636B657453656E64007265636569C6
:10F04000766564496E7465676572007265636569AB
:10F050007665644D65737361676554797065007298
:10F0600065636569766564537472696E670073657C
:10F070006E64496E74656765720073656E64506195
:10F0800069720073656E64537472696E67007365AC
:10F09000744368616E6E656C0073657447726F755A
:10F0A0007000736574506F776572007369676E6185
:10F0B0006C537472656E6774680064657669636525
:10F0C0004944006C6173744D6573736167654944AD
:10F0D00000556E6B6E6F776E207072696D69746922
:10F0E0007665205B25733A25735D00000000000003
:10F0F000963007772C610EEEBA51099919C46D0745
:10F100008FF46A7035A563E9A395649E3288DB0E9F
:10F11000A4B8DC791EE9D5E088D9D2972B4CB60982
:10F12000BD7CB17E072DB8E7911DBF906410B71D5F
:10F13000F220B06A4871B9F3DE41BE847DD4DA1A98
:10F14000EBE4DD6D51B5D4F4C785D38356986C13C9
:10F15000C0A86B647AF962FDECC9658A4F5C011442
:10F16000D96C0663633D0FFAF50D088DC8206E3B20
:10F170005E10694CE44160D5727167A2D1E4033C32
:10F1800047D4044BFD850DD26BB50AA5FAA8B53559
:10F190006C98B242D6C9BBDB40F9BCACE36CD83248
:10F1A000755CDF45CF0DD6DC593DD1ABAC30D926EF
:10F1B0003A00DE518051D7C81661D0BFB5F4B421F2
:10F1C00023C4B3569995BACF0FA5BDB89EB80228EF
:10F1D0000888055FB2D90CC624E90BB1877C6F2F74
:10F1E000114C6858AB1D61C13D2D66B69041DC766F
:10F1F0000671DB01BC20D2982A10D5EF8985B17148
:10F200001FB5B606A5E4BF9F33D4B8E8A2C90778F6
:10F2100034F9000F8EA8099618980EE1BB0D6A7F8D
:10F220002D3D6D08976C6491015C63E6F4516B6B46
:10F2300062616C1CD83065854E0062F2ED95066CFB
:10F240007BA5011BC1F4088257C40FF5C6D9B06570
:10F2500050E9B712EAB8BE8B7C88B9FCDF1DDD62CD
:10F26000492DDA15F37CD38C654CD4FB5861B24D33
:10F27000CE51B53A7400BCA3E230BBD441A5DF4AFD
:10F28000D795D83D6DC4D1A4FBF4D6D36AE96943C0
:10F29000FCD96E34468867ADD0B860DA732D04446B
:10F2A000E51D03335F4C0AAAC97C0DDD3C71055096
:10F2B000AA41022710100BBE86200CC925B568573D
:10F2C000B3856F2009D466B99FE461CE0EF9DE5E86
:10F2D00098C9D9292298D0B0B4A8D7C7173DB35937
:10F2E000810DB42E3B5CBDB7AD6CBAC02083B8EDC8
:10F2F000B6B3BF9A0CE2B6039AD2B1743947D5EAD5
:10F30000AF77D29D1526DB048316DC73120B63E303
:10F31000843B64943E6A6D0DA85A6A7A0BCF0EE462
:10F320009DFF099327AE000AB19E077D44930FF01D
:10F33000D2A3088768F2011EFEC206695D5762F714
:10F34000CB67658071366C19E7066B6E761BD4FE51
:10F35000E02BD3895A7ADA10CC4ADD676FDFB9F92E
:10F36000F9EFBE8E43BEB717D58EB060E8A3D6D6F0
:10F370007E93D1A1C4C2D83852F2DF4FF167BBD11E
:10F380006757BCA6DD06B53F4B36B248DA2B0DD821
:10F390004C1B0AAFF64A0336607A0441C3EF60DFC4
:10F3A00055DF67A8EF8E6E3179BE69468CB361CBAD
:10F3B0001A8366BCA0D26F2536E2685295770CCCD2
:10F3C00003470BBBB91602222F260555BE3BBAC513
:10F3D000280BBDB2925AB42B046AB35CA7FFD7C204
:10F3E00031CFD0B58B9ED92C1DAEDE5BB0C2649BF5
:10F3F00026F263EC9CA36A750A936D02A906099C28
:10F400003F360EEB8567077213570005824ABF959A
:10F41000147AB8E2AE2BB17B381BB60C9B8ED2921D
:10F420000DBED5E5B7EFDC7C21DFDB0BD4D2D38674
:10F4300042E2D4F1F8B3DD686E83DA1FCD16BE81E7
:10F440005B26B9F6E177B06F7747B718E65A0888B8
:10F45000706A0FFFCA3B06665C0B0111FF9E658F49
:10F4600069AE62F8D3FF6B6145CF6C1678E20AA0F3
:10F47000EED20DD75483044EC2B30339612667A779
:10F48000F71660D04D476949DB776E3E4A6AD1AEC8
:10F49000DC5AD6D9660BDF40F03BD83753AEBCA957
:10F4A000C59EBBDE7FCFB247E9FFB5301CF2BDBDC4
:10F4B0008AC2BACA3093B353A6A3B4240536D0BACD
:10F4C0009306D7CD2957DE54BF67D9232E7A66B36A
:10F4D000B84A61C4021B685D942B6F2A37BE0BB417
:10F4E000A18E0CC31BDF055A8DEF022D416C6C20E1
:10F4F0007461736B732073746F7070656400763120
:10F50000373500202573202573004D656D6F7279A6
:10F5100020636C6561726564004E6F20667265657C
:10F52000207461736B20656E7472696573000000EE
:10F53000B0F50000F1780000BDF500001572000084
:10F54000C9F50000C1780000CFF50000D1780000B7
:10F55000D5F50000E1780000DBF5000099770000A8
:10F56000F1F50000A97A0000FFF5000049720000E3
:10F5700009F60000357B000011F6000095750000CB
:10F580001AF60000717300002BF6000051740000A1
:10F5900037F600002573000040F60000A573000058
:10F5A00048F600009D74000073656E736F727300FF
:10F5B000616363656C65726174696F6E0074656D1B
:10F5C00070657261747572650074696C745800744A
:10F5D000696C74590074696C745A00736574416382
:10F5E00063656C65726F6D6574657252616E676597
:10F5F000006D61676E657469634669656C6400746B
:10F600006F75636852656164006932635265616455
:10F6100000693263577269746500693263536574B7
:10F62000436C6F636B5370656564007370694578F4
:10F630006368616E67650073706953657475700007
:10F6400072656164444854006D6963726F70686FDD
:10F650006E65000059E30000157C00005EE30000C9
:10F66000C17B00008BF60000597D000081E30000A3
:10F67000DD7B000090F60000E17C000096F60000C3
:10F68000397C000073657269616C007265616400A9
:10F69000777269746500777269746542797465730D
:10F6A0000000000028F70000897D000035F7000009
:10F6B0008D7D00003EF70000997D000048F70000B6
:10F6C0009D7D000051F70000A17D000056F700006D
:10F6D000A57D00005BF70000A97D000067F7000032
:10F6E000AD7D00006EF70000B17D000077F70000EF
:10F6F000B57D00007CF70000B97D000088F70000B0
:10F70000BD7D000093F70000C17D00009EF7000062
:10F71000C57D0000A8F70000917D0000B2F7000051
:10F72000957D0000746674007365744261636B6C50
:10F730006967687400676574576964746800676511
:10F740007448656967687400736574506978656C9E
:10F75000006C696E65007265637400726F756E642B
:10F7600065645265637400636972636C65007472EA
:10F7700069616E676C650074657874006D657267A9
:10F78000654269746D617000647261774275666686
:10F79000657200746674546F75636865640074669E
:10F7A00074546F7563685800746674546F75636839
:10F7B0005900746674546F7563685072657373751D
:10F7C0007265007661727300E8F7000055820000F0
:10F7D000F2F7000035820000FBF700001182000004
:10F7E00007F800009F8100007661724578697374A4
:10F7F00073007661724E616D656400736574566165
:10F80000724E616D6564007661724E616D65466F22
:10F8100072496E6465780057656C636F6D6520741E
:10F820006F204D6963726F426C6F636B7321007060
:10F830005F73706920213D204E554C4C002F686F3E
:10F840006D652F6769742F2E706C6174666F726DB1
:10F85000696F2F7061636B616765732F6672616D8D
:10F8600065776F726B2D61726475696E6F6E6F7202
:10F870006469636E7266352F6C6962726172696564
:10F88000732F5350492F5350492E637070005350BB
:10F8900049436C6173733A3A535049436C617373D3
:10F8A000284E52465F5350495F547970652A2C2088
:10F8B00075696E74385F742C2075696E74385F7466
:10F8C0002C2075696E74385F7429000000000000F8
:10F8D0000000000029840000E58300000B84000084
:10F8E000158400001F84000009840000030000004C
:10F8F00002000000010000000400000005000000FC
:10F90000110000000C0000000B00000012000000BD
:10F910000A000000060000001A00000014000000A9
:10F920001700000016000000150000001000000085
:10F93000FFFFFFFFFFFFFFFF000000001E000000B1
:10F940001900000018000000070000000800000077
:10F95000090000000D0000000E0000000F00000074
:10F960001C0000001B0000001D0000001300000030
:10F970000000000000000000158800004990000011
:10F9800095880000A98800009F8800001188000069
:10F9900005880000B588000031880000018800005B
:10F9A000000000000000304300000000000030C3F1
:10F9B0007371727400000000FB21F93FFB210940C4
:10F9C0007CD91240FB2119407A6A1F407CD9224021
:10F9D000BBFD2540FB2129403A462C407A6A2F4046
:10F9E0005C4731407CD932409C6B3440BBFD354094
:10F9F000DB8F3740FB2139401BB43A403A463C404C
:10FA00005AD83D407A6A3F404C7E40405C47414076
:10FA10006C1042407CD942408CA243409C6B4440D5
:10FA2000AC344540BBFD4540CBC64640DB8F47402C
:10FA3000EB584840FB21494083F9A200444E6E0038
:10FA4000FC291500D1572700DD34F50062DBC0002A
:10FA50003C999500419043006351FE00BBDEAB0032
:10FA6000B761C5003A6E2400D24D42004906E0005D
:10FA700009EA2E001C92D100EB1DFE0029B11C00EA
:10FA8000E83EA700F535820044BB2E009CE98400C7
:10FA9000B4267000417E5F00D6913900538339004F
:10FAA0009CF439008B5F840028F9BD00F81F3B00EF
:10FAB000DEFF97000F980500112FEF000A5A8B0008
:10FAC0006D1F6D00CF7E360009CB2700464FB70073
:10FAD0009E663F002DEA5F00BA277500E5EBC70080
:10FAE0003D7BF100F739070092528A00FB6BEA0078
:10FAF0001FB15F00085D8D00300356007BFC46009F
:10FB0000F0AB6B0020BCCF0036F49A00E3A91D00D7
:10FB10005E619100081BE60085996500A0145F00F6
:10FB20008D40680080D8FF0027734D000606310025
:10FB3000CA561500C9A873007BE260006B8CC00038
:10FB400000000040FB21F93F000000002D44743EFE
:10FB5000000000809846F83C0000006051CC783BE3
:10FB600000000080831BF0390000004020257A3817
:10FB7000000000802282E336000000001DF369359A
:10FB80000200000003000000040000000600000066
:10FB9000D4AC00007EAC00007EAC0000ACAD000038
:10FBA0007AAC00007AAC0000A2AD0000ACAD000061
:10FBB0007AAC0000A2AD00007AAC0000ACAD000051
:10FBC000B0AD0000B0AD0000B0AD0000B8AD0000B9
:10FBD000B0B7000022B6000066B60000CAB500004B
:10FBE00066B6000056B7000066B60000CAB5000051
:10FBF00022B6000022B6000056B70000CAB50000C9
:10FC0000C2B50000C2B50000C2B5000064B7000074
:10FC1000D8BE0000DABD0000DABD0000F8C0000068
:10FC2000D4BD0000D4BD0000E0C00000F8C000005A
:10FC3000D4BD0000E0C00000D4BD0000F8C000004A
:10FC4000EEC00000EEC00000EEC00000FCC00000EE
:10FC50002C2066756E6374696F6E3A200061737351
:10FC6000657274696F6E2022257322206661696C4B
:10FC700065643A2066696C6520222573222C206C0D
:10FC8000696E65202564257325730A0090000020A5
:10FC9000232D302B2000686C4C0065666745464775
:10FCA00000303132333435363738394142434445F8
:10FCB0004600303132333435363738396162636467
:10FCC0006566000000000000000000000000000069
:10FCD0000000000000000000000000000000000024
:10FCE0000000000000000000000000000000000014
:10FCF0000000000000000000000000000000000004
:10FD000000000000000000000000000000000000F3
:10FD100000000000000000000000000000000000E3
:10FD200000000000504F53495800002020202020A0
:10FD3000202020202828282828202020202020209B
:10FD4000202020202020202020202088101010108B
:10FD500010101010101010101010100404040404DF
:10FD6000040404040410101010101010414141410B
:10FD700041410101010101010101010101010101F3
:10FD80000101010101011010101010104242424205
:10FD900042420202020202020202020202020202C3
:10FDA00002020202020210101010200000000000E7
:10FDB0000000000000000000000000000000000043
:10FDC0000000000000000000000000000000000033
:10FDD0000000000000000000000000000000000023
:10FDE0000000000000000000000000000000000013
:10FDF0000000000000000000000000000000000003
:10FE000000000000000000000000000000000000F2
:10FE100000000000000000000000000000000000E2
:10FE200000000000000000000000000000000000D2
:08FE3000D802FF7F0100000071
:10FE3800FFFFFFFFE803000001000000E803DC0506
:10FE4800DC05DC05DC050000FFFFFFFFFFFFFFFF0F
:10FE58001800000019FCFFFFFFFFFFFF0200000071
:10FE680040420F00FFFF01FF0024F40002000000E1
:10FE780003000000FFFFFFFF00000000010000007A
:10FE88000000020001000000FFFFFFFF000000006B
:10FE9800020000000000040002000000FFFFFFFF56
:10FEA800000000000300000000000800030000003C
:10FEB8000A00000008000000010000009000002077
:10FEC80000000000E4FC000004FD0000C4FC000089
:10FED800000000000000000000000000000000001A
:10FEE800000000000000000000000000000000000A
:10FEF80000000000000000000000000000000000FA
:10FF080000000000000000000000000000000000E9
:10FF180000000000000000000000000000000000D9
:10FF28004300000000000000000000000000000086
:10FF380000000000000000000000000000000000B9
:10FF48004300000000000000000000000000000066
:10FF58000000000000000000000000000000000099
:10FF68004300000000000000000000000000000046
:10FF78000000000000000000000000000000000079
:10FF88004300000000000000000000000000000026
:10FF98000000000000000000000000000000000059
:10FFA8004300000000000000000000000000000006
:10FFB8000000000000000000000000000000000039
:10FFC80043000000000000000000000000000000E6
:10FFD8000000000000000000000000000000000019
:10FFE80043000000000000000000000000000000C6
:08FFF800000000000000000001
:020000021000EC
:10000000000000000000000005E000001DDA000014
:10001000000000002AFD000068E20000A0E70000E8
:10002000A0E70000A0E70000A0E70000A0E70000B4
:10003000A0E70000A0E70000A0E70000A0E70000A4
:10004000FFFFFFFFFFFFFFFFFFFFFFFFFFFF0000BE
:100050000100415343494900000000000000000036
:100060000000000000000000000000000000000090
:100070000000415343494900000000000000000017
:100080000000000000000000000000000000000070
:1000900000000000E9000000B583000009870000AF
:0800A000618B0000C1000000AB
:04000003000087A5CD
:00000001FF
